:020000040800F2
:1000000000060020E1010008E3010008E301000808
:10001000E3010008E3010008E3010008E301000830
:10002000E3010008E3010008E30100086D2F000868
:10003000E3010008E3010008E3010008E301000810
:10004000E3010008E3010008E3010008E301000800
:10005000E3010008E3010008153200083D32000802
:10006000653200088D320008B5320008E30100084F
:10007000E3010008E3010008E3010008E3010008D0
:10008000E3010008E3010008E3010008E3010008C0
:10009000E3010008E3010008E3010008DD32000885
:1000A000E3010008E3010008E3010008E3010008A0
:1000B000B1330008E3010008E3010008E301000890
:1000C000E3010008E3010008E3010008E301000880
:1000D000E3010008E3010008E3010008E301000870
:1000E00041330008E3010008E3010008E3010008D0
:1000F000E3010008E3010008E3010008E301000850
:10010000E3010008E3010008E3010008E30100083F
:10011000E3010008E3010008E3010008E30100082F
:10012000E3010008E3010008E3010008E30100081F
:10013000E3010008E3010008E3010008E30100080F
:10014000E3010008E3010008E3010008212700089B
:10015000E3010008E3010008E3010008E3010008EF
:10016000E3010008E3010008E3010008E3010008DF
:10017000E3010008E3010008E3010008E3010008CF
:10018000E3010008E3010008E3010008E3010008BF
:10019000E3010008E3010008E3010008E3010008AF
:1001A000E3010008E3010008E3010008E30100089F
:1001B000E3010008E3010008E3010008E30100088F
:1001C000E3010008E3010008E3010008E30100087F
:1001D000E3010008E3010008E3010008E30100086F
:1001E00002E000F000F8FEE772B6374880F30888B6
:1001F000364880F3098836483649086040F20000E6
:10020000CCF200004EF63471CEF200010860BFF36C
:100210004F8FBFF36F8F40F20000C0F2F0004EF638
:100220008851CEF200010860BFF34F8FBFF36F8F8C
:100230004FF00000E1EE100A4EF63C71CEF20001E4
:100240000860062080F31488BFF36F8F01F030FF41
:1002500002F02AFE4FF055301F491B4A91423CBF25
:1002600041F8040BFAE71D49184A91423CBF41F896
:10027000040BFAE71A491B4A1B4B9A423EBF51F83E
:10028000040B42F8040BF8E700201849184A914281
:100290003CBF41F8040BFAE701F00EFF02F058FEF4
:1002A000144C154DAC4203DA54F8041B8847F9E7A7
:1002B00000F042F8114C124DAC4203DA54F8041B22
:1002C0008847F9E701F0F6BE000600200022002072
:1002D0000000000808ED00E00000002000060020FB
:1002E0007837000800220020402200204022002011
:1002F000602E0020E0010008E0010008E001000895
:10030000E00100082DE9F04F2DED108AC1F80CD066
:10031000C3689D46BDEC108ABDE8F08F002383F3CF
:1003200011882846A047002001F072FAFEE701F08C
:1003300001FA00DFFEE7000038B500F0BBFB01F07A
:1003400087FE054601F0AAFE0446C8B90E4B9D4241
:1003500018D001339D4218BF044641F2883504BFCE
:1003600001240025002001F07DFE0CB100F074F89E
:1003700000F000FD284600F0BFF800F06DF8F9E746
:100380000025EFE70546EDE7010007B008B500F0EE
:1003900063FBA0F120035842584108BD07B541F264
:1003A0001203022101A8ADF8043000F073FB03B082
:1003B0005DF804FB38B5302383F3118817480368D0
:1003C0000BB101F0F1FA164A144800234FF47A7188
:1003D00001F0E0FA002383F31188124C236813B173
:1003E0002368013B2360636813B16368013B63606A
:1003F0000D4D2B7833B963687BB9022000F024FCE3
:10040000322363602B78032B07D163682BB902205A
:1004100000F01AFC4FF47A73636038BD402200206C
:10042000B50300086023002058220020084B1870F4
:1004300003280CD8DFE800F008050208022000F0CD
:10044000F9BB022000F0ECBB024B00225A6070475F
:100450005822002060230020234B244A10B51C465C
:10046000196801313FD004339342F9D16268A24246
:1004700039D31F4B9B6803F1006303F540439A4255
:1004800031D2002000F030FB0220FFF7CFFF194BE4
:100490001A6C00221A64196E1A66196E596C5A6425
:1004A000596E5A665A6E5A6942F080025A615A6908
:1004B00022F080025A615A691A6942F000521A61A8
:1004C0001A6922F000521A611B6972B64FF0E023DC
:1004D0003021C3F8084DD4E9003281F311889D46DC
:1004E00083F30888104710BD00C0000820C0000832
:1004F00000220020003802402DE9F04F93B0AA4BB3
:1005000000902022FF210AA89D6800F0DDFBA74A89
:100510001378A3B9A648012103601170302383F337
:10052000118803680BB101F03FFAA24AA0480023EA
:100530004FF47A7101F02EFA002383F31188009BA7
:1005400013B19D4B009A1A609C4A009C1378032BB0
:100550001EBF00231370984A4FF0000A18BF536063
:10056000D3465646D146012000F064FB24B1924B9D
:100570001B68002B00F01182002000F06DFA039040
:10058000039B002BF2DB012000F04AFB039B213B85
:10059000162BE8D801A252F823F000BFF905000895
:1005A00021060008B5060008670500086705000871
:1005B000670500083F0700080F0900082908000820
:1005C0008B080008B3080008D90800086705000870
:1005D000EB080008670500085D0900089906000897
:1005E00067050008A109000805060008990600082B
:1005F000670500088B0800080220FFF7C7FE0028E7
:1006000040F0F581009B0221BAF1000F08BF1C46A3
:1006100005A841F21233ADF8143000F03BFAA2E71E
:100620004FF47A7000F018FA071EEBDB0220FFF798
:10063000ADFE0028E6D0013F052F00F2DA81DFE8A9
:1006400007F0030A0D10133605230593042105A8AE
:1006500000F020FA17E054480421F9E75848042133
:10066000F6E758480421F3E74FF01C08404600F035
:100670003DFA08F104080590042105A800F00AFAE3
:10068000B8F12C0FF2D1012000FA07F747EA0B0B63
:100690005FFA8BFB4FF0000900F062FB26B10BF014
:1006A0000B030B2B08BF0024FFF778FE5BE74648DF
:1006B0000421CDE7002EA5D00BF00B030B2BA1D10D
:1006C0000220FFF763FE074600289BD0012000F0C0
:1006D0000BFA0220FFF7AAFE00261FFA86F8404612
:1006E00000F012FA044690B10021404600F01CFAD6
:1006F00001360028F1D1BA46044641F21213022114
:1007000005A8ADF814303E4600F0C4F92BE70120EF
:10071000FFF78CFE2546244B9B68AB4207D9284641
:1007200000F0E4F9013040F067810435F3E7234B32
:1007300000251D70204BBA465D603E46ACE7002E9A
:100740003FF460AF0BF00B030B2B7FF45BAF022089
:10075000FFF76CFE322000F07FF9B0F10008FFF6E1
:1007600051AF18F003077FF44DAF0F4A926808EBC2
:10077000050393423FF646AFB8F5807F3FF742AF9F
:10078000124B0193B84523DD4FF47A7000F064F901
:100790000390039A002AFFF635AF019B039A03F8F2
:1007A000012B0137EDE700BF002200205C23002071
:1007B00040220020B50300086023002058220020BA
:1007C00004220020082200200C2200205C220020AD
:1007D000C820FFF7DBFD074600283FF413AF1F2DAD
:1007E00011D8C5F1200242450AAB25F0030028BF0D
:1007F000424683490192184400F040FA019A804829
:10080000FF2100F061FA4FEAA8037D490193C8F384
:100810008702284600F060FA064600283FF46DAFD4
:10082000019B05EB830537E70220FFF7AFFD0028AA
:100830003FF4E8AE00F0A4F900283FF4E3AE00274F
:10084000B846704B9B68BB4218D91F2F11D80A9B22
:1008500001330ED027F0030312AA134453F8203CAF
:1008600005934046042205A900F0AEFA04378046FD
:10087000E7E7384600F03AF90590F2E7CDF8148042
:10088000042105A800F006F906E70023642104A866
:10089000049300F0F5F800287FF4B4AE0220FFF7CF
:1008A00075FD00283FF4AEAE049800F051F90590B4
:1008B000E6E70023642104A8049300F0E1F800288F
:1008C0007FF4A0AE0220FFF761FD00283FF49AAE4E
:1008D000049800F04DF9EAE70220FFF757FD0028E1
:1008E0003FF490AE00F05CF9E1E70220FFF74EFD27
:1008F00000283FF487AE05A9142000F057F9042121
:100900000746049004A800F0C5F83946B9E732203C
:1009100000F0A2F8071EFFF675AEBB077FF472AEBB
:10092000384A926807EB090393423FF66BAE022008
:10093000FFF72CFD00283FF465AE27F003074F4476
:10094000B9453FF4A9AE484600F0D0F8042105901F
:1009500005A800F09FF809F10409F1E74FF47A7057
:10096000FFF714FD00283FF44DAE00F009F9002810
:1009700044D00A9B01330BD008220AA9002000F0C2
:10098000ABF900283AD02022FF210AA800F09CF9F8
:10099000FFF704FD1C4800F041FF13B0BDE8F08FE5
:1009A000002E3FF42FAE0BF00B030B2B7FF42AAE7F
:1009B0000023642105A8059300F062F8074600288B
:1009C0007FF420AE0220FFF7E1FC804600283FF4D0
:1009D00019AEFFF7E3FC41F2883000F01FFF0598E5
:1009E00000F0F0F9464600F0BBF93C46BBE5064690
:1009F00052E64FF0000905E6BA467EE637467CE649
:100A00005C22002000220020A086010070B50F4B60
:100A10001B780133DBB2012B0C4611D80C4D296831
:100A20004FF47A730E6AA2FB03320146224628462F
:100A3000B047844204D1074B00221A70012070BDD8
:100A40004FF4FA7000F0EAFE0020F8E710220020D0
:100A5000082600209423002007B500230246012128
:100A60000DF107008DF80730FFF7D0FF20B19DF89A
:100A7000070003B05DF804FB4FF0FF30F9E700001A
:100A80000A4608B50421FFF7C1FF80F00100C0B29B
:100A9000404208BD30B4054C2368DD69044B0A466A
:100AA000AC460146204630BC604700BF0826002007
:100AB000A086010070B501F0D1F9094E094D3080D2
:100AC000002428683388834208D901F0C1F92B68D3
:100AD00004440133B4F5404F2B60F2D370BD00BF26
:100AE000962300206823002001F066BA00F1006020
:100AF00000F540400068704700F10060920000F58A
:100B0000404001F0F1B90000054B1A68054B1B8805
:100B10009B1A834202D9104401F09AB90020704711
:100B2000682300209623002038B5084D044629B1DB
:100B300028682044BDE8384001F0AAB9286820445C
:100B400001F08EF90028F3D038BD00BF68230020E3
:100B500010F003030AD1B0F5047F05D200F1005074
:100B6000A0F51040D0F80038184670470023FBE786
:100B700000F10050A0F51040D0F8100A70470000B6
:100B8000064991F8243033B10023086A81F82430F3
:100B90000822FFF7B1BF0120704700BF6C2300207F
:100BA000014B1868704700BF002004E070B5194B76
:100BB0001D68194B0138C5F30B0408442D0C0422A1
:100BC0001E88A6420BD15C680A46013C824213464D
:100BD0000FD214F9016F4EB102F8016BF6E7013A3A
:100BE00003F10803ECD181420B4602D22C2203F818
:100BF000012B0A4A05241688AE4204D1984284BFCC
:100C0000967803F8016B013C02F10402F3D1581A03
:100C100070BD00BF002004E0943400088034000858
:100C2000022802BF024B4FF480429A61704700BF16
:100C300000080240022802BF024B4FF080429A6136
:100C4000704700BF00080240022801BF024A5369F2
:100C500083F48043536170470008024070B5044636
:100C60004FF47A764CB1412C254628BF412506FB2E
:100C700005F000F0D3FD641BF4E770BD10B5002350
:100C8000934203D0CC5CC4540133F9E710BD00009B
:100C900010B5013810F9013F3BB191F900409C4279
:100CA00003D11AB10131013AF4E71AB191F90020E8
:100CB000981A10BD1046FCE703460246D01A12F9F6
:100CC000011B0029FAD1704702440346934202D027
:100CD00003F8011BFAE770472DE9F8431F4D14464E
:100CE00095F824200746884652BBDFF870909CB3E5
:100CF00095F824302BB92022FF2148462F62FFF7B8
:100D0000E3FF95F82400C0F10802A24228BF224662
:100D1000D6B24146920005EB8000FFF7AFFF95F891
:100D20002430A41B1E44F6B2082E17449044E4B2AB
:100D300085F82460DBD1FFF723FF0028D7D108E036
:100D40002B6A03EB82038342CFD0FFF719FF002801
:100D5000CBD10020BDE8F8830120FBE76C23002005
:100D6000024B1A78024B1A70704700BF9423002080
:100D70001022002010B5104C104800F0B5F82146A4
:100D80000E4800F0DDF82468626DD2F8043843F0B4
:100D90000203C2F804384FF47A70FFF75FFF084986
:100DA000204600F0D3F9626DD2F8043823F0020334
:100DB000C2F8043810BD00BF6035000808260020C6
:100DC000683500087047000030B5094D0A4491426B
:100DD0000DD011F8013B5840082340F30004013BBB
:100DE0002C4013F0FF0384EA5000F6D1EFE730BD4A
:100DF0002083B8ED026843681143016003B11847CE
:100E00007047000013B5446BD4F894341A68117815
:100E1000042915D1217C022912D1197912890123C3
:100E20008B4013420CD101A904F14C0001F0F8FEF3
:100E3000D4F89444019B21790246206800F0D0F94F
:100E400002B010BD143001F07BBE00004FF0FF3344
:100E5000143001F075BE00004C3001F04DBF0000B1
:100E60004FF0FF334C3001F047BF0000143001F069
:100E700049BE00004FF0FF31143001F043BE0000C6
:100E80004C3001F019BF00004FF0FF324C3001F040
:100E900013BF00000020704710B5D0F894341A68D2
:100EA00011780429044617D1017C022914D15979FB
:100EB000528901238B4013420ED1143001F0DCFD26
:100EC000024648B1D4F894444FF4807361792068A5
:100ED000BDE8104000F072B910BD0000406BFFF794
:100EE000DBBF0000704700007FB5124B036000239A
:100EF0004360C0E90233012502260F4B0574044606
:100F00000290019300F18402294600964FF4807309
:100F1000143001F08DFD094B0294CDE9006304F516
:100F200023724FF48073294604F14C0001F054FE03
:100F300004B070BDB4340008DD0E0008050E0008D2
:100F40000B68302282F311880A7903EB82029061E8
:100F50004A79093243F822008A7912B103EB8203FD
:100F600098610223C0F894140374002080F3118860
:100F70007047000038B5037F044613B190F8543031
:100F8000ABB9201D01250221FFF734FF04F1140045
:100F900025776FF0010100F069FC84F8545004F1EA
:100FA0004C006FF00101BDE8384000F05FBC38BD77
:100FB00010B5012104460430FFF71CFF00232377FE
:100FC00084F8543010BD000038B5044600251430B4
:100FD00001F046FD04F14C00257701F015FE201DBF
:100FE00084F854500121FFF705FF2046BDE8384042
:100FF000FFF752BF90F8443003F06003202B07D175
:1010000090F84520212A4FF0000303D81F2A06D864
:1010100000207047222AFBD1C0E90E3303E0034AC7
:1010200082630722C26303640120704711220020FB
:1010300037B5D0F894341A681178042904461AD1C7
:10104000017C022917D11979128901238B4013429F
:1010500011D100F14C05284601F096FE58B101A9C6
:10106000284601F0DDFDD4F89444019B2179024625
:10107000206800F0B5F803B030BD0000F0B500EB1B
:10108000810385B09E6904460D46FEB1302383F38B
:10109000118804EB8507301D0821FFF7ABFEFB68C4
:1010A0005B691B6806F14C001BB1019001F0C6FDA5
:1010B000019803A901F0B4FD024648B1039B2946FB
:1010C000204600F08DF8002383F3118805B0F0BDB1
:1010D000FB685A691268002AF5D01B8A013B13404D
:1010E000F1D104F14402EAE7093138B550F8214062
:1010F000DCB1302383F31188D4F894241368527937
:1011000003EB8203DB689B695D6845B104216018CD
:10111000FFF770FE294604F1140001F0B7FC2046E9
:10112000FFF7BAFE002383F3118838BD7047000033
:1011300001F016B8012303700023C0E90133C36135
:1011400083620362C36243620363704738B5044637
:10115000302383F311880025C0E90355C0E9055504
:10116000416001F00DF80223237085F311882846B1
:1011700038BD000070B500EB810305465069DA60A8
:101180000E46144618B110220021FFF79DFDA069FC
:1011900018B110220021FFF797FD31462846BDE81F
:1011A000704001F0B7B80000826802F0011282605E
:1011B0000022C0E90422826101F038B9F0B400EBEA
:1011C00081044789E4680125A4698D403D43458138
:1011D00023600023A2606360F0BC01F053B90000FB
:1011E000F0B400EB81040789E468012564698D404F
:1011F0003D43058123600023A2606360F0BC01F0E1
:10120000CDB9000070B50223002504460370C0E983
:101210000255C0E90455C564856180F8345001F079
:1012200015F863681B6823B129462046BDE8704065
:10123000184770BD0378052B10B504460AD080F816
:1012400050300523037043681B680BB10421984795
:101250000023A36010BD00000178052906D190F895
:101260005020436802701B6803B1184770470000A4
:1012700070B590F83430044613B1002380F8343050
:1012800004F14402204601F0F3F863689B68B3B9A7
:1012900094F8443013F0600535D00021204601F069
:1012A00093FB0021204601F085FB63681B6813B1A6
:1012B000062120469847062384F8343070BD204626
:1012C00098470028E4D0B4F84A30E26B9A4288BFCD
:1012D000E36394F94430E56B002B4FF0300380F268
:1012E0000381002D00F0F280092284F8342083F37A
:1012F00011880021D4E90E232046FFF771FF002357
:1013000083F31188DAE794F8452003F07F0343EA7A
:10131000022340F20232934200F0C58021D8B3F597
:10132000807F48D00DD8012B3FD0022B00F0938056
:10133000002BB2D104F14C02A2630222E2632364C7
:10134000C1E7B3F5817F00F09B80B3F5407FA4D166
:1013500094F84630012BA0D1B4F84C3043F002038E
:1013600032E0B3F5006F4DD017D8B3F5A06F31D090
:10137000A3F5C063012B90D8636894F846205E689B
:1013800094F84710B4F848302046B047002884D07D
:101390004368A3630368E3631AE0B3F5106F36D0C4
:1013A00040F6024293427FF478AF5C4BA363022382
:1013B000E3630023C3E794F84630012B7FF46DAF5D
:1013C000B4F84C3023F00203C4E90E55A4F84C30B5
:1013D000256478E7B4F84430B3F5A06F0ED194F8E3
:1013E000463084F84E30204600F088FF63681B6862
:1013F00013B1012120469847032323700023C4E939
:101400000E339CE704F14F03A3630123C3E7237862
:10141000042B10D1302383F311882046FFF7C4FE3C
:1014200085F311880321636884F84F5021701B688D
:101430000BB12046984794F84630002BDED084F854
:101440004F300423237063681B68002BD6D0022121
:1014500020469847D2E794F848301D0603F00F0164
:1014600020460AD500F0F6FF012804D002287FF4B8
:1014700014AF2B4B9AE72B4B98E700F0DDFFF3E717
:1014800094F84630002B7FF408AF94F8483013F0FE
:101490000F01B3D01A06204602D501F0A9FAADE734
:1014A00001F09CFAAAE794F84630002B7FF4F5AEE1
:1014B00094F8483013F00F01A0D01B06204602D547
:1014C00001F082FA9AE701F075FA97E7142284F89E
:1014D000342083F311882B462A4629462046FFF7FD
:1014E0006DFE85F31188E9E65DB1152284F834209C
:1014F00083F311880021D4E90E232046FFF75EFE16
:10150000FDE60B2284F8342083F311882B462A460B
:1015100029462046FFF764FEE3E700BFE4340008F5
:10152000DC340008E034000838B590F83430044664
:10153000002B3ED0063BDAB20F2A34D80F2B32D81C
:10154000DFE803F0373131082232313131313131C6
:1015500031313737C56BB0F84A309D4214D2C36879
:101560001B8AB5FBF3F203FB12556DB9302383F3ED
:1015700011882B462A462946FFF732FE85F311884B
:101580000A2384F834300EE0142384F834303023F6
:1015900083F3118800231A4619462046FFF70EFEF2
:1015A000002383F3118838BD036C03B198470023EF
:1015B000E7E70021204601F007FA0021204601F06C
:1015C000F9F963681B6813B1062120469847062382
:1015D000D7E7000010B590F83430142B044629D01A
:1015E00017D8062B05D001D81BB110BD093B022B23
:1015F000FBD80021204601F0E7F90021204601F048
:10160000D9F963681B6813B1062120469847062361
:1016100019E0152BE9D10B2380F83430302383F304
:10162000118800231A461946FFF7DAFD002383F3D9
:101630001188DAE7C3689B695B68002BD5D1036C1E
:1016400003B19847002384F83430CEE700230375B4
:10165000826803691B6899689142FBD25A680360EB
:101660004260106058607047002303758268036908
:101670001B6899689142FBD85A6803604260106009
:101680005860704708B50846302383F311880B7DF6
:10169000032B05D0042B0DD02BB983F3118808BD83
:1016A0008B6900221A604FF0FF338361FFF7CEFF92
:1016B0000023F2E7D1E9003213605A60F3E700003B
:1016C000FFF7C4BF054BD9680875186802681A602F
:1016D000536001220275D860FEF714BE98230020E3
:1016E00030B50C4BDD684B1C87B004460FD02B4641
:1016F000094A684600F04EF92046FFF7E3FF009BD9
:1017000013B1684600F050F9A86907B030BDFFF783
:10171000D9FFF9E79823002085160008044B1A68C2
:10172000DB6890689B68984294BF00200120704756
:1017300098230020084B10B51C68D86822681A60EE
:10174000536001222275DC60FFF78EFF01462046C0
:10175000BDE81040FEF7D6BD9823002038B5074CF1
:1017600007490848012300252370656001F044FB08
:101770000223237085F3118838BD00BF00260020A6
:10178000EC3400089823002000F044B9034A516863
:1017900053685B1A9842FBD8704700BF001000E006
:1017A0008B60022308618B82084670478368A3F12F
:1017B000840243F8142C026943F8442C426943F82C
:1017C000402C094A43F8242CC26843F8182C022202
:1017D00003F80C2C002203F80B2C044A43F8102CBD
:1017E000A3F12000704700BF1D03000898230020CC
:1017F00008B5FFF7DBFFBDE80840FFF761BF000059
:10180000024BDB6898610F20FFF75CBF9823002034
:10181000302383F31188FFF7F3BF000008B50146BA
:10182000302383F311880820FFF75AFF002383F346
:10183000118808BD064BDB6839B1426818605A60F0
:10184000136043600420FFF74BBF4FF0FF30704739
:10185000982300200368984206D01A6802605060FE
:1018600099611846FFF72CBF7047000038B5044651
:101870000D462068844200D138BD036823605C6057
:101880008561FFF71DFFF4E710B503689C68A2426D
:101890000CD85C688A600B604C6021605960996864
:1018A0008A1A9A604FF0FF33836010BD1B68121BC9
:1018B000ECE700000A2938BF0A2170B504460D463E
:1018C0000A26601901F092FA01F07EFA041BA54283
:1018D00003D8751C2E460446F3E70A2E04D9BDE84A
:1018E0007040012001F0C8BA70BD0000F8B5144B7B
:1018F0000D46D96103F1100141600A2A196982601D
:1019000038BF0A22016048601861A818144601F027
:101910005FFA0A2701F058FA431BA342064606D392
:101920007C1C281901F062FA27463546F2E70A2F97
:1019300004D9BDE8F840012001F09EBAF8BD00BF0F
:1019400098230020F8B506460D4601F03DFA0F4AEF
:10195000134653F8107F9F4206D12A46014630466F
:10196000BDE8F840FFF7C2BFD169BB68441A2C1923
:1019700028BF2C46A34202D92946FFF79BFF2246E7
:1019800031460348BDE8F840FFF77EBF98230020AA
:10199000A823002010B4C0E9032300235DF8044B02
:1019A0004361FFF7CFBF000010B5194C236998427F
:1019B0000DD0D0E90032816813605A609A680A44F9
:1019C0009A60002303604FF0FF33A36110BD2346EC
:1019D000026843F8102F53600022026022699A4285
:1019E00003D1BDE8104001F0FBB9936881680B4456
:1019F000936001F0E9F92269E1699268441AA24210
:101A0000E4D91144BDE81040091AFFF753BF00BFE5
:101A1000982300202DE9F047DFF8BC8008F110077B
:101A20002C4ED8F8105001F0CFF9D8F81C40AA6815
:101A3000031B9A423ED81444D5E900324FF0000906
:101A4000C8F81C4013605A60C5F80090D8F81030F0
:101A5000B34201D101F0C4F989F31188D5E903310A
:101A600028469847302383F311886B69002BD8D020
:101A700001F0AAF96A69A0EB04094A4582460DD231
:101A8000022001F0F9F90022D8F81030B34208D151
:101A900051462846BDE8F047FFF728BF121A2244F6
:101AA000F2E712EB090938BF4A4629463846FFF7E4
:101AB000EBFEB5E7D8F81030B34208D01444211A31
:101AC000C8F81C00A960BDE8F047FFF7F3BEBDE809
:101AD000F08700BFA8230020982300200020704733
:101AE000FEE70000704700004FF0FF307047000035
:101AF00002290CD0032904D00129074818BF00206F
:101B00007047032A05D8054800EBC2007047044817
:101B100070470020704700BFC43500082022002015
:101B20007835000870B59AB00546084601A91446F4
:101B300000F0C2F801A8FFF7BFF8431C5B00C5E93D
:101B400000340022237003236370C6B201AB023459
:101B50001046D1B28E4204F1020401D81AB070BD11
:101B600013F8011B04F8021C04F8010C0132F0E721
:101B700008B5302383F311880348FFF759FA00238F
:101B800083F3118808BD00BF0826002090F8443078
:101B900003F01F02012A07D190F845200B2A03D138
:101BA0000023C0E90E3315E003F06003202B08D1B9
:101BB000B0F848302BB990F84520212A03D81F2AC5
:101BC00004D8FFF717BA222AEBD0FAE7034A826358
:101BD0000722C26303640120704700BF182200205F
:101BE00007B5052917D8DFE801F0191603191920E0
:101BF000302383F31188104A01900121FFF7BAFACC
:101C000001980E4A0221FFF7B5FA0D48FFF7DCF9FB
:101C1000002383F3118803B05DF804FB302383F3C2
:101C200011880748FFF7A6F9F2E7302383F31188FC
:101C30000348FFF7BDF9EBE7183500083C3500080D
:101C40000826002038B50C4D0C4C0D492A4604F1ED
:101C50000800FFF767FF05F1CA0204F11000094907
:101C6000FFF760FF05F5CA7204F118000649BDE8E8
:101C70003840FFF757BF00BFD02A002020220020A5
:101C8000F8340008023500080D35000870B5044628
:101C900008460D46FFF710F8C6B220460134037817
:101CA0000BB9184670BD32462946FEF7F1FF0028F1
:101CB000F3D10120F6E700002DE9F04705460C4678
:101CC000FEF7FAFF2B49C6B22846FFF7DFFF08B13F
:101CD0000636F6B228492846FFF7D8FF08B1103675
:101CE000F6B2632E0BD8DFF88C80DFF88C90234F90
:101CF000DFF894A02E7846B92670BDE8F087294613
:101D00002046BDE8F04701F09DBB252E2ED10722CD
:101D100041462846FEF7BCFF70B9194B224603F135
:101D20000C0153F8040B42F8040B8B42F9D11B78D9
:101D3000137007350D34DDE7082249462846FEF7C3
:101D4000A7FF98B90F4BA21C197809090232C95D87
:101D500002F8041C13F8011B01F00F015345C95D83
:101D600002F8031CF0D118340835C3E704F8016BFE
:101D70000135BFE7E43500080D350008FA350008E5
:101D8000EC350008107AFF1F1C7AFF1FBFF34F8F3E
:101D9000024AD368DB03FCD4704700BF003C02401A
:101DA00008B5094B1B7873B9FFF7F0FF074B1A69A9
:101DB000002ABFBF064A5A6002F188325A601A6888
:101DC00022F480621A6008BD2E2D0020003C0240E3
:101DD0002301674508B50B4B1B7893B9FFF7D6FF76
:101DE000094B1A6942F000421A611A6842F48052A3
:101DF0001A601A6822F480521A601A6842F48062EB
:101E00001A6008BD2E2D0020003C02400B28F0B5C2
:101E100016D80C4C0C4923787BB90C4D0E460C237C
:101E20004FF0006255F8047B46F8042B013B13F099
:101E3000FF033A44F6D10123237051F82000F0BD8E
:101E40000020FCE7602D0020302D00200C3600081B
:101E5000014B53F8200070470C3600080C207047E7
:101E60000B2810B5044601D9002010BDFFF7CEFFA6
:101E7000064B53F824301844C21A0BB90120F4E77A
:101E800012680132F0D1043BF6E700BF0C360008BF
:101E90000B2810B5044621D8FFF778FFFFF780FF25
:101EA0000F4AF323D360C300DBB243F4007343F063
:101EB00002031361136943F480331361FFF766FF74
:101EC000FFF7A4FF074B53F8241000F0D9F8FFF7F1
:101ED00081FF2046BDE81040FFF7C2BF002010BDC3
:101EE000003C02400C360008F8B512F0010314461D
:101EF00042D18218B2F1016F57D82D4B1B6813F0F5
:101F0000010352D02B4DFFF74BFFF323EB60FFF79C
:101F10003DFF40F20127032C15D824F00104661878
:101F2000244C401A40F20117B142236900EB01052D
:101F300024D123F001032361FFF74CFF0120F8BDFA
:101F4000043C0430E7E78307E7D12B6923F44073AF
:101F50002B612B693B432B6151F8046B0660BFF387
:101F60004F8FFFF713FF03689E42E9D02B6923F0E0
:101F700001032B61FFF72EFF0020E0E723F44073FD
:101F8000236123693B4323610B882B80BFF34F8F71
:101F9000FFF7FCFE2D8831F8023BADB2AB42C3D057
:101FA000236923F001032361E4E71846C7E700BF74
:101FB00000380240003C0240084908B50B7828B1BF
:101FC0001BB9FFF7EDFE01230B7008BD002BFCD001
:101FD000BDE808400870FFF7FDBE00BF2E2D0020B1
:101FE00010B50244064BD2B2904200D110BD441C41
:101FF00000B253F8200041F8040BE0B2F4E700BF50
:10200000502800400F4B30B51C6F240407D41C6FC0
:1020100044F400741C671C6F44F400441C670A4CB1
:10202000236843F4807323600244084BD2B2904289
:1020300000D130BD441C00B251F8045B43F820507D
:10204000E0B2F4E700380240007000405028004041
:1020500007B5012201A90020FFF7C2FF019803B0D4
:102060005DF804FB13B50446FFF7F2FFA04205D06C
:10207000012201A900200194FFF7C4FF02B010BDA6
:1020800070470000034B1A681AB9034AD2F8742843
:102090001A607047642D00200030024008B5FFF739
:1020A000F1FF024B1868C0F3407008BD642D00209A
:1020B00070470000FEE700000A4B0B480B4A9042B5
:1020C0000BD30B4BDA1C121AC11E22F003028B42F7
:1020D00038BF00220021FEF7F7BD53F8041B40F87B
:1020E000041BECE7B8370008602E0020602E0020AB
:1020F000602E002070B5D0E915439E6800224FF095
:10210000FF3504EB42135101D3F800090028BEBF8C
:10211000D3F8000940F08040C3F80009D3F8000B61
:102120000028BEBFD3F8000B40F08040C3F8000B7E
:10213000013263189642C3F80859C3F8085BE0D22D
:102140004FF00113C4F81C3870BD0000890141F044
:102150002001016103699B06FCD41220FFF716BB26
:1021600010B5054C2046FEF7E5FF4FF0A043636530
:10217000024BA36510BD00BF682D0020603600082B
:1021800070B50378012B054650D12A4B446D984217
:102190001BD1294B5A6B42F080025A635A6D42F0B0
:1021A00080025A655A6D5A6942F080025A615A6932
:1021B00022F080025A610E2143205B6900F022FC6C
:1021C0001E4BE3601E4BC4F800380023C4F8003EE9
:1021D000C02323606E6D4FF40413A3633369002B97
:1021E000FCDA012333610C20FFF7D0FA3369DB07F7
:1021F000FCD41220FFF7CAFA3369002BFCDA002660
:10220000A6602846FFF776FF6B68C4F81068DB68A5
:10221000C4F81468C4F81C684BB90A4BA3614FF0AA
:10222000FF336361A36843F00103A36070BD064BF5
:10223000F4E700BF682D0020003802404014004041
:1022400003002002003C30C0083C30C0F8B5446DAB
:10225000054600212046FFF779FFA96D00234FF0C6
:1022600001128F68C4F834384FF00066C4F81C2897
:102270004FF0FF3004EB431201339F42C2F8006974
:10228000C2F8006BC2F80809C2F8080BF2D20B685A
:102290006A6DEB65636210231361166916F0100610
:1022A000FBD11220FFF772FAD4F8003823F4FE6352
:1022B000C4F80038A36943F4402343F01003A3613A
:1022C0000923C4F81038C4F814380A4BEB604FF0F7
:1022D000C043C4F8103B084BC4F8003BC4F8106975
:1022E000C4F80039EB6D03F1100243F48013EA6582
:1022F000A362F8BD3C36000840800010426D90F8A3
:102300004E10D2F8003823F4FE6343EA0113C2F8FA
:10231000003870472DE9F84300EB8103456DDA681A
:10232000166806F00306731E022B05EB41130C46DC
:1023300080460FFA81F94FEA41104FF00001C3F8CF
:10234000101B4FF0010104F1100398BFB60401FA0D
:1023500003F391698EBF334E06F1805606F50046B1
:1023600000293AD0578A04F15801490137436F5088
:10237000D5F81C180B43C5F81C382B180021C3F8DE
:10238000101953690127611EA7409BB3138A928BD2
:102390009B08012A88BF5343D8F85C20981842EA6A
:1023A000034301F1400205EB8202C8F85C002146BC
:1023B00053602846FFF7CAFE08EB8900C3681B8AF2
:1023C00043EA8453483464011E432E51D5F81C3827
:1023D0001F43C5F81C78BDE8F88305EB4917D7F80B
:1023E000001B21F40041C7F8001BD5F81C1821EA96
:1023F0000303C0E704F13F0305EB83030A4A5A6075
:1024000028462146FFF7A2FE05EB4910D0F8003917
:1024100023F40043C0F80039D5F81C3823EA070735
:10242000D7E700BF0080001000040002826D126830
:10243000C265FFF75FBE00005831436D49015B582C
:1024400013F4004004D013F4001F0CBF022001203D
:10245000704700004831436D49015B5813F4004058
:1024600004D013F4001F0CBF0220012070470000AD
:1024700000EB8101CB68196A0B6813604B685360ED
:102480007047000000EB810330B5DD68AA6913686E
:10249000D36019B9402B84BF402313606B8A146842
:1024A000426D1C44013CB4FBF3F46343033323F05B
:1024B000030302EB411043EAC44343F0C043C0F8B6
:1024C000103B2B6803F00303012B09B20ED1D2F8A5
:1024D000083802EB411013F4807FD0F8003B14BFA2
:1024E00043F0805343F00053C0F8003B02EB41122D
:1024F000D2F8003B43F00443C2F8003B30BD00007B
:102500002DE9F041244D6E6D06EB40130446D3F8DF
:10251000087BC3F8087B38070AD5D6F814381907A2
:1025200006D505EB84032146DB6828465B6898479F
:10253000FA071FD5D6F81438DB071BD505EB840343
:10254000D968CCB98B69488A5A68B2FBF0F600FBAF
:1025500016228AB91868DA6890420DD2121AC3E9B5
:102560000024302383F311880B482146FFF78AFFAC
:1025700084F31188BDE8F081012303FA04F26B892A
:1025800023EA02036B81CB68002BF3D0214602487B
:10259000BDE8F041184700BF682D002000EB810323
:1025A00070B5DD68436D6C692668E6604A0156BB0C
:1025B0001A444FF40020C2F810092A6802F00302FE
:1025C000012A0AB20ED1D3F8080803EB421410F422
:1025D000807FD4F8000914BF40F0805040F00050D4
:1025E000C4F8000903EB4212D2F8000940F004409D
:1025F000C2F80009D3F83408012202FA01F10143BC
:10260000C3F8341870BD19B9402E84BF4020206033
:1026100020682E8A8419013CB4FBF6F440EAC440D9
:1026200040F000501A44C6E72DE9F8433B4D6E6D6B
:1026300006EB40130446D3F80889C3F8088918F05C
:10264000010F4FEA40171AD0D6F81038DB0716D51D
:1026500005EB8003D9684B691868DA68904230D27C
:10266000121A4FF000091A60C3F80490302383F364
:10267000118821462846FFF791FF89F3118818F049
:10268000800F1CD0D6F834380126A640334216D02D
:1026900005EB84036D6DD3F80CC0DCF81420013415
:1026A000E4B2D2F800E005EB04342F4451687145E0
:1026B00015D3D5F8343823EA0606C5F83468BDE8E2
:1026C000F883012303FA04F22B8923EA02032B8106
:1026D0008B68002BD3D0214628469847CFE7BCF81B
:1026E0001000AEEB0103834228BF0346D7F8180958
:1026F00080B2B3EB800FE2D89068A0F1040959F8DA
:10270000048FC4F80080A0EB09089844B8F1040FC6
:10271000F5D818440B4490605360C7E7682D00203B
:102720002DE9F74FA24C656D6E69AB691E4016F43A
:1027300080586E6107D02046FEF764FD03B0BDE807
:10274000F04F00F047BC002E12DAD5F8003E984852
:102750009B071EBFD5F8003E23F00303C5F8003EDB
:10276000D5F8043823F00103C5F80438FEF774FDEA
:10277000370505D58E48FFF7BDFC8D48FEF75AFD9D
:10278000B0040CD5D5F8083813F0060FEB6823F425
:1027900070530CBF43F4105343F4A053EB60310764
:1027A0001BD56368DB681BB9AB6923F00803AB6119
:1027B0002378052B0CD1D5F8003E7D489A071EBF23
:1027C000D5F8003E23F00303C5F8003EFEF744FDB4
:1027D0006368DB680BB176489847F30274D4B7029C
:1027E00027D5D4F85490DFF8C8B100274FF0010A7C
:1027F00009EB4712D2F8003B03F44023B3F5802FD6
:1028000011D1D2F8003B002B0DDA62890AFA07F3E6
:1028100022EA0303638104EB8703DB68DB6813B1FF
:10282000394658469847A36D01379B68FFB29F42CF
:10283000DED9F00617D5676D3A6AC2F30A1002F0C6
:102840000F0302F4F012B2F5802F00F08580B2F58C
:10285000402F08D104EB83030022DB681B6A07F5D5
:10286000805790426AD13003D5F8184813D5E10358
:1028700002D50020FFF744FEA20302D50120FFF796
:102880003FFE630302D50220FFF73AFE270302D57D
:102890000320FFF735FE75037FF550AFE00702D543
:1028A0000020FFF7C1FEA10702D50120FFF7BCFE03
:1028B000620702D50220FFF7B7FE23077FF53EAF80
:1028C0000320FFF7B1FE39E7636DDFF8E4A0019361
:1028D00000274FF00109A36D9B685FFA87FB9B45BA
:1028E0003FF67DAF019B03EB4B13D3F8001901F4C6
:1028F0004021B1F5802F1FD1D3F8001900291BDA30
:10290000D3F8001941F09041C3F80019D3F8001929
:102910000029FBDB5946606DFFF718FC218909FA95
:102920000BF321EA0303238104EB8B03DB689B6831
:1029300013B15946504698470137CCE7910708BF75
:10294000D7F80080072A98BF03F8018B02F1010233
:1029500098BF4FEA182884E7023304EB830207F597
:1029600080575268D2F818C0DCF80820DCE9001C57
:10297000A1EB0C0C002188420AD104EB83046368AC
:102980009B699A6802449A605A6802445A606AE7EE
:1029900011F0030F08BFD7F800808C4588BF02F8FC
:1029A000018B01F1010188BF4FEA1828E3E700BF5E
:1029B000682D0020436D03EB4111D1F8003B43F437
:1029C0000013C1F8003B7047436D03EB4111D1F890
:1029D000003943F40013C1F800397047436D03EB2D
:1029E0004111D1F8003B23F40013C1F8003B7047BC
:1029F000436D03EB4111D1F8003923F40013C1F802
:102A00000039704700F1604303F561430901C9B221
:102A100083F80013012200F01F039A4043099B0032
:102A200003F1604303F56143C3F880211A607047E6
:102A300030B5039C0172043304FB0325C0E906533F
:102A4000049B03630021059BC160C0E90000C0E94D
:102A50000422C0E90842C0E90A11436330BD000006
:102A6000416A0022C0E90411C0E90A22C2606FF085
:102A70000101FEF7FBBE0000D0E90432934201D110
:102A8000C2680AB9181D70470020704703691960B1
:102A9000C2680132C260C269134482690361934211
:102AA00024BF436A03610021FEF7D4BE38B5044653
:102AB0000D46E3683BB16269131D1268A3621344BB
:102AC000E362002007E0237A33B929462046FEF767
:102AD000B1FE0028EDDA38BD6FF00100FBE7000021
:102AE000C368C269013BC36043691344826943619F
:102AF000934224BF436A436100238362036B03B1A3
:102B00001847704770B53023044683F31188866AEE
:102B10003EB9FFF7CBFF054618B186F3118828466A
:102B200070BDA36AE26A13F8015BA362934202D309
:102B30002046FFF7D5FF002383F31188EFE700005D
:102B40002DE9F84F04460E46174698464FF03009D7
:102B500089F311880025AA46D4F828B0BBF1000FEC
:102B600009D141462046FFF7A1FF20B18BF3118820
:102B70002846BDE8F88FD4E90A12A7EB050B521AD4
:102B8000934528BF9346BBF1400F1BD9334601F153
:102B9000400251F8040B43F8040B9142F9D1A36AA7
:102BA00040334036A3624035D4E90A239A4202D327
:102BB0002046FFF795FF8AF31188BD42D8D289F3EA
:102BC0001188C9E730465A46FEF758F8A36A5B44B5
:102BD0005E44A3625D44E7E710B5029C01720433D2
:102BE00003FB0421C0E906130023C0E90A33039B59
:102BF0000363049BC460C0E90000C0E90422C0E98B
:102C00000842436310BD0000026AC260426AC0E924
:102C100004220022C0E90A226FF00101FEF726BE5D
:102C2000D0E904239A4201D1C26822B9184650F86B
:102C3000043B0B60704700231846FAE7C368C2697B
:102C40000133C3604369134482694361934224BFE3
:102C5000436A43610021FEF7FDBD000038B504461C
:102C60000D46E3683BB123691A1DA262E269134471
:102C7000E362002007E0237A33B929462046FEF7B5
:102C8000D9FD0028EDDA38BD6FF00100FBE7000048
:102C900003691960C268013AC260C269134482695B
:102CA0000361934224BF436A036100238362036B81
:102CB00003B118477047000070B530230D46044635
:102CC000114683F31188866A2EB9FFF7C7FF10B14A
:102CD00086F3118870BDA36A1D70A36AE26A01338E
:102CE0009342A36204D3E16920460439FFF7D0FF81
:102CF000002080F31188EDE72DE9F84F04460D46DA
:102D0000904699464FF0300A8AF311880026B34660
:102D1000A76A4FB949462046FFF7A0FF20B187F3C5
:102D200011883046BDE8F88FD4E90A073A1AA8EBB3
:102D30000607974228BF1746402F1BD905F14003CD
:102D400055F8042B40F8042B9D42F9D1A36A403377
:102D5000A3624036D4E90A239A4204D3E1692046AB
:102D60000439FFF795FF8BF311884645D9D28AF3D2
:102D70001188CDE729463A46FDF780FFA36A3B4418
:102D80003D44A3623E44E5E7D0E904239A4217D1CB
:102D9000C3689BB1836A8BB1043B9B1A0ED013604E
:102DA000C368013BC360C3691A44836902619A42E4
:102DB00024BF436A036100238362012318467047DE
:102DC0000023FBE700F030B94FF08043586A7047AA
:102DD0004FF08043002258631A610222DA60704784
:102DE0004FF080430022DA60704700004FF08043CC
:102DF00058637047FEE7000070B51B4B0163002568
:102E0000044686B0586085620E4600F0BFF804F1B3
:102E10001003C4E904334FF0FF33C4E90635C4E9B5
:102E20000044A560E562FFF7CFFF2B460246C4E9E8
:102E3000082304F134010D4A256580232046FEF75E
:102E4000AFFC0123E0600A4A0375009272680192A8
:102E5000B268CDE90223074B6846CDE90435FEF799
:102E6000C7FC06B070BD00BF002600206C3600080D
:102E700071360008F52D0008024AD36A1843D06263
:102E8000704700BF982300204B6843608B688360C5
:102E9000CB68C3600B6943614B6903628B69436212
:102EA0000B6803607047000008B5264B26481A6976
:102EB00040F2FF110A431A611A6922F4FF7222F0EC
:102EC00001021A611A691A6B0A431A631A6D0A43DE
:102ED0001A651E4A1B6D1146FFF7D6FF02F11C0151
:102EE00000F58060FFF7D0FF02F1380100F5806047
:102EF000FFF7CAFF02F1540100F58060FFF7C4FF3D
:102F000002F1700100F58060FFF7BEFF02F18C0155
:102F100000F58060FFF7B8FF02F1A80100F58060BE
:102F2000FFF7B2FF02F1C40100F58060FFF7ACFFCC
:102F300002F1E00100F58060FFF7A6FFBDE8084060
:102F400000F0EEB800380240000002407836000879
:102F500008B500F059FAFEF701FCFFF793F8BDE859
:102F60000840FEF76FBE000070470000EFF30983D2
:102F700005494A6B22F001024A63683383F30988EA
:102F8000002383F31188704700EF00E0302080F3C6
:102F9000118862B60C4B0D4AD96821F4E06109042E
:102FA000090C0A43DA60D3F8FC20094942F0807228
:102FB000C3F8FC200A6842F001020A602022DA7796
:102FC00083F82200704700BF00ED00E00003FA051F
:102FD000001000E010B5302383F311880E4B5B68BE
:102FE00013F4006314D0F1EE103AEFF30984683C57
:102FF0004FF08073E361094BDB6B236684F3098830
:10300000FEF78CFB10B1064BA36110BD054BFBE72F
:1030100083F31188F9E700BF00ED00E000EF00E066
:103020002F030008320300080F4B1A6C42F0010214
:103030001A641A6E42F001021A660C4A1B6E9368FB
:1030400043F0010393604FF0804353229A624FF0A4
:10305000FF32DA6200229A615A63DA605A60012212
:103060005A611A60704700BF00380240002004E037
:103070004FF0804208B51169D3680B40D9B2C943FB
:103080009B07116107D5302383F31188FEF77CFB82
:10309000002383F3118808BD1F4B1A696FEAC252DF
:1030A0006FEAD2521A611A69C2F308021A614FF02C
:1030B000FF301A695A69586100215A6959615A6981
:1030C0001A6A62F080521A621A6A02F080521A6218
:1030D0001A6A5A6A58625A6A59625A6A1A6C42F0F3
:1030E00080521A641A6E42F080521A661A6E0B4AA7
:1030F000106840F480701060186F00F44070B0F5F4
:10310000007F1EBF4FF4803018671967536823F49F
:103110000073536000F054B9003802400070004062
:10312000334B4FF080521A64324A4FF440411160E1
:103130001A6842F001021A601A689107FCD59A6871
:1031400022F003029A602A4B9A6812F00C02FBD11B
:10315000196801F0F90119609A601A6842F4803226
:103160001A601A689203FCD55A6F42F001025A673E
:103170001F4B5A6F9007FCD51F4A5A601A6842F0DD
:1031800080721A601B4A53685904FCD5184B1A68A0
:103190009201FCD5194A9A60194B1A68194B9A4248
:1031A000194B21D1194A1168194A91421CD140F298
:1031B00005121A60144A136803F00F03052BFAD1A5
:1031C0000B4B9A6842F002029A609A6802F00C0275
:1031D000082AFAD15A6C42F480425A645A6E42F478
:1031E00080425A665B6E704740F20572E1E700BFAD
:1031F00000380240007000400854400700948838AE
:10320000002004E011640020003C024000ED00E0DA
:1032100041C20F41074A08B5536903F001035361E6
:1032200023B1054A13680BB150689847BDE80840C0
:10323000FFF7D0BE003C0140E02D0020074A08B552
:10324000536903F00203536123B1054A93680BB13C
:10325000D0689847BDE80840FFF7BCBE003C01407D
:10326000E02D0020074A08B5536903F004035361B9
:1032700023B1054A13690BB150699847BDE808406E
:10328000FFF7A8BE003C0140E02D0020074A08B52A
:10329000536903F00803536123B1054A93690BB1E5
:1032A000D0699847BDE80840FFF794BE003C014054
:1032B000E02D0020074A08B5536903F0100353615D
:1032C00023B1054A136A0BB1506A9847BDE808401C
:1032D000FFF780BE003C0140E02D0020164B10B5EA
:1032E0005C6904F478725A61A30604D5134A936AA0
:1032F0000BB1D06A9847600604D5104A136B0BB126
:10330000506B9847210604D50C4A936B0BB1D06BD8
:103310009847E20504D5094A136C0BB1506C9847E5
:10332000A30504D5054A936C0BB1D06C9847BDE852
:103330001040FFF74FBE00BF003C0140E02D0020D1
:10334000194B10B55C6904F47C425A61620504D5DE
:10335000164A136D0BB1506D9847230504D5134AD7
:10336000936D0BB1D06D9847E00404D50F4A136EEE
:103370000BB1506E9847A10404D50C4A936E0BB163
:10338000D06E9847620404D5084A136F0BB1506F92
:103390009847230404D5054A936F0BB1D06F984723
:1033A000BDE81040FFF716BE003C0140E02D0020B4
:1033B00008B5FFF75DFEBDE80840FFF70BBE000053
:1033C000062108B50846FFF71DFB06210720FFF779
:1033D00019FB06210820FFF715FB06210920FFF73E
:1033E00011FB06210A20FFF70DFB06211720FFF72E
:1033F00009FB06212820FFF705FBBDE8084007214F
:103400001C20FFF7FFBA000008B5FFF745FE00F0EB
:103410000BF8FDF78DFEFDF765FDFFF7A5FDBDE897
:103420000840FFF7CFBC00000023054A19460133CE
:10343000102BC2E9001102F10802F8D1704700BF59
:10344000E02D0020034611F8012B03F8012B002A80
:10345000F9D1704753544D3332463F3F3F005354E8
:103460004D3332463430780053544D333246343283
:10347000780053544D3332463434365858000000E7
:10348000012033000010410001105A0003105900C0
:10349000071031000000000054340008130400003D
:1034A0005E3400081904000068340008210400009C
:1034B0007234000800000000610E00084D0E000884
:1034C000890E0008750E0008810E00086D0E0008B8
:1034D000590E0008450E0008950E00080000000077
:1034E000010000000000000063300000E834000824
:1034F000F0230020002600204172647550696C6F33
:10350000740025424F415244252D424C002553451D
:103510005249414C2500000002000000000000005C
:103520007D100008E910000840004000A02A00209B
:10353000B02A00200200000000000000030000008C
:10354000000000002D110008000000001000000025
:10355000C02A002000000000010000000000000060
:10356000682D002001010200E11B0008F11A00088B
:103570008D1B0008711B0008430000008035000807
:1035800009024300020100C03209040000010202E6
:103590000100052400100105240100010424020299
:1035A0000524060001070582030800FF0904010045
:1035B000020A000000070501024000000705810221
:1035C0004000000012000000CC350008120110017C
:1035D00002000040091241570002010203010000ED
:1035E0000403090425424F41524425005442535FCD
:1035F0004C554349445F50524F00303132333435DB
:103600003637383941424344454600000040000007
:1036100000400000004000000040000000000100E9
:103620000000020000000200000002000000020092
:103630000000020000000200000002000000000084
:103640007112000829150008D51500084000400037
:10365000C82D0020C82D002001000000D82D00201A
:103660008000000040010000030000006D61696EF1
:103670000069646C650000000001806A00000000C1
:10368000AAAAAAAA00010064FFFF0000000000002F
:1036900000A00A000000000100000000AAAAAAAAD7
:1036A00000000001FFFF000000000000000000001B
:1036B0000000001000000000AAAAAAAA0000000052
:1036C000FFBF00000000000000000000000000003C
:1036D00000000000AAAAAAAA00000000FFFF000044
:1036E00000000000000000000000000000000000DA
:1036F000AAAAAAAA00000000FFFF00000000000024
:10370000000000000000000000000000AAAAAAAA11
:1037100000000000FFFF00000000000000000000AB
:103720000000000000000000AAAAAAAA00000000F1
:10373000FFFF00000000000000000000000000008B
:10374000000000000A00000000000000030000006C
:103750000000000000000000000000000000000069
:103760000000000000000000000000000000000059
:1037700000000000000000008314000000000000B2
:1037800000400F0000000000FF009600000000084D
:10379000009600000000080004000000E03500086A
:1037A0000000000000000000000000000000000019
:1037B0000000000000000000FFFFFFFFFFFFFFFF11
:1037C000FFFFFFFFFFFFFFFFFFFFFFFFFFFFFFFF09
:1037D000FFFFFFFFFFFFFFFFFFFFFFFFFFFFFFFFF9
:1037E000FFFFFFFFFFFFFFFFFFFFFFFFFFFFFFFFE9
:1037F000FFFFFFFFFFFFFFFFFFFFFFFFFFFFFFFFD9
:10C000000006002099D20008B9F2090815F20908C3
:10C0100081F2090815F209084DF209089BD20008BF
:10C020009BD200089BD200089BD20008C5470C0891
:10C030009BD200089BD200089BD200089BD200082C
:10C040009BD200089BD200089BD200089BD200081C
:10C050009BD200089BD20008E1590C08095A0C0831
:10C06000315A0C08595A0C08815A0C08D9060C0888
:10C0700001070C082D070C0859070C0885070C0848
:10C08000AD070C08D9070C085D060C089BD2000808
:10C090009BD200089BD200089BD20008A95A0C082A
:10C0A000F55B0C08F95B0C080D5C0C08115C0C08C6
:10C0B0009BD20008155C0C08295C0C08650D0C0867
:10C0C0000D0F0C089BD200089BD200089BD20008E1
:10C0D0009BD200087D5B0C08915B0C08A55B0C08EB
:10C0E0000D5B0C089BD200089BD200089BD2000875
:10C0F0009BD200089BD200089BD2000805080C08C0
:10C100009BD200089BD200083D5C0C089BD2000823
:10C11000B95B0C08CD5B0C089BD200089BD20008D1
:10C1200031080C0859080C0885080C08B1080C08DF
:10C13000DD080C089BD200089BD200089BD20008A7
:10C140009BD200089BD200089BD20008F14E0C083D
:10C1500005090C0831090C085D090C08E15B0C08A5
:10C160009BD200089BD200089BD200089BD20008FB
:10C170009BD200089BD200089BD200089BD20008EB
:10C180009BD200089BD200089BD200089BD20008DB
:10C190009BD200089BD200089BD200089BD20008CB
:10C1A0009BD200089BD200089BD200089BD20008BB
:10C1B0009BD200089BD200089BD200089BD20008AB
:10C1C0009BD200089BD200089BD200089BD200089B
:10C1D0009BD200089BD200089BD200089BD200088B
:10C1E0004DF5000825260108796001085DBE0108AB
:10C1F00095070208D1810208F909040825D305082A
:10C200002DD90508E1370608E9890608AD91060829
:10C21000E594060871FA0608C51A070831D7070819
:10C22000614F080871EB09083D1D0B0881770B0869
:10C23000599E0B0819B40B08D9E10B08A1E70B08AC
:10C2400081F0004102E000BF83F0004330B54FEAC7
:10C2500041044FEA430594EA050F08BF90EA020F34
:10C260001FBF54EA000C55EA020C7FEA645C7FEAC7
:10C27000655C00F0E2804FEA5454D4EB5555B8BFEA
:10C280006D420CDD2C4480EA020281EA030382EA5B
:10C29000000083EA010180EA020281EA0303362DED
:10C2A00088BF30BD11F0004F4FEA01314FF4801CC0
:10C2B0004CEA113102D0404261EB410113F0004FD2
:10C2C0004FEA03334CEA133302D0524263EB430389
:10C2D00094EA050F00F0A780A4F10104D5F1200E27
:10C2E0000DDB02FA0EFC22FA05F2801841F1000182
:10C2F00003FA0EF2801843FA05F359410EE0A5F156
:10C3000020050EF1200E012A03FA0EFC28BF4CF086
:10C31000020C43FA05F3C01851EBE37101F000453C
:10C3200007D54FF0000EDCF1000C7EEB00006EEB49
:10C330000101B1F5801F1BD3B1F5001F0CD34908D3
:10C340005FEA30004FEA3C0C04F101044FEA44522A
:10C3500012F5800F80F09A80BCF1004F08BF5FEAB1
:10C36000500C50F1000041EB045141EA050130BD91
:10C370005FEA4C0C404141EB0101013C28BFB1F5A3
:10C38000801FE9D291F0000F04BF01460020B1FAEE
:10C3900081F308BF2033A3F10B03B3F120020CDAC1
:10C3A0000C3208DD02F1140CC2F10C0201FA0CF09F
:10C3B00021FA02F10CE002F11402D8BFC2F1200C04
:10C3C00001FA02F120FA0CFCDCBF41EA0C019040BA
:10C3D000E41AA2BF01EB0451294330BD6FEA040403
:10C3E0001F3C1CDA0C340EDC04F11404C4F12002EE
:10C3F00020FA04F001FA02F340EA030021FA04F300
:10C4000045EA030130BDC4F10C04C4F1200220FA56
:10C4100002F001FA04F340EA0300294630BD21FA94
:10C4200004F0294630BD94F0000F83F4801306BF5A
:10C4300081F480110134013D4EE77FEA645C18BF4E
:10C440007FEA655C29D094EA050F08BF90EA020FE5
:10C4500005D054EA000C04BF1946104630BD91EADD
:10C46000030F1EBF0021002030BD5FEA545C05D1E0
:10C470004000494128BF41F0004130BD14F580041F
:10C480003CBF01F5801130BD01F0004545F0FE4193
:10C4900041F470014FF0000030BD7FEA645C1ABFC8
:10C4A000194610467FEA655C1CBF0B46024650EAFF
:10C4B000013406BF52EA033591EA030F41F400212B
:10C4C00030BD00BF90F0000F04BF0021704730B5B1
:10C4D0004FF4806404F132044FF000054FF0000186
:10C4E00050E700BF90F0000F04BF0021704730B547
:10C4F0004FF4806404F1320410F0004548BF40421C
:10C500004FF000013EE700BF42004FEAE2014FEA70
:10C5100031014FEA02701FBF12F07F4393F07F4F4B
:10C5200081F06051704732F07F4208BF704793F04E
:10C530007F4F04BF41F40021704730B54FF4607461
:10C5400001F0004521F000411CE700BF50EA010264
:10C5500008BF704730B54FF000050AE050EA01020D
:10C5600008BF704730B511F0004502D5404261EB7D
:10C5700041014FF4806404F132045FEA915C3FF4BE
:10C58000D8AE4FF003025FEADC0C18BF03325FEA5B
:10C59000DC0C18BF033202EBDC02C2F1200300FA0C
:10C5A00003FC20FA02F001FA03FE40EA0E0021FA31
:10C5B00002F11444BDE600BF70B54FF0FF0C4CF41F
:10C5C000E06C1CEA11541DBF1CEA135594EA0C0FD1
:10C5D00095EA0C0F00F0DEF82C4481EA030621EA0C
:10C5E0004C5123EA4C5350EA013518BF52EA033547
:10C5F00041F4801143F4801338D0A0FB02CE4FF0F9
:10C600000005E1FB02E506F00042E0FB03E54FF028
:10C610000006E1FB03569CF0000F18BF4EF0010E20
:10C62000A4F1FF04B6F5007F64F5407404D25FEA1C
:10C630004E0E6D4146EB060642EAC62141EA5551CF
:10C640004FEAC52040EA5E504FEACE2EB4F1FD0C11
:10C6500088BFBCF5E06F1ED8BEF1004F08BF5FEA8F
:10C66000500E50F1000041EB045170BD06F0004641
:10C6700046EA010140EA020081EA0301B4EB5C04EE
:10C68000C2BFD4EB0C0541EA045170BD41F48011E6
:10C690004FF0000E013C00F3AB8014F1360FDEBF0B
:10C6A000002001F0004170BDC4F10004203C35DAE7
:10C6B0000C341BDC04F11404C4F1200500FA05F36A
:10C6C00020FA04F001FA05F240EA020001F000420B
:10C6D00021F0004110EBD37021FA04F642EB060181
:10C6E0005EEA430E08BF20EAD37070BDC4F10C04AB
:10C6F000C4F1200500FA04F320FA05F001FA04F26F
:10C7000040EA020001F0004110EBD37041F100015A
:10C710005EEA430E08BF20EAD37070BDC4F1200565
:10C7200000FA05F24EEA020E20FA04F301FA05F2CD
:10C7300043EA020321FA04F001F0004121FA04F275
:10C7400020EA020000EBD3705EEA430E08BF20EA45
:10C75000D37070BD94F0000F0FD101F0004640007F
:10C7600041EB010111F4801F08BF013CF7D041EA01
:10C77000060195F0000F18BF704703F00046520005
:10C7800043EB030313F4801F08BF013DF7D043EAD6
:10C790000603704794EA0C0F0CEA135518BF95EA8C
:10C7A0000C0F0CD050EA410618BF52EA4306D1D113
:10C7B00081EA030101F000414FF0000070BD50EA32
:10C7C000410606BF1046194652EA430619D094EABC
:10C7D0000C0F02D150EA013613D195EA0C0F05D1A6
:10C7E00052EA03361CBF104619460AD181EA0301FA
:10C7F00001F0004141F0FE4141F470014FF00000B2
:10C8000070BD41F0FE4141F4780170BD70B54FF04C
:10C81000FF0C4CF4E06C1CEA11541DBF1CEA1355CC
:10C8200094EA0C0F95EA0C0F00F0A7F8A4EB0504AE
:10C8300081EA030E52EA03354FEA013100F08880A5
:10C840004FEA03334FF0805545EA131343EA12636E
:10C850004FEA022245EA111545EA10654FEA002623
:10C860000EF000419D4208BF964244F1FD0404F5DC
:10C87000407402D25B084FEA3202B61A65EB030538
:10C880005B084FEA32024FF480104FF4002CB6EBF5
:10C89000020E75EB030E22BFB61A754640EA0C0075
:10C8A0005B084FEA3202B6EB020E75EB030E22BFB5
:10C8B000B61A754640EA5C005B084FEA3202B6EBF6
:10C8C000020E75EB030E22BFB61A754640EA9C00B5
:10C8D0005B084FEA3202B6EB020E75EB030E22BF85
:10C8E000B61A754640EADC0055EA060E18D04FEA43
:10C8F000051545EA16754FEA06164FEAC30343EAE3
:10C9000052734FEAC2025FEA1C1CC0D111F4801FAF
:10C910000BD141EA00014FF000004FF0004CB6E7A8
:10C9200011F4801F04BF01430020B4F1FD0C88BF47
:10C93000BCF5E06F3FF6AFAEB5EB030C04BFB6EB52
:10C94000020C5FEA500C50F1000041EB045170BD45
:10C950000EF0004E4EEA113114EB5C04C2BFD4EB72
:10C960000C0541EA045170BD41F480114FF0000EF6
:10C97000013C90E645EA060E8DE60CEA135594EA72
:10C980000C0F08BF95EA0C0F3FF43BAF94EA0C0F75
:10C990000AD150EA01347FF434AF95EA0C0F7FF4EA
:10C9A00025AF104619462CE795EA0C0F06D152EA3E
:10C9B00003353FF4FDAE1046194622E750EA410622
:10C9C00018BF52EA43067FF4C5AE50EA41047FF433
:10C9D0000DAF52EA43057FF4EBAE12E74FF0FF3C98
:10C9E00006E000BF4FF0010C02E000BF4FF0010C69
:10C9F0004DF804CD4FEA410C7FEA6C5C4FEA430CE2
:10CA000018BF7FEA6C5C1BD001B050EA410C0CBF30
:10CA100052EA430C91EA030F02BF90EA020F002092
:10CA2000704710F1000F91EA030F58BF994208BFF9
:10CA300090422CBFD8176FEAE37040F001007047B6
:10CA40004FEA410C7FEA6C5C02D150EA013C07D10D
:10CA50004FEA430C7FEA6C5CD6D152EA033CD3D058
:10CA60005DF8040B704700BF8446104662468C4652
:10CA70001946634600E000BF01B5FFF7B7FF002885
:10CA800048BF10F1000F01BD4DF808EDFFF7F4FFAE
:10CA90000CBF012000205DF808FB00BF4DF808ED39
:10CAA000FFF7EAFF34BF012000205DF808FB00BF5C
:10CAB0004DF808EDFFF7E0FF94BF012000205DF87E
:10CAC00008FB00BF4DF808EDFFF7CEFF94BF012033
:10CAD00000205DF808FB00BF4DF808EDFFF7C4FF2C
:10CAE00034BF012000205DF808FB00BF4FEA410C75
:10CAF0007FEA6C5C02D150EA013C0AD14FEA430C58
:10CB00007FEA6C5C02D152EA033C02D14FF0000094
:10CB100070474FF0010070474FEA410212F50012D2
:10CB200015D211D56FF47873B3EB625212D94FEA74
:10CB3000C12343F0004343EA505311F0004F23FA5E
:10CB400002F018BF404270474FF00000704750EAB3
:10CB5000013005D111F0004008BF6FF00040704770
:10CB60004FF00000704700BF4A0011D212F50012CA
:10CB700011D20DD56FF47873B3EB62520ED44FEA35
:10CB8000C12343F0004343EA505323FA02F07047B5
:10CB90004FF00000704750EA013002D14FF0FF30F3
:10CBA00070474FF0000070474FEA4102B2F1E04396
:10CBB00024BFB3F5001CDCF1FE5C0DD901F0004C84
:10CBC0004FEAC0024CEA5070B2F1004F40EB8300D4
:10CBD00008BF20F00100704711F0804F21D113F100
:10CBE0003872BCBF01F00040704741F480114FEA39
:10CBF0005252C2F11802C2F1200C10FA0CF320FAC2
:10CC000002F018BF40F001004FEAC1234FEAD323DE
:10CC100003FA0CFC40EA0C0023FA02F34FEA430348
:10CC2000CCE77FEA625307D150EA01331EBF4FF0D1
:10CC3000FE4040F44000704701F0004040F0FE40EC
:10CC400040F40000704700BF80F0004002E000BFE9
:10CC500081F0004142001FBF5FEA410392EA030FE7
:10CC60007FEA226C7FEA236C6AD04FEA1262D2EB31
:10CC70001363C1BFD218414048404140B8BF5B4236
:10CC8000192B88BF704710F0004F40F4000020F0CF
:10CC90007F4018BF404211F0004F41F4000121F0E5
:10CCA0007F4118BF494292EA030F3FD0A2F101022F
:10CCB00041FA03FC10EB0C00C3F1200301FA03F16D
:10CCC00000F0004302D5494260EB4000B0F5000F90
:10CCD00013D3B0F1807F06D340084FEA310102F14F
:10CCE0000102FE2A51D2B1F1004F40EBC25008BF01
:10CCF00020F0010040EA03007047490040EB0000CB
:10CD0000013A28BFB0F5000FEDD2B0FA80FCACF1CB
:10CD1000080CB2EB0C0200FA0CF0AABF00EBC250F8
:10CD200052421843BCBFD0401843704792F0000FE6
:10CD300081F4000106BF80F400000132013BB5E739
:10CD40004FEA41037FEA226C18BF7FEA236C21D0AF
:10CD500092EA030F04D092F0000F08BF0846704714
:10CD600090EA010F1CBF0020704712F07F4F04D1E2
:10CD7000400028BF40F00040704712F100723CBFF5
:10CD800000F50000704700F0004343F0FE4040F41F
:10CD9000000070477FEA226216BF08467FEA2363DD
:10CDA0000146420206BF5FEA412390EA010F40F4C8
:10CDB000800070474FF0000304E000BF10F0004314
:10CDC00048BF40425FEA000C08BF704743F09643FB
:10CDD00001464FF000001CE050EA010208BF704716
:10CDE0004FF000030AE000BF50EA010208BF70479D
:10CDF00011F0004302D5404261EB41015FEA010CB2
:10CE000002BF84460146002043F0B64308BFA3F1A9
:10CE10008053A3F50003BCFA8CF2083AA3EBC2538B
:10CE200010DB01FA02FC634400FA02FCC2F12002AA
:10CE3000BCF1004F20FA02F243EB020008BF20F0E1
:10CE40000100704702F1200201FA02FCC2F1200247
:10CE500050EA4C0021FA02F243EB020008BF20EA3C
:10CE6000DC7070477BB972B90029BEBF00204FF05B
:10CE7000004106E008BF00281CBF6FF000414FF0E2
:10CE8000FF3000F007BAADF1080C6DE904CE0029BF
:10CE900009DB002B1ADB00F095F8DDF804E0DDE992
:10CEA000022304B07047404261EB4101002B1BDBC1
:10CEB00000F088F8DDF804E0DDE9022304B0404228
:10CEC00061EB4101524263EB43037047524263EB13
:10CED000430300F077F8DDF804E0DDE9022304B055
:10CEE000404261EB41017047524263EB430300F063
:10CEF00069F8DDF804E0DDE9022304B0524263EB97
:10CF00004303704753B94AB9002908BF00281CBF22
:10CF10004FF0FF314FF0FF3000F0BCB9ADF1080C1D
:10CF20006DE904CE00F04EF8DDF804E0DDE90223FF
:10CF300004B07047430803F05533C01A830803F068
:10CF4000333300F03330184400EB101000F00F3092
:10CF500000EB002000EB0040000E704707EE900A47
:10CF6000F5EEC07AF1EE10FA01D400F00BB8F1EE54
:10CF7000677A08B517EE900A00F004F8404261EBBA
:10CF8000410108BDD0B5FFF7BFFA0C4B00220646A1
:10CF90000F46FFF711FBFFF7E7FD0446FFF792FA94
:10CFA000074B0022FFF708FB02460B463046394686
:10CFB000FFF74AF9FFF7D8FD2146D0BD0000F03D4C
:10CFC0000000F0412DE9F047089D04468E46002BF5
:10CFD0004DD18A42944669D9B2FA82F252B101FA2D
:10CFE00002F3C2F1200120FA01F10CFA02FC41EA3D
:10CFF000030E94404FEA1C48210CBEFBF8F61FFAC2
:10D000008CF708FB16E341EA034306FB07F199425C
:10D010000AD91CEB030306F1FF3080F01F8199420F
:10D0200040F21C81023E63445B1AA4B2B3FBF8F0E9
:10D0300008FB103344EA034400FB07F7A7420AD970
:10D040001CEB040400F1FF3380F00A81A74240F298
:10D0500007816444023840EA0640E41B00261DB103
:10D06000D4400023C5E900433146BDE8F0878B4238
:10D0700009D9002D00F0EF800026C5E900013046F7
:10D080003146BDE8F087B3FA83F6002E4AD18B42D1
:10D0900002D3824200F2F980841A61EB030301207B
:10D0A0009E46002DE0D0C5E9004EDDE702B9FFDE67
:10D0B000B2FA82F2002A40F09280A1EB0C014FEA12
:10D0C0001C471FFA8CFE0126200CB1FBF7F307FB6F
:10D0D000131140EA01410EFB03F0884208D91CEB12
:10D0E000010103F1FF3802D2884200F2CB804346AF
:10D0F000091AA4B2B1FBF7F007FB101144EA01448E
:10D100000EFB00FEA64508D91CEB040400F1FF311C
:10D1100002D2A64500F2BB800846A4EB0E0440EA0A
:10D1200003409CE7C6F12007B34022FA07FC4CEA13
:10D13000030C20FA07F401FA06F31C43F9404FEA06
:10D140001C4900FA06F3B1FBF9F8200C1FFA8CFE1B
:10D1500009FB181140EA014108FB0EF0884202FA6F
:10D1600006F20BD91CEB010108F1FF3A80F0888030
:10D17000884240F28580A8F102086144091AA4B2ED
:10D18000B1FBF9F009FB101144EA014100FB0EFE6E
:10D190008E4508D91CEB010100F1FF346CD28E459D
:10D1A0006AD90238614440EA0840A0FB0294A1EB2E
:10D1B0000E01A142C846A64656D353D05DB1B3EB8B
:10D1C000080261EB0E0101FA07F722FA06F3F140BB
:10D1D0001F43C5E9007100263146BDE8F087C2F162
:10D1E0002003D8400CFA02FC21FA03F391400143DA
:10D1F0004FEA1C471FFA8CFEB3FBF7F007FB103613
:10D200000B0C43EA064300FB0EF69E4204FA02F4BE
:10D2100008D91CEB030300F1FF382FD29E422DD911
:10D22000023863449B1B89B2B3FBF7F607FB163346
:10D2300041EA034106FB0EF38B4208D91CEB0101C6
:10D2400006F1FF3816D28B4214D9023E6144C91A46
:10D2500046EA004638E72E46284605E70646E3E656
:10D260001846F8E64B45A9D2B9EB020864EB0C0E60
:10D270000138A3E74646EAE7204694E74046D1E76F
:10D28000D0467BE7023B614432E7304609E764441D
:10D29000023842E7704700BF02E000F000F8FEE706
:10D2A00072B6374880F30888364880F309883648D4
:10D2B0003649086040F20000CCF200004EF63471AE
:10D2C000CEF200010860BFF34F8FBFF36F8F40F2C3
:10D2D0000000C0F2F0004EF68851CEF20001086066
:10D2E000BFF34F8FBFF36F8F4FF00000E1EE100AD6
:10D2F0004EF63C71CEF200010860062080F31488DF
:10D30000BFF36F8FB7F0BCFAB8F006FA4FF05530A4
:10D310001F491B4A91423CBF41F8040BFAE71D49E3
:10D32000184A91423CBF41F8040BFAE71A491B4ADC
:10D330001B4B9A423EBF51F8040B42F8040BF8E72E
:10D3400000201849184A91423CBF41F8040BFAE703
:10D35000B7F09AFAB8F034FA144C154DAC4203DA2F
:10D3600054F8041B8847F9E702F0E0F8114C124D1D
:10D37000AC4203DA54F8041B8847F9E7B7F082BAE5
:10D38000000600200022002000C0000808ED00E098
:10D390000000002000060020F0180F0800220020E6
:10D3A000302C0020302C0020D8560120E0C100088D
:10D3B00040C2000840C2000840C200082DE9F04FFA
:10D3C0002DED108AC1F80CD0C3689D46BDEC108AC3
:10D3D000BDE8F08F002383F311882846A047002082
:10D3E000B6F042FAFEE7B6F0AFF800DFFEE7000065
:10D3F00001F0FF01102A2BDB10F0070F08D010F806
:10D40000013B013A8B422DD010F0070F42B3F6D109
:10D41000F0B441EA012141EA014122F007047FF022
:10D4200000070023F0E80256083C85EA010586EA79
:10D43000010685FA47F5A3FA87F586FA47F6A5FAB5
:10D4400087F68EB9EED1F0BC01F0FF0102F00702C1
:10D4500032B110F8013B013A83EA010313B1F8D16C
:10D460000020704701387047002D06BF354603384D
:10D47000073815F0010F07D1013015F4807F02BF86
:10D48000013015F4C03F0130F0BC0138704700BFD7
:10D4900010F8012B11F8013B012A28BF9A42F7D05E
:10D4A000D01A7047034613F8012B002AFBD1181A33
:10D4B0000138704738B50022002304460D46FFF7B7
:10D4C000EDFA28B920462946BDE8384000F00AB8F0
:10D4D000204605F1004100F005F8404261EB4101B2
:10D4E00038BD00BFD0B50C4B002206460F46FFF7F3
:10D4F00063F8FFF739FB0446FEF7E4FF074B002211
:10D50000FFF75AF802460B4630463946FEF79CFEB6
:10D51000FFF72AFB2146D0BD0000F03D0000F0419E
:10D52000036800221B6818477FB503914021054618
:10D5300080F0E8FB039A18B90124204604B070BDBE
:10D54000134E039296F98A34002BF5D062F0C6FC94
:10D55000437A039A53B962F0C1FC847A039A2CB9D6
:10D560000C4B4021284680F0D5FBE6E7D6F8443E38
:10D57000B6F98C14B3F906309942DDDD064B009301
:10D580004021064B284680F0C5FB0024D5E700BFAC
:10D59000384C002018CE0C0837CE0C0825CE0C08CD
:10D5A000F0B50D469DB02021044680F0ABFB00286D
:10D5B00000F0A180514E96F98A34ABB1D6F8442ED2
:10D5C000B6F98C34B2F90A1003F10A02914203DD74
:10D5D00040F28D32934207DC494B2A4620212046F7
:10D5E00080F098FB002084E096F97934022B05D175
:10D5F000444B2A462021204680F08CFBB6F84C3460
:10D60000A3F57A739BB241F6583293420FD83E4F3E
:10D61000D7F8843E06F5976292ED007AD3ED097A49
:10D62000B4EEE77AF1EE10FA03DD384BD5E7384B6C
:10D63000D3E706F2BC4292ED007AD3ED0B7AB4EE5A
:10D64000E77AF1EE10FAF0DCB6F98634002B01DC53
:10D65000304BC2E796F8DC240D2A06D8012393400C
:10D6600013F4215F01D02C4BB7E72C480FF0CAFE12
:10D67000012806D1D7F8900E87F05CFB98B10128FD
:10D680001AD00021602204A80391BBF08FF824492E
:10D69000D7F88C0E642303AA86F06EFF00BB03ABA1
:10D6A0000093204B02E0204B0093204B2A46202180
:10D6B000204680F02FFB95E796F8583E73B11C4842
:10D6C000192150F033FB48B11948D6F86464192188
:10D6D00050F052FB8642D4DD164BE5E7164BE3E7EC
:10D6E0001649D7F8840E642303AA83F005FE0028A8
:10D6F000D5D01DB0F0BD0120FBE700BF384C0020A5
:10D7000040CE0C0853CE0C08386C00208BCE0C0891
:10D710007BCE0C08A5CE0C08BACE0C08E082002007
:10D7200034CF0C0838CF0C08FFCE0C08DACE0C082A
:10D73000683B00201ECF0C080FCF0C084ACF0C0806
:10D7400007B5044888F04EFE00F0010003B05DF814
:10D7500004FB00BFA07A00202DE9F043DFF84491DC
:10D760000446D9F854020368A5B01B690D469847D2
:10D77000804615F073F90021074660220CA80B9132
:10D78000BBF014F864230BAA4146384614F05AFC47
:10D79000064648B93A4A0BAB2946204680F0C2FCFF
:10D7A000304625B0BDE8F083A9F608506EF03EFA89
:10D7B000B8F1000F03D194F91E30012B0AD1314882
:10D7C00012F02CF980B9304A2946204680F0AAFC94
:10D7D0000026E5E710F0060FE2D0A9F5405012F060
:10D7E0001DF908B9294AEFE703A9384614F05CFA95
:10D7F00028B19DF80D305B0601D5254AE4E7DFF836
:10D80000A880D8ED007AF5EEC07AF1EE10FA4FF06C
:10D810000003C5DD089309930A930DF1200907ABB6
:10D82000019305AA06AB04A9CDF80090384614F080
:10D830001DFE484630F0CEF8D8ED007AB4EEE70A87
:10D84000F1EE10FA01DB134ABEE79DED057AF4EE26
:10D85000C77AF1EE10FA01D80F4AB5E79DED047AC8
:10D86000F4EEC77AF1EE10FA01D80C4AACE79DED60
:10D87000067AF4EEC77AF1EE10FA91D8084AA3E7D7
:10D8800050CF0C08382C002059CF0C0870CF0C0852
:10D8900096CF0C08A4CF0C08B9CF0C08CFCF0C083A
:10D8A000E5CF0C08385C0020E050002008B5064B9E
:10D8B00093F86D329B0704D5044A80F033FC0020B6
:10D8C00008BD0120FCE700BF385C0020FCCF0C083D
:10D8D00070B50C4C0546D4F8540203685B690E46DB
:10D8E000984710B10124204670BDA4F5405012F0B5
:10D8F000A7F804460028F5D1034A3146284680F0AF
:10D9000011FCF0E7385C00200CD00C082DE9F04643
:10D91000464ED6F8783293F8CB509BB081468A4673
:10D9200065B9434B1B68986A03685B6B984704466C
:10D9300040B9404A5146484680F0F4FB28461BB0A7
:10D94000BDE8F08662F0CAFA202163F0CBFA58B144
:10D9500062F0C4FA1F2163F0C5FA88B3364A514613
:10D96000484680F0DFFB002496F84A3203F01403A7
:10D97000142B05D1314A5146484680F0D3FB002490
:10D980005146484681F07EFA002188424FF06002FD
:10D9900002A808BF0C460191BAF008FFD6F8780239
:10D9A000036801AA1B6864219847054680B9244A88
:10D9B00001AB5146484680F0B5FB2C462546BDE7F5
:10D9C00062F08CFAA52163F08DFA0028C6D1CBE76E
:10D9D000002CF3D0D9F808303BB9D9F800305146C3
:10D9E0005B6B484698470446E8E751464846FFF7D0
:10D9F000D7FD514607464846FFF758FF3840C4B2A6
:10DA000051464846FFF790FD514604404846FFF70F
:10DA10005FFF51460440484680F0ACFB514604404D
:10DA2000484681F047FA0440C8E700BF385C002050
:10DA30006885002020D00C0837D00C0851D00C0885
:10DA400069D00C0808B5FFF761FF054A92F8481243
:10DA500060F3041182F84812024A907108BD00BFB9
:10DA6000385C00203D870020F7B505460F4680F062
:10DA700085F9044678B10221284680F043F906462C
:10DA800048B1154888F0AEFCC205C0F30723C0F3C7
:10DA9000002403D53446204603B0F0BD9B07F9D5DA
:10DAA0000D4888F0ADFC0D4B03F63463D3ED007ADE
:10DAB000F8EEE77A30EE670ADFED097AB0EEC00AD9
:10DAC000B4EEE70AF1EE10FAE4DD064B3A46022125
:10DAD000284680F01FF9DEE7A07A0020386C00208D
:10DAE0000000C84274D00C08F8B504460F4680F018
:10DAF000F7FB10210546204680F004F958B1204676
:10DB0000FFF71EFE064630B9044B3A461021204668
:10DB100080F000F935462846F8BD00BF88D00C08D3
:10DB200070B505460E4680F091F8044678B1802124
:10DB3000284680F0E7F850B1074B93F8153843B109
:10DB4000064B32468021284680F0E4F80024204627
:10DB500070BD0446FBE700BF385C00209CD00C0879
:10DB600038B50D4D0446D5F8900E87F0E3F801283E
:10DB700010D0D5F8900E87F0DDF8022804D02046AA
:10DB8000BDE8384080F064B804480FF03BFC012841
:10DB9000F5D138BD0020FCE7386C0020E082002081
:10DBA000F0B5134C04F5005385B0D3F83C2E009229
:10DBB000D3F8402E0192D3F8442E0292D3F8483E77
:10DBC00003936A4606460F4681F00EF9394605462C
:10DBD000304680F0F9F804F54054284094F8483273
:10DBE00060F3C303C3F3C00084F8483205B0F0BD4E
:10DBF000382C00202DE9F84306462748DFF8A89086
:10DC0000DFF8A8800F466EF011F80446D9F85402E8
:10DC100003681B699847054630B914F0060F03D115
:10DC2000D9F88832022B09D13946304680F09EF966
:10DC3000054618B9002488F807400AE039463046FE
:10DC4000FFF78AFD04460028F4D02DB9012388F897
:10DC500007302046BDE8F8830821304680F052F8AE
:10DC60000028F3D00D4822F0EFFB0028EED00C4B3B
:10DC700093F81424B02101FB023203F50053B2F8EB
:10DC80001E22B3F97A349A42E0DD064B3A46082167
:10DC9000304680F03FF8CDE7304F0020582D00206F
:10DCA000382C0020B0D00C08385C00203D870020C4
:10DCB0002DE9F3410E46054614F0D0FE804613F0E0
:10DCC000B5FF044640B9514A0121284680F02AFA9E
:10DCD000204602B0BDE8F0814D4FD7F854020368EA
:10DCE00031469B699847044658B9D7F854020368EF
:10DCF0001B6C9847474A03460121284680F012FAD8
:10DD0000E6E7AB68002BE3D0102128467FF0FAFF4E
:10DD100020B3D8ED937A98ED920A20EE270AB8F056
:10DD2000E3FADFED3D7AA7F5805320EE270AB3F939
:10DD30004C34DFED3A7A20EE270A07EE903AF8EEFF
:10DD4000E77AB4EEE70AF1EE10FA07DD344B012270
:10DD5000102128467FF0DEFF0024B9E74021284645
:10DD60007FF0D0FF38B3012E1ED0232E1CD0042EFE
:10DD70001AD02C4CD4F8443EB3F9083000EE103AD7
:10DD8000A4F50050B8EEC00A00F0C4FBB5EEC00A1E
:10DD9000F1EE10FA1DDD244B00930122234B4021AC
:10DDA00028467FF0B7FFD7E7D7F854020368DB6B4C
:10DDB00098470028DDD01E4B1B68D86A0368DB69D2
:10DDC00098470128014619D11A4A284680F0AAF935
:10DDD000C2E7D7F8540203685B69984730B1D4F8BA
:10DDE000443EB3F90830002BE5DDD4E7D7F8540200
:10DDF00003681B6898470B28DDD1F0E731462846B9
:10DE000002B0BDE8F04180F033BD00BFC0D00C08C7
:10DE1000385C0020D1D00C08E02E65420000C842DA
:10DE2000E5D00C08384C002037CE0C08EDD00C089B
:10DE300068850020F9D00C0870B505460E46FFF73E
:10DE40008BFC084B0446D87131462846FFF740FD4D
:10DE500031460028284608BF002480F0ADFE20404F
:10DE600070BD00BF3D8700202DE9F0414E4F3B784B
:10DE7000002B40F096804D4CD4F8785295F8CB505A
:10DE800001263E701DB13B702846BDE8F08181F04F
:10DE9000B9F8054630B9464A3870137843F00103A3
:10DEA0001370F1E757F026FB314656F05DFCA4F500
:10DEB000405006F01FFD3F4B1E710B264AF01AFD25
:10DEC000013E4AF0CDFC16F0FF06F7D13A4800F0CB
:10DED00095FF14F0C3FDD0F80022C4F8A02290F8FA
:10DEE0007C32DA074DD414F023F957F003FB3C21C0
:10DEF00057F03CFA0023C4F8603200212E482F4E20
:10DF000001F006F82C4811F089FD01462C488CF0F0
:10DF1000DBF92C4B1B68D86A036801211B68984702
:10DF2000D4F8780203689B6A98470121D4F87802F4
:10DF300089F012FA57F0DEFA8046D4F854020368EA
:10DF40001B68984796F80C240146404656F0E4FDBD
:10DF5000A6F5005006F0C0FC54F0BAFC53F0F6FFF2
:10DF600000233B7091F0DEF9B4F84A3206F5005612
:10DF700023F4087343F02003C6F89C0EA4F84A3239
:10DF800082E79B07B9D431460B4804F03DFD0E48AB
:10DF900088F036FADFED0D7A20EE270A84ED980A34
:10DFA000ABE7002570E700BF302C0020385C002074
:10DFB0005C8700203D870020382C0020384C002052
:10DFC0007C58002068850020A07A00200AD7233CD6
:10DFD0002DE9F043374DD5F8783293F8CB3087B040
:10DFE000002B64D062B1012901D0232908D195F911
:10DFF0004832002B04DB0024204607B0BDE8F08344
:10E0000081F0ACF804460028F5D014F027FD07464F
:10E010001AF0B8FE8046384613F012FBD8B198F9D2
:10E020002430022B17D100264FF00009F1B203AAC9
:10E0300038460191CDF80C90CDF81090CDF81490A1
:10E0400013F09CFE019918B103AA40461AF04AFB4E
:10E050000136032EEAD11848012106F0B5FE164814
:10E06000012106F0E5FD0021D5F8780289F074F968
:10E07000124832F0B9F957F03DFA002156F074FB1E
:10E080000F4B1B68D86A036800211B68984795F8F6
:10E090004A32D5F854120B486FF3451385F84A32CB
:10E0A0000B1A594259413C308FF0F4FAA4E701248D
:10E0B000A2E700BF385C0020382C0020647D0020DF
:10E0C00068850020007F002010B5064CD4F854026B
:10E0D00003685B6A984718B1D4F8783293F8CB009C
:10E0E00010BD00BF385C002030B52DED028B89B02B
:10E0F0000C46B0EE408AFFF7E7FF0546002838D00F
:10E10000B4EE488AF1EE10FA7CBFDFED1C8ADFED39
:10E110001C7A226863689FED1A0A68BFDFED198ACE
:10E12000029278BF68EE288A02A878BF68EEA78AB4
:10E13000D4ED027A0393F1EE677ACDED047A2FF0F5
:10E140004BF8B4EE488A00220123F1EE10FACDE933
:10E1500000238DED050ACDED060A9FED0A0A0A4857
:10E160008DED071AF0EE680A68BF134605A90DF099
:10E1700029FA284609B0BDEC028B30BDE02E65427D
:10E180000000C842000000008481002007B5019112
:10E19000FFF79AFF30B10199044803B05DF804EB32
:10E1A00000F0FCBA03B05DF804FB00BF382C00207F
:10E1B00001486DF0C7BE00BF304F002008B500F524
:10E1C000405090F84832C3F340128A420BD061F3BA
:10E1D000451380F8483231B157F08CF9BDE808405A
:10E1E0000F2157F0C3B808BD70B500F5405605467D
:10E1F000D6F888328B420C4611D0012910D0022962
:10E2000018D051B957F076F91B2157F0AFF80E4AE4
:10E2100006213046203059F077FAC6F8884270BDA2
:10E2200057F068F91A2157F0A1F8084A062105F5B8
:10E230004050EFE7012100F06BFE57F05BF91D2124
:10E2400057F094F8024AF1E764D10C0879D10C0830
:10E2500074D10C0810B500F540520C4692F86D329E
:10E2600003F00101A14209D064F3000382F86D328A
:10E27000DB0704D405F01CFF024B9C7210BD06F0B6
:10E28000EFF8F9E73D87002000F5405090F86D3237
:10E2900061F3410380F86D32014B1973704700BF81
:10E2A0003D87002010B5044661F018FE202162F081
:10E2B00019FE04F54053003893F84A2218BF012094
:10E2C00060F3820283F84A2210BD000010B50446B4
:10E2D00054F0FEFA04F54052436FD2F8782204F568
:10E2E0008044D360D4F8842E9366D4F88C2EC2F880
:10E2F000FC32D4F8840E03685B6D9847D4F8840E22
:10E300000368BDE810409B6D1847000070B52DED07
:10E31000028B00F540550446D5F8783293F8CB309F
:10E32000002B74D095F94832002B70DB00F5A04328
:10E3300093F85030002B6AD1D5F8540203685B691A
:10E340009847002863D1334BD3F8540203681B6805
:10E3500098470B285BD004F580469FED2F7AD6F8BE
:10E360008C3ED3EDDB7AF0EEE77AF4EEC77AF1EE8D
:10E3700010FA4CD5D5F87802443058F0EFFC03463B
:10E38000DFED260A93ED000A9F20B7EE001A2BF06E
:10E39000A3FCB5EEC00AF1EE10FA38DD04F59C409E
:10E3A000683088F039F8DFED1E7AB0EEC00AB4EEBE
:10E3B000E70AF1EE10FA2AD504F58054D6F8840E57
:10E3C000D4F8E03507EE903A0368D3F89830B8EE09
:10E3D000E78A984738EE400ADFED127AB0EEC00ABD
:10E3E000B4EEE70AF1EE10FA11D5D4F8E43540F2B4
:10E3F000E63203F2F313934209D8BDEC028BD5F851
:10E4000078029FED090ABDE870408AF027BABDEC9A
:10E41000028B70BD385C002000000034000000005A
:10E42000000070420000FA430AD7233C08B500F50B
:10E430004050D0F8780203681B699847F6EE007ADE
:10E4400020EE270AB5EEC00AF1EE10FA48BF9FEDA4
:10E45000010A08BD0000000038B52DED028B00F563
:10E4600080450446D5F8843EDFED110A93ED370A66
:10E4700004F540547120B7EE001A2BF02DFCD4F8AF
:10E480007802D5F88C5E03681B69B0EE408A984725
:10E4900038EE400ABDEC028BDFED067A05F5057516
:10E4A000284620EE270ABDE8384078F03FBC00BF80
:10E4B0000000000000007A4400F5805000F5C763BA
:10E4C00000F24460D3ED005AD2ED007AD0ED006A3C
:10E4D00091ED006A26EEE77A67EEA57AA6EE257A38
:10E4E000E6EE267A81ED007AC2ED007A70470000F0
:10E4F00000F50050B0F9F43C33B9B0F986040028B7
:10E50000B8BF404280B2704783EAE370A0EBE3708B
:10E51000F8E7000070B52DED028B00F5405382B096
:10E5200093F86D1211F00106044605D09FED2E0AF6
:10E5300002B0BDEC028B70BD8DED010A61F0CEFC26
:10E54000037F002BF2D0DFED298ADFED270A9DED56
:10E55000010AB0EE681A4E202BF0BEFB04F5005500
:10E560004FF4C8723146B5F98E04B0EE408A2BF0F4
:10E57000F1FBA5F88E04204610F0F6FFB5F98E34B5
:10E5800007EE900AB8EEE77A07EE903AF8EEE77AEF
:10E5900077EE676AB4EEE68AF1EE10FA0DD5204602
:10E5A000FFF7A6FF07EE900A38EE668AB8EEE70A94
:10E5B00020EE088A88EE260ABAE777EE877AB4EE6C
:10E5C000E78AF1EE10FAB1DDB5F9863400EE103AC3
:10E5D00038EE678AB8EEC00A78EEE77A20EE088A4D
:10E5E00088EE270AA4E700BF0000000000007A447C
:10E5F00000207047002070477047000000F512505F
:10E600001C307047004870474C010D0800F5405021
:10E61000D0F8540203681B681847000003480860DC
:10E620003121117008221A60704700BF20D50C08F4
:10E6300000F54050D0F854020368DB6C1847000026
:10E6400000F54050D0F8540203689B6C1847000056
:10E6500000F5405300F5A140D3F8543270301B1A36
:10E66000584258417047000010B500F540500C4624
:10E67000D0F854020368DB6D984707EE900A9FEDCF
:10E68000057AF8EE677A012067EE877AC4ED007AA2
:10E6900010BD00BF0AD7233C10B500F540500C4612
:10E6A000D0F8540203689B6D984707EE900A9FEDDF
:10E6B000057AF8EEE77A012067EE877AC4ED007AF2
:10E6C00010BD00BF0AD7233C10B500F540500C46E2
:10E6D000D0F8540203681B6E9847DFED047A20EEF1
:10E6E000270A012084ED000A10BD00BF0AD7233C91
:10E6F00066F05EBF63F0B6BC54F034B828F072BF69
:10E7000056F0B0B918F0C0B864F02CB861F040B859
:10E710005FF048B910F0C4BB11F01EB806F092BD0E
:10E7200012F040B805F018BD05F068BA05F08EB9D2
:10E7300068F0BEBC0FF004BDFFF7E8BD10F0F4BCFC
:10E7400010F062BF03F014B910F078BC10F0F0BB09
:10E7500061F012BB4BF0F6BA23F024B906F036B9DB
:10E7600002F0E2BC64F00EB810F06CBF06F020BD01
:10E7700004F036B906F070BE05F0FAB906F0D6B965
:10E7800010F01ABBFFF7A2BD29F01EBB05F0E6BED4
:10E790000AF048BA0AF032B90AF0C6B81FB500F557
:10E7A00040530446D3F85402039103685B6A9847C8
:10E7B00060B1DFED070A0399002304F5AA40009336
:10E7C000B0EE600A1A464C300CF052FD04B010BD99
:10E7D0000000000010B52DED028B00F540530446FB
:10E7E000D3F8540203685B6AB0EE408A984720B9B8
:10E7F0000024BDEC028B204610BD9FED080A04F5F5
:10E80000AA4028EE000A4C300BF0FCFF044600281A
:10E81000EED003480121FFF7D1FCEAE70000C8422F
:10E82000382C00200A4A92F94822002A0B4605DAC1
:10E8300000228A604A600A600120704700F580402B
:10E84000D0F8842E783207CA83E80700F4E700BFC7
:10E85000385C002070B5234B036000F5405304463C
:10E86000D3F8DC01204A1A6208B119F0C3FC1F4B2F
:10E87000236004F5005393F8C42042B9D3F8C05084
:10E880002DB1284627F03CFC284619F0AFFC04F5D2
:10E89000975010307EF080FC04F59550143063F0F2
:10E8A00015FE04F6E46504F68466B54204D0183D0E
:10E8B000284627F07BF8F8E70D4BC4F8C83804F673
:10E8C000282057F027FF04F6FC1057F023FF04F62A
:10E8D0005C1057F01FFF04F5136057F01BFF204634
:10E8E00070BD00BF04D90C08E0EA0D0884CB0D0808
:10E8F000B88C0D0838B54D4B044640F8043B66F023
:10E9000077FF04F1100017F061FC04F1680053F088
:10E91000B7FC04F5907021F0A7FC04F58C6016F0AC
:10E920006FF904F2845019F067FC04F6C80028F06F
:10E930009FFC04F5666066F039FD04F573604FF0E6
:10E940001BF904F58F5055F06FFE04F59450183004
:10E950006CF04EFC04F59550143063F09FFD04F507
:10E96000975010307EF004FC04F598500C3054F0B1
:10E9700049F804F59B5068F0E5F804F5805300254C
:10E980002B4A83F8845304F59C5004F59C530433BC
:10E990001430136049F0D8FD04F59F502946083023
:10E9A00012F034FB04F5D250103078F0FDFB04F582
:10E9B000FA5014307BF0FCFB04F501502C307DF054
:10E9C00031FD04F5035010307EF066F904F5045073
:10E9D000283012F01DF904F50A50083079F0B6F924
:10E9E00004F50B50134920304DF0F8FE04F50B50A0
:10E9F00038306CF0BFFF04F50E5034307EF054FF19
:10EA000004F5005304F5105083F80C540A4D2430DB
:10EA10007FF06CF82B6813B1084890F051FC204649
:10EA200007494DF0DBFE2C60204638BD84CB0D0835
:10EA3000EC900020CC910E081C88002088D10C0896
:10EA40008CCA0D0810B510F007FD61F047FA036895
:10EA5000BDE810405B681847FFF7F4BF10B50446E7
:10EA600006F0FEF8204611F003F8204603F008FEF9
:10EA70002046BDE8104003F069BF0000FFF7EEBF7D
:10EA800070B500F54A5524350446284617F078FA43
:10EA90001AF078F990F9213093B390F840337BB3B2
:10EAA00004F5405304F28456D3F87802443058F009
:10EAB00055F90346DFED130A93ED000A9F20B7EEE8
:10EAC000001A2BF009F994F9B835012B284608BF34
:10EAD00086ED0E0A002116F0E7FFDFED0B7A04F257
:10EAE000DC7494ED287A20EE270ADFED087AA7EE91
:10EAF000270A304684ED280ABDE870401AF052B863
:10EB000070BD00BF00000000CDCCCC3D6666663F06
:10EB1000FFF7B6BF10B50121044610F0E5FF60B164
:10EB2000114BD3F8540203689B6A984728B92046D2
:10EB300002F008FA204602F015FA4FF400112046C0
:10EB400010F0D2FF18B12AF055FB28F061FA4FF40B
:10EB50008021204610F0C8FF28B12AF04BFBBDE809
:10EB6000104028F059B910BD385C0020FFF7D2BF23
:10EB700070B500F580450446D5F8840E9FED5A0A1D
:10EB800086B06C302EF028FB04F59F5003A90830A6
:10EB90008DED030ACDED040A8DED051A12F0E2F8B1
:10EBA0000221204610F0A0FF70B10121204610F094
:10EBB0009BFF48B94D4BD3F8540203689B6A9847B2
:10EBC00010B9204602F0BEF90121204610F08CFF5A
:10EBD00048B9464BD3F8540203689B6A984710B96A
:10EBE000204602F0BFF90121204610F07DFF10B948
:10EBF000204602F00FFA4FF40031204610F074FF67
:10EC000030B104F54053D3F8780203685B6C984741
:10EC10004021204610F068FF60B104F58F5001904C
:10EC200055F0C0F804F58053019893F9B4320BB154
:10EC300055F0FAF94FF48061204610F055FF18B1F5
:10EC400004F58F5055F048F92021204610F04CFF74
:10EC500058B104F54056D6F8540203681B6998472A
:10EC600018B3D5F88C0E84F0C3FB8021204610F039
:10EC70003BFF38B32AF0BEFA28F0F2F81021204604
:10EC800010F032FF18B1D5F8840E81F0F7F84FF488
:10EC90000041204610F028FF18B304F59E402430B0
:10ECA00006B0BDE8704063F09FBE20460DF09AF9B3
:10ECB0000028D6D1D6F8540203685B69984700282B
:10ECC000CFD0D2E74FF48021204610F00DFF00286E
:10ECD000D0D14FF40021204610F006FF0028C9D102
:10ECE000CCE706B070BD00BFE02E6542385C002066
:10ECF000FFF73EBF10B50121044610F0F5FE10B13C
:10ED0000204602F087F98021204610F0EDFE58B130
:10ED10004FF48021204610F0E7FE28B92AF06AFA65
:10ED2000BDE8104028F078B810BD0000FFF7E2BF42
:10ED300010B5044605F0E6FC204605F031FB204600
:10ED400005F026FD204611F097FD2046BDE8104055
:10ED500003F072BCFFF7ECBF70B54FF6FF710446CD
:10ED600010F0C2FE04F5405528B1D5F8482207211D
:10ED7000204602F07FF9D5F8783293F8CB308BB982
:10ED80002046FFF78FFAD5F8780204F500530268A1
:10ED900093F8DC14166A93F8A224B047D5F87802E9
:10EDA00089F028FD62F088FE62F084FB204611F0B5
:10EDB00061FD95F848320F4A04F58044DB43D4F8EE
:10EDC000845EC3F3C01353712B681E6F53F080FD34
:10EDD00053F0E8F92846B047D4F88C4E53F078FD4C
:10EDE00004F5057453F0DEF92046BDE8704077F075
:10EDF00003BE00BF3D870020FFF7AEBF70B500F532
:10EE0000805606F5C76300F540541B68C4F88C3281
:10EE100006F2446305461B68C4F89032D6F8E8054C
:10EE200000F58C4050302AF02BFFD4F88C32C4F817
:10EE30009832D4F89032C4F89402C4F89C324FF659
:10EE4000FF71284610F050FE38B1D6F8E825284664
:10EE50000921BDE8704002F0E5B870BD30B500F59D
:10EE60004053D3F88842002C50D093F84922D10760
:10EE70004CD56FF3000283F8492200F50052012CB3
:10EE8000D2F83C1ED2F8405EB1F908400BBFD3ED7A
:10EE9000A45AD3EDA75AD3EDA37AD3EDA67A07EE01
:10EEA000104AB5F9084006EE904A0CBFF8EEE66A43
:10EEB000F8EEE66AB8EEC77A25EEE66A00F580500D
:10EEC000A7EE276A00F5C76300F2446067EEA67AF2
:10EED000D3ED006AE7EE257A90ED007A27EE877A87
:10EEE000A6EE267ABDEEC77A17EE104A0C8193ED96
:10EEF000007AD2F8402E67EE877A90ED007AE6EE3F
:10EF0000477AFDEEE77A17EE903A138130BD0000A4
:10EF100038B505462DED028B00F5405471B12846F9
:10EF200010F022F9D4F894321B1A03F2F31340F2D2
:10EF3000E63293420CD8BDEC028B38BDD4F888324F
:10EF4000022BF8D110F0F4F8B0F57A7FE7D2F2E7AF
:10EF5000C4F8940200F58C405030642390FBF3F326
:10EF600008EE103ADFED097AB8EEC88A28EE278A53
:10EF7000B0EE480AB6F0FEFF84EDA60AB0EE480AED
:10EF8000B7F04EF984EDA70AD5E700BF35FA8E3CFD
:10EF900000F59F500121083013F0C4BCFFF7F8BF03
:10EFA00010B5044610F0E6FA1021204610F09CFD42
:10EFB00070B1204601F020FF4FF40011204610F000
:10EFC00093FD28B92AF016F9BDE8104028F020B8C2
:10EFD00010BD0000FFF7E4BFF8B50446254606F073
:10EFE0006DF9224B45F83C3B214BA465C4E917342D
:10EFF000204BC4E91934204BE36604F1800018F07B
:10F0000069FD04F19C0018F065FD04F1B80018F0EA
:10F0100061FD4FF6FF76194BC4F8CC30A4F8D060F0
:10F0200004F1D40018F056FD4FF0FF37144B15498A
:10F03000C4F8307128461D604DF0D0FBA4F87870FC
:10F04000A4F8946004F5A27018F044FD04F5B070C3
:10F0500018F040FD04F5BE7018F03CFD002384F864
:10F060009031C4F8B4312046F8BD00BFEC2D0D0836
:10F0700091E7000895E7000899E700080000FFFF06
:10F080000C8700208C9A0D0810B5044606F016F97E
:10F090000A4B23600123A38704F1400018F01AFDF6
:10F0A00004F1500018F016FD04F1600018F012FD94
:10F0B00004F1700018F00EFD204610BD98360D08C2
:10F0C0002DE9F043044689B0FFF714FCA54B2360FB
:10F0D00004F51350083004F5005502F001F904F569
:10F0E00012531033C5F8503E04F53957062385F8FE
:10F0F000543E4FF07C5805A907F12000CDF814804C
:10F1000057F01EFF07F138008FF068FA04F59C46AF
:10F110000023683685F8903E04F53A50192304A977
:10F1200085F89C3EC5F8986E2830CDF8108057F0D1
:10F1300007FF04F53B508FF051FA4FF001081823F8
:10F1400004F53B5004F53D5785F8E43E85F8D88E2C
:10F15000C5F8E06E2037383062F0B2FD38467EF0F8
:10F1600081FD06AE804BC5F8603F3146381D8DF8F5
:10F1700018804EF051F904F53E5018304AF0A0FDC9
:10F1800004F53F5018307EF057FD784BC5F8D83F56
:10F1900004F53F50764D06953146303057F0D0FE9D
:10F1A00004F53F5031463C30069557F0C9FE04F552
:10F1B00040500695314604F54055083057F0C0FEE2
:10F1C00005F120086B4B2B6208F114008FF006FA52
:10F1D00004F5415704F54259183709F13C093846FE
:10F1E00014375CF0A7FCB945F9D10723C5F8E03125
:10F1F0000023A5F8E4314FF4CB7018F0F5FFC5F803
:10F20000DC0104F5475028308FF0E8F904F5485048
:10F210002C308FF0E3F9584B1A680AB9C3F8008014
:10F2200004F5AE47554B2B62343704F54950C5F809
:10F23000547218307FF0B2FF514B07934FF07E5855
:10F24000504BC5F88C82C5F898820694009304F55B
:10F250004A5096E80C004FF40071243016F0CCFAB6
:10F2600004F56050183070F09BFD04F59C4003A934
:10F270003830CDF80C8057F089FE04F59C4003A986
:10F280004C30CDF80C8057F05BFE04F59C4004F543
:10F290008045583018F01EFC05F6686300261E6095
:10F2A0005E609E6005F6746304F59D401E605E60BE
:10F2B0009E6004F59F530833C5F8803E002385F80F
:10F2C000A13E4FF40041243017F064F804F59E404D
:10F2D000243063F031FA04F59F4028306EF064FC6E
:10F2E00004F59F4064304EF0CDF9274BC5F8E43F5C
:10F2F00004F59F40254B2649783004F5A04504F5D8
:10F30000A048186008F118084DF068FAFF2385F846
:10F31000283085F830301F4940464DF05FFA1E4ACC
:10F32000136813B11D488FF0CBFF1D491D48C2F86B
:10F33000008004F5A042403208604FF0140E1FFA1E
:10F3400083FC0EFB0C010133097C0029F7D1164B1D
:10F35000A3F800C0154BD3F80080B8F1000F29D0F6
:10F360001348E0E704D90C0810D10C0850D10C0860
:10F370000000A040E0EA0D08608B002084D90C0852
:10F380008DE70008F4D80C0860D10C08F490002038
:10F3900038FD0D0858900E08849100209CD10C086F
:10F3A000DC870020581B0D08DA8700209887002092
:10F3B000BDD10C0804F5A0401A6003A94C4B03937F
:10F3C000543057F0BDFD04F5A040743005F076FFD1
:10F3D000484B6B6704F5A140343005F06FFF04F52E
:10F3E000A549454BC5F8B43004F5A14009F14809D9
:10F3F0007030FFF7F1FD484605F060FF3F4BC5F860
:10F40000C83209F13C008CF0CDFD3D4BC5F804330A
:10F4100004F5A940083005F051FF3A4BC5F888348F
:10F4200004F5A94085F8C484483005F047FF364B01
:10F43000C5F8C83404F5AA40043005F03FFF334B4B
:10F44000C5F8408504F5AA40C5F804354C3005F0F0
:10F4500035FF2F4BC5F84C3504F5AB40C5F8888512
:10F46000103005F02BFF2B4BC5F8903504F5AB4061
:10F47000583005F023FF284BC5F8D83504F5AC40CB
:10F48000143005F01BFF254BC5F8143605F28C63CC
:10F4900004F5AD401E605E602830FFF7F5FD38468C
:10F4A00005F00CFF1E4BC5F8343704F5AE40703044
:10F4B00005F004FF1B4BC5F8703704F5AF40A5F805
:10F4C000AC874030FFF7E0FD174BC5F8C03701238C
:10F4D00085F8493805F5056504F5B0402E606E6085
:10F4E000AE605C300AF04AFA204609B0BDE8F0830D
:10F4F000CDCC4C3DE4290D08882A0D08902E0D082E
:10F50000202F0D08DC2F0D087C300D08B8320D08B7
:10F5100058330D08E8330D0880340D0820350D08E8
:10F52000F4370D0890390D0850370D0838B5054BE4
:10F530001C6823680A461D68034B01462046A847FD
:10F54000002038BD68850020382C002010B58FF0D1
:10F550000BFB064C064B18602046FFF7B1FD20461A
:10F56000044A0549BDE81040B6F0DEBB382C002047
:10F570006885002084EA002055E8000801207047D3
:10F5800090F89C308B4286BF283150F82100002033
:10F590007047000090F89C308B4286BF283150F8AD
:10F5A0002100002070470000FA207047014B93F8BB
:10F5B00052047047384C0020034BD3F88802431E96
:10F5C00058425841704700BF385C0020034BD3F8C5
:10F5D0008802831E58425841704700BF385C0020A3
:10F5E000034BD3F8780208B187F0AEBF01487047EB
:10F5F000385C002070D90C0838B5C36A2E4D43F42E
:10F60000E052C262026B42F4E0520263426B42F487
:10F61000E0524263D5F88C2E0446E2B143F4F8433D
:10F62000C362D5F88C0E83F0A3FA38B1236B43F490
:10F6300080432363636B43F480436363D5F88C0E8C
:10F6400083F0B8FB38B1236B43F400532363636B3F
:10F6500043F400536363194B1D6845B119212846D3
:10F660004EF064FB18B1E36A43F48073E362144B19
:10F6700093F8583E6BB1236B43F48073236345B119
:10F68000192128464EF08AFB18B1636B43F480734E
:10F690006363E36A43F08043E362236B43F0804398
:10F6A0002363084BD3F8783293F8C1301BB9636BEE
:10F6B00043F08043636338BD386C0020E887002046
:10F6C000384C0020385C002013B54FF44470CDE96D
:10F6D000002118F083FD044628B1DDE900215FF028
:10F6E00035F9024B2360204602B010BDC8DB0C0880
:10F6F00000207047704700000320704708207047C3
:10F70000014B93F854047047384C0020034B93F995
:10F71000D304003818BF0120704700BF384C0020C8
:10F72000014B93F956047047384C00207047000095
:10F730007047000008B50C4BD3F88C0E70B910233D
:10F740000A4AD2F8782243F0400022B192F8CB2046
:10F750000AB143F0C00040F0010008BD83F008FA90
:10F760000028ECD01823EBE7386C0020385C002030
:10F7700038B5C5780B46352D044628BF35253522CA
:10F7800000211846B9F012F82A4604F10C01BDE830
:10F790003840B8F0C1BF00001FB5184C94F876127D
:10F7A00004F5947011F01EFA78B194F8761204F50D
:10F7B000947011F019FA40B194F8761204F594702F
:10F7C00004B0BDE8104011F011BA00230193029378
:10F7D000039313F043F901A912F00CFF20B101A823
:10F7E0002EF0F8F804B010BD22F01AF990F8F432B7
:10F7F000B02202FB030090ED3B0AF3E7384C0020F7
:10F8000008B50D4BD3F87802A8B1443057F0A6FAEA
:10F81000034693ED000ADFED090A9F20B7EE001AB8
:10F820002AF05AFADFED067A20EE270ABDEEC00A6A
:10F8300010EE103A18B208BD385C0020000000003D
:10F840000000C8422DE9F04FDFF8D880344F8DB06A
:10F850000446042508F5005617F8019BB8F9AC34A6
:10F8600009F1FF3A43FA0AF3D90742D5207C58F050
:10F8700015FF8346207C59F015FE00F121039B45BE
:10F8800005D2207C0DB0BDE8F04F58F05DB9BAF15B
:10F89000030F2ED8DFE80AF00234393ED6F8840E82
:10F8A00003689B68984700F194035A69D3F800A055
:10F8B000D3F804E0D8681969D3F818C008925A6AD6
:10F8C0001B6ACDF82520CDF8293062222123CDE90D
:10F8D000003206900791207CCDF80CA0192303AAD2
:10F8E000C221CDF810E0CDF814C08DF8249058F066
:10F8F0003FFF013D15F0FF05AED10DB0BDE8F08F23
:10F90000D6F8840E0368DB68CCE7D6F8840E03686B
:10F910001B69C7E7D6F88C3E03F52A73C5E700BF1D
:10F920009CDC0C08384C002013B5044607480191B4
:10F9300008F0ACFF30B90199204602B0BDE8104094
:10F9400059F0F0BF042002B010BD00BF287D002098
:10F95000014808F077BD00BF287D002037B5044678
:10F960000D460648019211468BF0E0F8019A2946AF
:10F97000204603B0BDE830405DF0B4BE38590020E9
:10F9800010B588B004465BF0CBF90C4BD3F8780285
:10F9900038B90B4A0621204608B0BDE810405BF09C
:10F9A000A7B969461E2287F0D3FD064A6B46062199
:10F9B00020465BF09DF908B010BD00BF385C002008
:10F9C000BCD90C0862270D08034A92F8383E01336F
:10F9D00082F8383E5AF068BA384C002007B508461D
:10F9E000019118F04DF938B10448019902F0C0FCBA
:10F9F000002003B05DF804FB0420FAE774850020C2
:10FA0000F7B58B8BCD2B06460C4617461DD1D1ED95
:10FA1000067AFCEEE77ACDED017A9DF80430022BF0
:10FA200013D10E4D95F89D1F05F6247062F0BAFEB5
:10FA300058B195F89D1F05F6247062F0BBFE20B901
:10FA400094ED020A064802F073FC3A46214630461D
:10FA500003B0BDE8F0405AF0B9BA00BF386C0020DE
:10FA600074850020162A10B40C4605D0542A03D001
:10FA70005DF8044B59F072BF0323237001205DF839
:10FA8000044B704708B55AF0C5F940F41C6040F0CB
:10FA90000D0008BD10B5044618F0A8FB204610BDA7
:10FAA00010B50C4C94F94832002B0FDBD4F85402FB
:10FAB0000368DB6C984758B9D4F8540203689B6C10
:10FAC000984700280CBF0220032010BD0120FCE74E
:10FAD0000420FAE7385C002010B44C69012C05D1F1
:10FAE00001465DF8044B034802F0D6BF5DF8044BB5
:10FAF0005AF0F4B9382C00202DE9F341B1F9043063
:10FB0000002B06460C46154635DB4FF00008CDE9C4
:10FB100000281A4FB1F902209FED190AD7F83C1EB0
:10FB20004FF47A735EF0C6F80123CDE900539FEDE0
:10FB3000140AB4F90020D7F8401E4FF47A73304607
:10FB40005EF0B8F89FED0F0AB4F90420D7F8441E10
:10FB500043463046CDE900585EF0ACF8CDE9005898
:10FB60009FED070AB4F90620D7F8481E4FF47A73C0
:10FB700030465EF09FF802B0BDE8F081384C0020BE
:10FB80000000FA4400007A44044B187820B9044B72
:10FB900093F84A02C0F38010704700BFE08600204F
:10FBA000385C00200B4B93F815287AB993F86D2236
:10FBB00092060BD193F94822002A09DB93F84932C7
:10FBC00013F0200F14BF0420012070470520704758
:10FBD00003207047385C002008B5074B93F9A03428
:10FBE000032B03D0BDE808405BF0FAB8034A0221BA
:10FBF0005BF07EF8042008BD384C0020D4D90C08F6
:10FC0000094BD3F8D424920701D459F09BBE03F5D5
:10FC1000005303F65C6393ED000ADFED047AB8EE5F
:10FC2000C00A20EE270A7047384C00200AD7233C30
:10FC300010B594B0044603A817F04CFF1C4BD3F842
:10FC40005402036803A95B6D984778B3002103A8A9
:10FC500017F0D8FF50B3247C8FF064FB059BDDEDDB
:10FC6000047A0893069B09930023F8EEE77A9FED48
:10FC7000117A0B930C930D930E930F931093119392
:10FC800012934FF6F853ADF84C300023962267EEEE
:10FC9000877A8DF84E303323CDE90032079007AADA
:10FCA00057212046CDED0A7A58F062FD14B010BD00
:10FCB000385C00200AD7233C30B52DED0A8B774CF9
:10FCC0000546D4F85402036899B05B6A9847002847
:10FCD0005BD004F50054D4F88835062B00F2C980B7
:10FCE000DFE803F00404045788AB53006C489FED31
:10FCF0006D8A0BF085FC9FED6C0A01684268836891
:10FD00000D930BA80B910C922DF066FAF0EE489A29
:10FD1000B0EE40CAF0EE60BAB0EE419AB0EE48AA3A
:10FD2000F0EE488AF0EE48AAB0EE48BA40F6F85431
:10FD30002D7C8FF0F7FA00231593169301238C2264
:10FD40008DF85E303323CDE900320B90B1EE499A45
:10FD5000F1EE688AB1EE488A0BAA552128468DED4E
:10FD60000CCACDED0DBA8DED0E9A8DED0FBACDED1D
:10FD700010AACDED118A8DED12AACDED139A8DED5D
:10FD8000148AADF85C4058F0F3FC19B0BDEC0A8B56
:10FD900030BD43480BF034FC9FED430A01684268D4
:10FDA00083680D930BA80B910C922DF015FA3C482B
:10FDB000F0EE60BAB0EE419AB0EE40CA0BF024FC0F
:10FDC0009FED390A2DF008FA3548B0EE40BAF0EE52
:10FDD00060AAF0EE418A0BF01BFC9FED330A2DF078
:10FDE000FBF94FF44064B0EE40AAF0EE609AB0EE3A
:10FDF000418A9DE72A489FED2B9A0BF005FC9FED69
:10FE00002A0A2DF0E9F92648B0EE40BAF0EE60AAD1
:10FE1000F0EE418A0BF0FCFB9FED230A2DF0DCF99C
:10FE2000F0EE49BAB0EE40AAF0EE609AB0EE418A28
:10FE3000B0EE49CA40F607447AE71948DFED198A5F
:10FE40000BF0E6FB9FED180A2DF0C6F9F0EE68AA5C
:10FE5000B0EE40AAF0EE609AB0EE418AB0EE68BA19
:10FE6000B0EE689AF0EE68BAB0EE68CA40F63F4469
:10FE70005EE79FED0C8A0024F0EE489AB0EE48AAA7
:10FE8000F0EE488AF0EE48AAB0EE48BAB0EE489AD2
:10FE9000F0EE48BAB0EE48CA4AE700BF385C00202E
:10FEA00084810020000000000AD7233C2DE9F041A6
:10FEB0002DED068B3B4D95F8493299068CB00446E2
:10FEC0006AD505F580579FED380AD7F8840EDFED27
:10FED000378A6C302DF080F98DED041A21EE281A46
:10FEE000D5F854628DED020ABDEEC11ACDED030ABC
:10FEF00011EE103A1DB2336894F810809B6D3046B5
:10FF000060EE289A20EEA89A984707EE900AF8EE3D
:10FF1000E77A304667EEA87AFDEEE77A17EE903A78
:10FF20001CB23368DB6D984707EE900AB8EE678A1B
:10FF3000D7F88C3EDFED1E7A93ED0FAA336828EEDA
:10FF4000288A1B6EB4EEE78AF1EE10FA58BFB0EEC5
:10FF5000678A30469847BCEEC88A0023089318EE9B
:10FF6000103AB7222AEE28AA20EE280AADF82C3043
:10FF70001A23CDE900323E2105AA4046CDED059A6F
:10FF80008DED069A8DED07AA8DED090AADF8285082
:10FF9000ADF82A4058F0ECFB0CB0BDEC068BBDE888
:10FFA000F08100BF385C00209F0CB3450AD7233C8A
:10FFB00000FF7F472DE9F04F2DED028B1A4B047C9B
:10FFC000D3F8843E8DB0D3F88480D3F88870D3F80A
:10FFD0008C60D3F8905093ED258AD3F898B0D3F87D
:10FFE0009CA0D3F8DC908FF09DF900238DF82C3085
:10FFF00016222523CDE90032029002AA5321204681
:020000040801F1
:100000008DED078ACDF820B0CDF824A0CDF828904A
:10001000CDF80C8004970596069558F0A9FB0DB015
:10002000BDEC028BBDE8F08F386C002070B58A7A89
:100030004B7A43EA0223CA7A43EA02439D2B0646DF
:100040000C4621D1134D95F89D1F05F6247062F0E2
:10005000A9FBC8B195F89D1F05F6247062F0B6FBA8
:10006000022811D195F89D1F05F6247062F0A2FBBD
:1000700050B9D4ED057A9FED080A0848F8EEE77A02
:1000800027EE800A02F054F921463046BDE8704060
:1000900059F00ABE386C00200AD7233C7485002032
:1000A000054BD3F878322BB193F8CA00002808BF6B
:1000B0000220704702207047385C002008B5034BCF
:1000C000D3F8540203681B68984708BD385C0020C9
:1000D000024B93F84902C0F340107047385C00208F
:1000E00070B52C4E2DED028B0546D6F8540291EDDD
:1000F000018A036886B05B6A0C46984750B9BDEE2A
:10010000C88A18EE103ADB0704D4022006B0BDEC12
:10011000028B70BDD4E904012AF0B8FE0028F4D0A7
:1001200002A817F0D7FC02AA214628465DF032FD4E
:100130000028EAD0184902A817F0AEFD03460028AF
:10014000E3D1DFED160A00900246B0EE600A1448D3
:1001500002A90BF08DF8D8B1D6F8540203685B6A97
:100160009847044608B10020D0E70E480222042137
:1001700005F032FC60B1DFED090A0948009423461E
:10018000B0EE600A224602A90BF072F80028EAD10C
:100190000420BBE7385C0020907A002000000000BB
:1001A00084810020382C002008B591F82030032BE2
:1001B0001CD1D1ED027A9FED0E7A91ED060A0D4B1E
:1001C000F0EEE77AF4EEC77ADFED0B7AD3F854025B
:1001D000F1EE10FA4CBF0121002120EE270A0FF0AA
:1001E0009FFF002814BF0020042008BD0220FCE768
:1001F00000000034385C00200000C84210B52DED2E
:10020000028BD1ED007AF5EEC07AF1EE10FA82B0F1
:100210000C4604DA042002B0BDEC028B10BD9FED49
:10022000197AF4EEC77AF1EE10FAF3D891ED030AD9
:100230009FED158AF0EEC07AF4EEC87AF1EE10FA6E
:1002400019D5D4ED037A1148D4ED010A94ED000AD2
:10025000F4EEC87AD4ED027AFDEEE77AF1EE10FA08
:10026000CDED017A9DF90410ACBF0122002201F00E
:10027000C1FF0020CFE7F7EE000A29F029FC002893
:10028000C8D0DEE70000B4430000003474850020CD
:1002900091ED010AB5EEC00AF1EE10FA08B501DCE5
:1002A000042008BD9FED107A104BD1ED007AD3F8F1
:1002B000540220EE070A9FED0E7A0368F4EEC77A27
:1002C000F1EE10FA05DDDB6E98470028E8D000203B
:1002D000E7E79FED087AF4EEC77AF1EE10FACCBFAB
:1002E0009B6E5B6EF0E700BF0000C842385C0020E8
:1002F0009A9939403333F33F08B5D1ED007A9FED39
:10030000157AF0EEE77AF4EEC77AF1EE10FA1DD521
:10031000D1ED017AF0EEE77AF4EEC77AF1EE10FA59
:1003200014D50D480222032105F056FB80B10A487E
:100330000121FDF743FF094890F83031012B03D02C
:1003400000F5967030F0A6FA002000E0022008BD0B
:100350000420FCE700000034382C0020387C00200A
:1003600010B5D1ED007AFCEEE77A17EE903A9CB228
:10037000012C02D0022C06D04CB90648214667F069
:1003800019F8002010BD044803F046F9F9E70420ED
:10039000F8E700BF307C0020382C00201FB5D1EDDD
:1003A000017A0B7CFCEEE77ACDED027AD1ED007A92
:1003B0000093FCEEE77AD1ED030ACDED037A91EDDF
:1003C000020A9DF808309DF80C20014602480EF004
:1003D00059FC05B05DF804FB382C002010B50A4C20
:1003E00094F86D32DB070CD402220521A4F54050AD
:1003F00005F0F2FA28B902221146A4F5405005F0A2
:10040000EBFA002010BD00BF385C002010B5D1ED24
:10041000007AFCEEE77A044617EE903A13F0FF03F9
:100420000FD10F4BD3F8540203689B6F984708B164
:10043000002010BD0B4A204606215AF059FC04202A
:10044000F7E7012B09D1064BD3F854020368DB6FA1
:1004500098470028ECD1044AEDE70220E9E700BF05
:10046000385C0020F8D90C0808DA0C089FED0B7AEC
:1004700001F10C03F1EC017AF4EE677AF1EE10FA77
:100480000AD6F0EEE77AF4EEC77AF1EE10FA03DC62
:100490009942EFD1012070470020704700007A4454
:1004A00030B52DED028B8DB00023054603930493E8
:1004B000059312F0D3FA03A912F09CF858B312F086
:1004C000CDFA00F55A7393E8070006AC84E80700FC
:1004D000DDED060A9DED070A2D7CF1EE600AB1EE16
:1004E000400AB5F069FF2046B0EE408A2DF072FA5E
:1004F000DFED0B7A089B0B93012228EE278A0C2351
:10050000CDE90032A82109AA28468DED098A8DED92
:100510000A0A58F02DF90DB0BDEC028B30BD00BFBA
:10052000E02E6542242938B505460FD003D81B2993
:1005300007D1012412E04029FBD0A1F14203012B95
:10054000F7D92846BDE838405DF010BD0C2157F0C2
:100550000DFB044610B12846FFF7A2FF204638BD28
:1005600038B5194C94F86D32DB070D460AD4D4F82F
:10057000783293F8CB303BB901221146A4F1A000A8
:10058000FDF772FC002038BD94F94832002B4FF083
:10059000020212DA0521A4F5405005F01DFA0028E8
:1005A000F0D095ED000ADFED097AD4F8540220EE80
:1005B000270A01210FF0B4FDE4E70921A4F540501A
:1005C00005F00AFADEE700BF385C00200000C842F0
:1005D00010B51B4C94F86D32DB070ED4D4F878328A
:1005E00093F8CB304BB194F94832002B07DA012253
:1005F0000821A4F1A000FDF7EBFC002010BDD1ED17
:10060000007A9FED107AF0EEE77AF4EEC77AF1EE19
:1006100010FA05D5022211460B4805F0DDF9ECE78A
:10062000D4F8540203681B6898470428E5D0D4F82E
:10063000540203681B6898471428EBD1DDE700BF1C
:10064000385C002000000034382C002073B58B8B00
:10065000C12B05460C4644D8BB2B0DD8202B63D0AC
:100660002ED8113B99B2052918D92146284602B047
:10067000BDE870405EF06EBDBC3B052BF5D801A116
:1006800051F823F0C3070108CD0701086B060108E4
:100690006B0601085B07010867070108052BE4D812
:1006A00001A151F823F000BFA90701086B0601085A
:1006B0006B060108BD070108CF0601087D07010888
:1006C000732B2CD006D8542B58D0552BCDD10222C9
:1006D00009216BE0B22BC8D102B0BDE87040FFF732
:1006E000D7BD4AF21146B34254D00BD8D12B40D0DB
:1006F000B3F5967F53D0D02BB7D102B0BDE8704090
:10070000FFF72EBE4AF21246B3423ED04AF21346DB
:10071000B342AAD102B0BDE87040FFF759BF02B0A2
:10072000BDE87040FFF76ABDD1ED007AF5EEC07A02
:10073000F1EE10FA4FDD9FED297AF4EEC77AF1EE73
:1007400010FA48D8FCEEE77A254ACDED017A9DF8FB
:100750000430A2F8023D00202EE0214602B0BDE8A0
:100760007040FFF7BDBC214602B0BDE87040FFF706
:100770004DBE02B0BDE87040FFF710BE21462846CE
:1007800002B0BDE87040FFF70FBD02B0BDE8704099
:10079000FFF7E6BE02B0BDE87040FFF71FBE02B033
:1007A000BDE87040FFF7A8BD022205210D4805F005
:1007B00013F90028CFD1042002B070BD0222062117
:1007C000F4E70221084806F085FAF2E7022106481C
:1007D00006F04AFAEDE70220EEE700BF00007F4393
:1007E000384C0020382C0020287D002008B591EDE1
:1007F000007AF6EE007AB4EEE77AF1EE10FA06DD52
:10080000044801220521FDF7E3FB002008BD042078
:10081000FCE700BF985B002030B52DED028BCD7852
:1008200093B0272D28BF27250C462722002108A892
:10083000B7F0BCFF2A4604F10C0108A8B7F06CFF22
:10084000424BD3F8540203685B6A9847002841D0B2
:100850009DF8465068063DD400244FF07E5329068B
:10086000049307940694059427D504A82BF05EFF03
:10087000EA0701940294039405F006032ED4002B9A
:100880002ED10D9B01930E9B02930F9B0393304837
:100890000AF09CFA9DED100A044630B340F2ED4098
:1008A000B7EE001AFFEE000A29F016FA2848234690
:1008B00001AA04A90AF092FA0CE0099B04930A9B8E
:1008C00005930B9B069304A80C9B07932BF034FF16
:1008D0000028CDD113B0BDEC028B30BD062BD6D095
:1008E00001211B480AF00EFAF4E7DFED1A0A4FF473
:1008F0009E60B7EE001A29F0EFF9F6EE000AB0EEAE
:10090000408A29F0E5F8E8B9B6EE000A124BB4EED9
:10091000C08AF1EE10FAD3F8903E08DD38EE400AB6
:1009200030EE008A93ED070A28EE000ABEE730EEAB
:10093000480AD3ED087A30EE000AF0EEE77A27EEA7
:10094000C00AB3E79FED030AB0E700BF385C0020A0
:100950008481002000000000386C00202DE9F04365
:100960009DB0814608460EA9FEF702FF844BD3F8DE
:10097000540203685B6A984750B19DF86C30012BB4
:1009800009D0DA1F022A06D97E4801210AF0BAF9F5
:100990001DB0BDE8F083BDF86840A20504F007066D
:1009A00004F0380704F4E07501D5002DF0D04FF0C5
:1009B0000008CDF81480CDF81880CDF81C803EBB1F
:1009C0009FED716A9DED107ADDED117ADDED0F6A14
:1009D00027EE067A67EEC67A66EE866A083B012B3A
:1009E000CDED056A8DED067ACDED077A04D867481E
:1009F00006AA05A9FDF760FD9DF86C30073B022BA8
:100A000006D8634885F0F8FC014605A82CF004FCE4
:100A1000CDF82080CDF82480CDF82880F7B9DDED21
:100A2000147A129B0893F1EE677A139B099308A935
:100A30004846CDED0A7AFFF719FD0028A4D09FEDB6
:100A4000520A08A82CF01CFC9DF86C30083B012BC6
:100A500004D84E4809AA08A9FDF72EFDCDF82C8030
:100A6000CDF83080CDF83480EDB99FED476A9DED2B
:100A7000167ADDED177ADDED156A9DF86C3027EEFC
:100A8000067A67EEC67A66EE866A083B012BCDEDE4
:100A90000B6A8DED0C7ACDED0D7A04D83B480CAA8B
:100AA0000BA9FDF709FD14F4806233D1DFED397A2B
:100AB0009DED180A9DF86C1020EE270ADFED327AC2
:100AC0000839012920EE270A8CBF0021012114F4E6
:100AD000006305BFDFED2F7ADDED190ADFED2E0A89
:100AE00060EEA70A04BFDFED287A60EEA70AAEB970
:100AF000002F35D1B3FA83F3B2FA82F25B095209BF
:100B00000291019300920BAB08AA05A91D480AF0B7
:100B100067FA3DE79FED200A0021D8E77FB9B3FAD5
:100B200083F35B0901200093B2FA82F3CDE901104F
:100B30005B0914480BAA08A90AF0EAFC28E7002D73
:100B40007FF422AF0120B3FA83F3B2FA82F2CDE947
:100B500000105B090B4852090BA90AF081FC17E74A
:100B6000002D3FF411AFB3FA83F3B2FA82F2CDE96C
:100B700000165B09520905A902480AF0B3FA07E713
:100B8000385C0020848100200000C842382C0020FE
:100B9000A07A0020E02E6542000000002DE9F04719
:100BA000A2B08046084614A9FEF7E2FD7E4BD3F8BA
:100BB000540203685B6A9847C0B1BDF88040A30542
:100BC00004F0070904F4E07700D57FB10CAE30469D
:100BD00016F080FFB9F1000F29D1DDE915012AF0E7
:100BE00055F930B9714801210AF08CF822B0BDE8FE
:100BF000F0879DF8841009AA40465CF0B5FF0028F4
:100C0000F0D0DDED177A9FED6A7A099B009367EECD
:100C1000877A10ADFDEEE77ADDE9151217EE903A0E
:100C2000284616F077FF95E80F0086E80F000025AC
:100C300014F0380A06950795089514D1DDED1A7A57
:100C4000189B0693F1EE677A199B079306A9404615
:100C5000CDED087AFFF70AFC0028C3D09FED540AB7
:100C600006A82CF00DFB09950A950B959FB99FEDF1
:100C7000506A9DED1C7ADDED1D7ADDED1B6A27EED5
:100C8000067A67EEC67A66EE866A8DED0A7ACDED53
:100C9000096ACDED0B7A14F4806805BFDFED457A63
:100CA0009DED1E0A9FED440A20EE270A04BFDFEDEA
:100CB000407A20EE270A14F4006405BFDFED3D7A88
:100CC000DDED1F0ADFED3C0A60EEA70A04BFDFED91
:100CD000387A60EEA70AB9F1000F31D1BAF1000FEE
:100CE00052D13046CDED050A8DED040A16F022FFF3
:100CF00003289DED040ADDED050A3FF473AF10A94A
:100D00003046CDED050A8DED040A1095119512952A
:100D100017F070F800283FF465AFB4FA84F4640962
:100D2000B8FA88F3DDED050A9DED040ACDF804A0BC
:100D300000945B0906AA10A91C480AF0C1F955E7FE
:100D4000BAF1000F0FD10123B4FA84F4CDE901A365
:100D50006409B8FA88F3154800945B0909AA06A942
:100D60000AF0D6FB42E7002F7FF43CAF0123CDE928
:100D70000073B8FA88F2B4FA84F30C485B0952099C
:100D800009A90AF06DFB31E7002F3FF42BAFB4FA4D
:100D900084F3B8FA88F2CDF800905B095209314625
:100DA00002480AF065FA21E7385C002084810020BF
:100DB0000000C842E02E65420000000010B44B7AEB
:100DC0008C7ACA7A43EA042343EA0243542B07D0BD
:100DD000562B09D0522B0BD15DF8044BFFF71CBDED
:100DE0005DF8044BFFF7BABD5DF8044BFFF7D6BEC4
:100DF0005DF8044B5DF088BB2DE9F0432DED028BCF
:100E000000F540560446D6F85402DFED4B8A0368DD
:100E100091B05B69984704F580490027002840F0AD
:100E20008780D9F88C3ED3EDDE7A93EDD88AFDEE3B
:100E3000E77A28EE288A17EE903A1DB204F53B585F
:100E400008F1280801A940460EF002FD18B954F037
:100E500051FB3A4B01933722002102A8B7F0A6FCC0
:100E6000A3238DF8083095238DF809308EF062FAAF
:100E7000D9F8843ECDF80B00D6F87802D3F8DC2000
:100E8000D3F8E030CDF80F104430CDF81320CDF872
:100E9000173055F063FF0346DFED290A93ED000A92
:100EA000B7EE001A9F2028F017FF10EE103AD6F880
:100EB0007802CDF81B3003681B69984710EE103A92
:100EC00004F59C46CDF81F30683618EE103A3046CF
:100ED000CDF8233085F094FA20EE280A404610EE33
:100EE000103ACDF82730D9F8343ECDF82B30019B9D
:100EF000CDF82F300EF0CEFC10EE103A3046CDF883
:100F00003330CDF83770ADF83B5085F085FABDEE43
:100F1000C00A372210EE103A02A904F58F50ADF83E
:100F20003D3053F039FC11B0BDEC028BBDE8F083CD
:100F300008EE107A002581E70AD7233C2292CA7F67
:100F40000000000010B500F58044D4F8840E7EF057
:100F50003FF9D4F88C1ED4F8840EBDE810407EF022
:100F60009DB9000070B54FF4805104460EF0BCFDF1
:100F700000284ED004F5804604F58F55D6F8840E2F
:100F800003689B689847692100F19402284653F052
:100F90009BFAD6F8840E0368DB6898476A2100F153
:100FA0009402284653F090FAD6F8840E03681B6921
:100FB00098476B2100F19402284653F085FAD6F841
:100FC0008C2E6C21284602F52A7253F07DFA2021DE
:100FD00020460EF089FDE0B104F54053D3F85402E9
:100FE00003681B69984778B1D6F88C2E2846903252
:100FF0006E2153F069FAD6F88C2E2846BC32BDE833
:1010000070406F2153F060BA20460AF0EBFF0028D1
:10101000EAD170BD08B511F021FDBDE8084011F01E
:101020009BBA00007FB50E464FF6FF710446154689
:101030000EF05AFDE0B1102200216846B7F0B6FB71
:10104000A3238DF8003095238DF8013003238DF80C
:1010500002308EF06FF91022CDF80300CDF80710A2
:1010600004F58F5069468DF80B60039553F014FC1E
:1010700004B070BD7FB50E464FF6FF7104461546AD
:101080000EF032FDE0B1102200216846B7F08EFB71
:10109000A3238DF8003095238DF8013004238DF8BB
:1010A00002308EF047F91022CDF80300CDF807107A
:1010B00004F58F5069468DF80B60039553F0ECFBF7
:1010C00004B070BD30B52DED048B87B004460D46DD
:1010D000182200216846B0EE409AF0EE608AB0EE29
:1010E000418AB7F063FBA3238DF8003095238DF878
:1010F000013006238DF802308EF01CF91822CDF84D
:101100000300CDF8071004F58F5069468DF80B5099
:101110008DED039ACDED048A8DED058A53F03CFBED
:1011200007B0BDEC048B30BD10B54FF48011044600
:101130000EF0DAFC30B104F59F500830BDE81040E5
:101140000FF0EABE10BD00002DE9F0438FB0144649
:10115000054689463122002101A8DDE91676984628
:10116000B7F024FBA3238DF8043095238DF80530C8
:1011700008238DF806308EF0DDF823680493636849
:101180000593A36806933B68CDF81D307B68CDF8C6
:101190002130BB68CDF825303368CDF8293073682D
:1011A000CDF80700CDF80B10CDF82D303122B36803
:1011B0008DF80F9001A905F58F508DF81C80CDF8A2
:1011C000313053F0E9FA0FB0BDE8F08370B52DED82
:1011D000068B8CB0144605460E462C22002101A831
:1011E000B0EE409AF0EE608AB0EE418AB0EE61AAAD
:1011F000F0EE429AB7F0DAFAA3238DF80430952383
:101200008DF805300B238DF806308EF093F8DFED66
:101210001A7A94ED007ACDF8070027EE277A29EEA6
:10122000279A8DED077A94ED017ACDF80B1027EE11
:10123000277A68EEA78A8DED087A94ED027A8DF808
:101240000F6028EE278A67EE277A2C2201A905F580
:101250008F508DED049ACDED058A8DED068ACDED8A
:10126000097A8DED0AAACDED0B9A53F095FA0CB0E0
:10127000BDEC068B70BD00BFE02E6542A02070471C
:1012800030B5154B89B004466946D3F8780204F5A9
:101290008F551E2286F05CF96A461049284653F0A5
:1012A00017FC04F54053D3F8540203681B689847B1
:1012B00004F50053014693F80C24284653F02CFC07
:1012C00004F59F50083011F02FFE04F590701FF0C8
:1012D00011FC09B030BD00BF385C002062270D084A
:1012E000274B70B54360044618305EF077FC254EFE
:1012F000254BA361682560195EF026FE66513035E6
:10130000B5F55A7FF7D1214D04F55A7060F0ACFA6B
:10131000002104F27C7088F00BFDC4F8305804F60C
:101320003800A5F5AB6589F0D9F99FED191ADFED05
:10133000190A9FED190AC4F8C85804F6DC007EF0BB
:1013400039FD9FED131A9FED150AF0EE410A04F6E0
:10135000F4007EF02FFD9FED0E1A9FED100AF0EEC7
:10136000410A04F60C107EF025FD20460C494BF096
:1013700035FA20460B494BF031FA204670BD00BFCC
:10138000983A0020CC240D08E0240D089484002015
:10139000000000009A99993E0000B44300804A433F
:1013A00058180D08C81A0D0870B54C4D4C49ADF5CC
:1013B0000E7DD02206465AA8B7F0AEF90FCD0EAC7E
:1013C0000FC40FCD0FC40FCD0FC495E80F0084E8F4
:1013D0000F0000245AAB18190021B7EE000A103490
:1013E0004AF0D8FBD02CF5D13E4B0FCB02AC84E8B1
:1013F0000F0001A920464AF081FB90B19DF904300D
:10140000DFED396AE06807EE103AB8EEC77AF0EE21
:10141000007AE7EE267AB7EE000A80EE270A4BF054
:1014200085FD00240EAB181900211034B7EE000A18
:101430004AF0B0FB402CF5D12C49902236A8B7F0E9
:101440006BF90022092136A84AF050FC96F9DC69B4
:10145000D6B9274D0FCD1EAC0FC40FCD0FC40FCD85
:101460000FC495E80F0084E80F00324604211EA83F
:101470004AF03CFC9FED1F0A1F484BF057FD1F48E8
:10148000B7EE000A4BF052FD1D4C9FED1E0A0FCC2B
:1014900006AD0FC594E80F0085E80F00002106A8EF
:1014A0004AF078FB9FED170A002128464AF072FBAC
:1014B00004F1100160221EA8B7F02EF900241EAB23
:1014C00018190021B7EE000A10344AF063FB602CB3
:1014D000F5D15FF055FF0DF50E7D70BD90CA0C087B
:1014E000C0C90C08D0CA0C08CDCCCC3DE0CA0C0851
:1014F00070CB0C080000000040170D084F170D08B6
:10150000B0CB0C08000034422DE9F04790B00DF14B
:1015100006011D2060F028F8002800F09E809DF84C
:101520000630614A0133DBB211210BA88DF8063079
:101530008DF07AF800220DF107010BA84AF064F84B
:101540009DF80630594A112105460BA88DF06CF81C
:1015500000220DF107010BA84AF056F89DF806305D
:10156000534A112106460BA88DF05EF800220DF1BA
:1015700007010BA84AF048F89DF806304D4A03F0E1
:101580003F03112107460BA88DF04EF800220DF104
:1015900007010BA84AF038F88046002D5DD0002ED8
:1015A0005BD0002F59D0002857D028464AF044FA83
:1015B000002852D130464AF03FFA00284DD1384633
:1015C0004AF03AFA002848D140464AF035FA002855
:1015D00043D1394C94E80F000DF10C0C10348CE819
:1015E0000F0094E80F000DF11C0989E80F0002A913
:1015F00060464AF083FA98B3BDF8084002A948460D
:101600004AF07CFA00284AD0BDF8083054BB23B316
:1016100040F2E2449C420FFA84FA0FFA83F927D889
:101620000DF10A013046ADF80A904BF075FF0DF14F
:101630000A012846ADF80AA04BF06EFF0DF10A0131
:101640003846ADF80AA04BF067FF00230DF10A0100
:101650004046ADF80A304BF079FF10B0BDE8F08796
:101660000024CBE740F2D662002B08BF1346D1E737
:101670000DF10A013046ADF80AA04BF04DFF0DF117
:101680000A012846ADF80A904BF046FF0DF10A0119
:101690003846ADF80A904BF03FFF0123D6E7002C07
:1016A000DBD040F2D663B5E760170D086C170D0864
:1016B00078170D0885170D0830CC0C0837B500F5E4
:1016C000115178221031044651F026FC00220C21E1
:1016D00026484AF00BFB2046FFF716FF04F5115091
:1016E0000022B7EE000A022124304AF087FB0125D0
:1016F00004F50B511E4A00950023383145204AF06D
:10170000F9FA1C4A1368D90709D41B49156004F576
:101710000A5308330B6004F594531833CB6004F577
:10172000135015490222083001254AF035FB134AAF
:101730000095002304F58F51FD204AF0DBFA104B91
:101740001A68D20705D40F4A1D6004F598540C346A
:1017500014600C4801214AF03BFB4BF045FA0A4A61
:10176000138843F00103138003B030BD98170D08B0
:10177000C08A0E086C8500200022002020D20D08AF
:101780007085002018220020CC8700200F299DBFE3
:10179000302303FB0100503000207047014B93F9C8
:1017A00097047047384C0020024B93F86D0200F00C
:1017B00001007047385C0020044BB3F85C34DB0751
:1017C0005ABF0069C0F3401000207047384C002019
:1017D000014BD3F8480E7047384C002008B5036819
:1017E0009B68984730B9044B93F96C02B0FA80F0CB
:1017F000400908BD0020FCE7385C002038B50D1E0C
:101800002DDB174C94F8542EEBB29A4227D3D4F820
:10181000503E0122595DA4F5005004F0DDF8F0B10E
:101820005EF05CFB03215FF05DFBC0B95EF056FB30
:101830000D215FF057FB90B994F97C34EB40DB0746
:101840005CBF94F99614E940A4F5005048BF02210A
:10185000BDE8384058BF01F00101FCF7C5BC38BDF8
:10186000384C0020022A10B50C4605D1BDE81040C6
:101870000948352204F0B0B8084BD3F85402036885
:101880001B689847A04205D15EF028FBBDE81040D8
:101890005EF0AEBA10BD00BF382C0020385C0020CE
:1018A00029B1022907D1044BC3F84C127047024BEF
:1018B0000122C3F84C227047385C002031B1022964
:1018C00007D1044B012283F850227047014B83F863
:1018D00050127047385C002010B500F50053DFED62
:1018E000186AD3F8402ED3F83C3EB2F90820B3F979
:1018F00008309FED147A07EE902AF8EEE77A044656
:10190000C7EEA60A00F59F500121083007EE903A75
:10191000F8EEE77A60EE870A87EEA60A20EE070A5D
:1019200011F03AF953F0E6FD262153F01FFD04F5BE
:101930004050054ABDE810400621203055F0E4BE75
:101940000000C84235FA8E3C9C220D0800F580420A
:10195000002382F8A03E044A00F54050137206218D
:10196000024A203055F0D0BE3D870020A8220D0845
:1019700070B500F58045044695F8A01E002957D0A3
:101980002C4B2D4AD3F85402904204D1D3F878322C
:1019900093F8CB3023B92046BDE87040FFF7D6BF9F
:1019A000264E95F8A10E04F54053012293F94832D2
:1019B0003272D0BB002B3BDB85F8A12E0139C9B2B6
:1019C00004F5005385F8A01ED3F8402ED3F83C3E12
:1019D000B2F90820DFED1A6AB3F908309FED197AE1
:1019E00007EE902AF8EEE77AB1FA81F1C7EEA60A7F
:1019F00004F59F504909083007EE903AF8EEE77A6F
:101A000060EE870A87EEA60A20EE070A11F0C4F8F6
:101A100095F8A03E63B904F5405033720A4ABDE818
:101A200070400621203055F06FBE002BC6DAB2E7B9
:101A300070BD00BF385C00206C8300203D87002013
:101A400000007A4535FA8E3CBC220D086D2900F362
:101A5000E380012901DC5FF089B88B1E6B2BFAD87B
:101A60000FF2040C5CF823F0771C0108711C0108CC
:101A7000771C0108771C0108571A0108771C010818
:101A8000571A0108571A0108711C0108571A010852
:101A9000771C0108711C0108711C0108571A010804
:101AA000771C0108771C0108771C0108571A0108E8
:101AB000571A0108711C0108771C0108711C0108E4
:101AC000571A0108711C0108711C0108571A0108F6
:101AD000571A0108571A0108571A0108571A01081E
:101AE000711C0108771C0108571A0108571A0108D0
:101AF000571A0108771C0108571A0108711C0108C0
:101B0000571A0108571A0108771C0108711C0108AF
:101B1000571A0108571A0108571A0108771C0108BB
:101B2000771C0108771C0108571A0108571A010889
:101B3000771C0108571A0108571A0108771C010879
:101B4000771C0108771C0108571A0108571A010869
:101B5000771C0108771C0108571A0108571A010859
:101B6000571A0108571A0108571A0108571A01088D
:101B7000771C0108771C0108771C0108771C0108F5
:101B8000771C0108771C0108571A0108711C01080D
:101B9000711C0108571A0108571A0108571A010841
:101BA000571A0108571A0108571A0108771C01082B
:101BB000711C0108571A0108571A0108571A010821
:101BC000571A0108571A0108571A0108571A01082D
:101BD000571A0108571A0108571A0108571A01081D
:101BE000571A0108571A0108571A0108771C0108EB
:101BF000571A0108571A0108571A0108571A0108FD
:101C0000571A0108571A0108571A0108571A0108EC
:101C1000571A0108711C0108A12921DC96297FF7B8
:101C20001AAFA1F197030A2B3FF615AF0FF2040C80
:101C30005CF823F0771C0108771C0108571A01088B
:101C4000771C0108571A0108571A0108571A01088A
:101C5000571A0108711C0108711C0108771C010842
:101C6000B42908D0DB2903D0B2297FF4F4AE704741
:101C700000235EF04DBF704770B563298AB00346FC
:101C800068DC012973DD881E612870D8DFE810F058
:101C90007C008400940099006F00B3006F006F0017
:101CA0000C016F006F008B001F016F000A013C01E7
:101CB00043016F006F004B01520159016F006A012F
:101CC00073016F006F006F006F006F007C016F0089
:101CD0006F006F006F0089016F006F006F006F0071
:101CE0008B016F006F006F006F006F006F006F005F
:101CF0006F006F0093016F006F00450147014901BC
:101D00006F006F006F006F006F006F006F006F005B
:101D10006F006F008D018F0191019501970199016D
:101D20006F00BA019B016F006F006F006F006F00C2
:101D30006F006F0003026F006F006F006F006F0095
:101D40006F006F006F006F006F006F006F006F001B
:101D50006F000F02B22900F066810EDC9A2900F0B4
:101D6000B2819F2900F09F81982900F0A281184636
:101D70000AB0BDE870405EF057BCB42900F0C680E0
:101D8000DB29F4D1012433E0022AFBD135220E21D4
:101D9000AF4803F021FEF5E7111E18BF0121AC4842
:101DA000FCF722FAEEE7012A04D0022A14BF002130
:101DB0000221F4E71146F2E706211846FFF752FD2B
:101DC000E0E7022ADED1A34DD5F854020368DB6AAE
:101DD000984704460028D5D0A5F58053D3F8443E53
:101DE000B3F90830002BCDD1A5F54050FFF774FDB5
:101DF00020460AB070BD022AC4D1964E964AD6F843
:101E000054129142BED0D6F8782292F8CB20002A04
:101E1000B8D006F50054A6F58056B4F960212AB969
:101E2000D6F8443EB3F90830002BABD01C22002179
:101E300003A805ADB6F0BAFC284615F04BFEB4F980
:101E40006031864C93B91623ADF80E30D4F85C3E61
:101E50008348642BB8BF642303A906932CF066F96A
:101E600020B153F047FB272153F080FA04F6586362
:101E70000FCB85E80F00D6F8443E7948B3F9083017
:101E8000002BCCBF1023152303A9ADF80E302CF086
:101E90004DF900283FF476AF53F02CFB272153F087
:101EA00065FA6FE7032188E7022A04D06D4B002210
:101EB00083F8582E66E76C4819214BF037FF04462B
:101EC0000028F3D0674B012283F8582E90E7012AAF
:101ED0000BD0022A11D0002A7FF454AF614B83F853
:101EE000C02453F007FB2B21D9E75E4B019283F806
:101EF000C02453F0FFFA2C21D1E75A4B83F8C024B9
:101F000053F0F8FA2D21CAE70F2156E7574811463A
:101F10008BF088FD36E709214FE704214DE70521C5
:101F20004BE7172149E7901E41424141504865F077
:101F300041FA27E7022A7FF425AF454801F06CFB00
:101F400020E7012A06D0022A07D0002A7FF41AAF20
:101F50001146EBE711460192E8E74548012165F09B
:101F600029FAEAE73D4B911ED3F8843E4A424A41A2
:101F700083F8202006E7931E59425941374BD3F886
:101F8000840E7FF023F8FDE6324B013A93F84A12B3
:101F9000012A8CBF0022012262F3041183F84A1245
:101FA000F0E6122109E7152107E7002105E71021D6
:101FB00003E7022101E70121FFE61621FDE60721E3
:101FC000FBE60B21F9E6022A2A4B0ED1012483F805
:101FD000504053F08FFA4A2153F0C8F95CF074FA7C
:101FE000254A062155F090FB02E7002283F8502095
:101FF00053F080FA4B2153F0B9F95CF065FA1F4AAF
:10200000062121E0012A09D0022A0AD0002A7FF401
:10201000B9AE01211A480DF053FCB3E6019200213C
:10202000F8E71146F6E77AB3022A7FF4ABAE094B24
:10203000D3F8540203689B6F984700287FF4A2AE40
:102040005CF042FA0F4A042155F05EFB9AE600BFAD
:10205000382C0020385C0020287D0020386C0020BF
:10206000647D0020384C0020683B00203C7F00202D
:10207000307C0020387C0020D4220D08E5220D0899
:10208000205B0020F7220D08184BD3F85402036898
:10209000DB6F984776E618461146FFF701FC1448B7
:1020A00004F050F86EE61146FFF708FC6AE61B21C3
:1020B00083E6022A7FF466AE0E48FCF79FFE5CF0D2
:1020C00003FA0D4A9CE711465EF0D0F90B487BF00D
:1020D0000DFE044600283FF455AE044A92F84B32F8
:1020E00043F0020382F84B3282E600BF385C0020E6
:1020F000AC7C0020382C002010230D08985B0020B9
:1021000010B50446044884F079F904F10801BDE8EB
:10211000104028F039BE00BFA07A002038B5044630
:102120002DED028B114884F06FF905462AF096FDDB
:102130000F48B0EE408A0DF071FC90B1DFED0D7AE2
:10214000B4EEE78AF1EE10FA0BDDD5ED000A95ED5D
:10215000010AB4F031F9DFED087A20EE270A84EDA8
:10216000080ABDEC028B94ED080A38BDA07A002065
:10217000382C002000401C46E02E6542074B93F9A6
:102180007D04022805D0032806D0003818BF01209E
:10219000704781F00100704704207047384C0020E0
:1021A00003688B4216D00429C0E9001302D0072926
:1021B0000ED07047084B9FED097A03F5BD63D3ED50
:1021C000007AF8EEE77A67EE877AC0ED087A704712
:1021D00000238362704700BF383C00200AD7233CAD
:1021E00008B50246FFF7CAFFBDE8084001461046A1
:1021F000FFF7D6BF70B52DED048B0446F0EE408A94
:10220000B0EE608A0D4616468DF08CF89FED329A3E
:10221000DFED329AE06176B3236843B9304B03F5C2
:10222000BD63D3ED007AF8EEE77AC4ED097A68EE83
:10223000898A002DB7EE000AFFEE007AB8BFB0EE33
:10224000670A68EE808AC4ED058A264BB4EEE98AF7
:10225000F1EE10FAD3F8840E30DA7DF095FE20EE20
:10226000090A84ED060ABDEC048B20460321BDE873
:102270007040FFF795BF94ED090A98EE890A27F0A0
:10228000D5FC002D84ED050A0BDAB4EEE90AF1EE77
:1022900010FADADBDFED147A30EE670A84ED050A16
:1022A000D3E7D2D0DFED117AB4EEE70AF1EE10FAFF
:1022B000CBD8DFED0D7A30EE270AEFE77DF064FE34
:1022C000B4EE480AF1EE10FA48BFB0EE408A28EEAC
:1022D000098A84ED068AC6E70000C842000000347F
:1022E000383C0020386C002000A00C47000000B4EF
:1022F00010B52DED028B0446B0EE608AF0EE408AF8
:102300008DF010F8DFED090AE06168EEA08A68EE52
:10231000200AC4ED098ABDEC028BC4ED0A0A2046EE
:102320000621BDE81040FFF73BBF00BF0000C842D8
:1023300010B52DED028B0446B0EE408A8CF0F2FF12
:1023400094ED090ADFED097AE061A8EE270A27F08B
:1023500057FCBDEC028B002384ED090AA3622046E2
:102360000621BDE81040FFF71BBF00BF0000C842B8
:1023700070B54B68154D06460C4673B98B6863B94A
:10238000C96851B91248FFF72BFF95F89D1F05F654
:102390002470BDE8704060F06DBB95F89D1F0D483E
:1023A00060F008FA48B906F10801204615F022FD50
:1023B00018B107480221FFF7F3FE95F89D1F054865
:1023C0002246BDE8704060F049BB00BF386C002079
:1023D000748500205C7B002008B50721FFF7E0FE34
:1023E00080ED0A0A08BD000008B50368032B23D15D
:1023F000D0ED057A9FED127AF0EEE77AF4EEC77A27
:10240000F1EE10FA1AD50F4B90ED090A03F5BD63F2
:10241000D3ED007AF8EEE77A37EEC00A27F006FC33
:10242000DFED097AB0EEC00AB4EEE70AF1EE10FA79
:1024300094BF0120002008BD0120FCE70020FAE73E
:1024400000000034383C00200000484330B50368E9
:10245000023B85B00446082B6DD8DFE803F0050D7C
:1024600030374B613F616100FFF74AFE84ED090A96
:1024700094ED090A05B030BD8CF054FFE369DFED3F
:10248000310AE061C31A07EE903AF8EE677A94EDEC
:10249000050A67EEA07AD4ED060AF12020EEA71A0D
:1024A00067EEE00A27F018FCD4ED057A77EEC07AE3
:1024B000C4ED057AD4ED097A37EE800AD6E7FFF746
:1024C0002DFEDFED217A20EE270ACFE71F4BD3ED5B
:1024D000A87AF8EEE77AC0ED097AC9E71C4DD5F87D
:1024E000980E82F025F90028C2D0D5F8983E1B6BD3
:1024F0006362BDE78CF016FFE3699FED127AD4EDBD
:102500000A6AE061C31A07EE903AF8EE677A67EE5E
:10251000877A94ED097AA6EEA77A84ED097AA7E77F
:102520000B4B9FED0C0AD3F8840E6C302AF054FE4E
:1025300084ED091A9CE7064BD3F88C3ED3F844335C
:10254000D6E700BF6F12833A0000C842385C002013
:10255000386C00209F0CB3450368092B08D8DFE8CE
:1025600003F0050A0505050507070510002383622A
:1025700090ED0A0A7047044BD3F88C3ED3F84833E9
:10258000F5E7C36AF3E700BF386C0020F8B5002315
:10259000214FCB6297F86D32204E13F0010F0446A5
:1025A0000D462DD1D7F8540203685B6F984738B3B6
:1025B000D7F8540203F0CAFBDFED197A85ED0B0A58
:1025C000B0EEC00AB4EEE70AF1EE10FA03D4092126
:1025D0003046FFF7E5FD1148FFF738FF0F4884ED5F
:1025E000000AFFF7B9FF336884ED010A0A2B0FD800
:1025F000DFE803F00C1010101010100C100C0C0081
:102600003368092BE7D105480021E2E70223A360E4
:102610002046F8BD0123FAE7385C002074850020CD
:1026200000000034034B01221A6000229A60DA6035
:102630001A6170477485002013B501A904460DF096
:1026400085F804F5804320B9012283F8CD2F02B02C
:1026500010BDDDED017ADFED096A03F57C62B8EEAD
:10266000E77AD2ED007A67EEA67AB4EEE77AF1EE79
:1026700010FA54BF01220022E7E700BF0000C84261
:102680002DE9F04F2DED068B00F500538DB000F5D0
:102690009F59019393F9D234054600F5A04409F1FE
:1026A000080933B100F54058D8F8783293F8CB7068
:1026B0007FB90021A4F84410484610F05DFC94F85E
:1026C000451048460DB0BDEC068BBDE8F04F10F04C
:1026D0005DBC8CF027FE05F5804B0090DBF88C0E7E
:1026E0009FED928A90EDDBAA80F042FA09AE0028B5
:1026F00000F0C980DBF88C3E03F55C7393E80700BB
:1027000086E8070030468DED0B8A2BF063F9B0EEBA
:10271000409A28460DF082F905F59C4A0AF1680AAC
:10272000002800F0B380504683F06EFE07C886E8AC
:10273000070030468DED0B8A2BF04CF9F0EE409AF5
:10274000D8F8540203681B689847122840F0A78005
:10275000002384F84430D8F8540203685B69984732
:1027600030B1019BD3F8443EB3F90830002B0ADCAA
:1027700098F94832002B06DA009BA364504683F098
:102780003FFE84ED130A94F8443053B1009BA06CD3
:10279000181A41F28833984240F28F80002384F85F
:1027A0004430DBF8840E9FED620A6C302AF014FD91
:1027B0008DED090ACDED0A0A8DED0B1A96E807009A
:1027C00006AB03AE9FED5B0A83E8070086E80700CF
:1027D00030462AF001FD2846B0EE408AF0EE608ACD
:1027E0008DED060ACDED070A8DED081A0DF016F9EC
:1027F000002872D0DFED507AF4EEE79AF1EE10FA8D
:1028000094BF01250025DBF88C0E80F0B1F930B1C2
:10281000DFED497AB4EEE79AF1EE10FA09D9002D0E
:1028200062D1D8F8540203681B689847022862D026
:102830000027DBF88C0E80F0BDFA0546002871D029
:10284000B5EEC0AAF1EE10FA6BD5DFED3C7AB4EE2E
:10285000E7AAF1EE10FAACBF01260026504683F03D
:10286000DBFD5EB9DFED367AB0EEC00AB4EEE70A02
:10287000F1EE10FA58D8002D08BF002794F8441044
:1028800084F8457018E7B0EE489A42E728460DF004
:1028900095F800287FF447AFDFED249A50E7D8F889
:1028A000783293F8CB30002B3FF455AF98F948328B
:1028B000002BBFF650AF01234BE7504683F0A0FD3D
:1028C000D4ED137A30EE670ADFED1E7AB4EEE70A34
:1028D000F1EE10FA3FF762AF63E728460DF06EF8AD
:1028E0000546002886D18EE7DBF88C0E80F040F993
:1028F000002896D19DE7B0EE680AB3F03BFBF0EEFE
:10290000408AB0EE480AB3F035FBDFED0F7A20EED7
:10291000280AB4EEE70AF1EE10FACCBF012700272F
:1029200087E700252E4699E73746A7E70000000015
:102930009F0CB345D30237390000FA420000C8C2E9
:10294000000070420000484255CF7D3F38B5044634
:102950000DF064F804F59F55083548B920460DF090
:102960002DF8014620B92846BDE838400FF050BD8B
:1029700004F54054D4F8540203689B6C984720B97E
:10298000D4F854020368DB6C98470146EBE700007B
:1029900030B5044689B0684604F59F5515F09AF89D
:1029A000083504A815F096F8694628460FF0EAFDA8
:1029B00098B104A928460FF035FE70B1059B01932C
:1029C00023680022DB6C69462046984728B104F54D
:1029D00031500121043087F077FC09B030BD000090
:1029E00000F5805292F86426D2070BD400F54052CD
:1029F000D2F8782292F8CB1009B1FFF7C9BF03686B
:102A00009B6C18477047000030B587B0044602A899
:102A1000019115F05FF804F59F5002A908300FF0FE
:102A2000B1FD019A18B90025284607B030BD2368CA
:102A300002A9DB6C2046984705460028F3D004F530
:102A400031500121043087F03FFCEDE7F0B504463A
:102A500085B004F59F56684608360F46154615F0B2
:102A600039F8694630460FF0DDFD10B9002005B099
:102A7000F0BD394630460FF03DFC0028F6D0002D61
:102A8000F5D004F58054284694F8643643F00203E8
:102A900084F86436EBE700002DE9F04F2DED0A8B4A
:102AA000BDB0044624220D4618A80021B5F07EFED4
:102AB0002422002121A8B5F079FE242200212AA891
:102AC000B5F074FE04F540562422002133A8B5F079
:102AD0006DFE0023CDE90D330F9396F8493213F0C4
:102AE000080839D104F5005943F0080399F8382E45
:102AF000079286F8493216F045F990F9213003B370
:102B000090F84033EBB104F28457384616F04AF897
:102B1000C34694F8A6355FFA8BF18B421FD938462D
:102B200016F01EF80BF1010B82460028F1D1C94ABC
:102B30000221284658F0DCF896F849326AF3C303BC
:102B400008E0C54A0221284658F0D2F896F84932E2
:102B50006FF3C30386F849324FF001083EE304F5F2
:102B60003D532033012118460BEE903AFBF718F83D
:102B7000824608B9B94ADBE720460CF06DFCD9F86B
:102B8000443EB3F908A0BAF1000F01D0B44AD9E726
:102B900096F94832002B01DBB24AC9E7204601F022
:102BA000A9FE04F54A532433184652460CA90CEEEC
:102BB000103A12F0C9FF002814BF02230123039327
:102BC000F123CDE9133A8F210A23CDE9003113AA6D
:102BD000287CADF854A003234D2155F0C9FDA24B2C
:102BE0009FEDA28A01225A720621A14A284658F076
:102BF0007FF8039B022B0CBF9E4A9F4A0621284662
:102C00004FF0000A58F074F889F88AA45146384603
:102C100015F012FF94F8A6355FFA8AF18B420CD9B1
:102C200013AA38468DED138A8DED148A8DED158A21
:102C30000AF1010A15F082FDECE7384615F0B2FF03
:102C40004FF0000A4FF07C0B94F8A6255FFA8AF942
:102C50004A4519D94946384615F062FCC0B20BFB0B
:102C600000403CAA0C2300F2146003FB092C07C8A7
:102C7000ACF1900C8CE807003CAA02EB890909ED45
:102C80002F8A0AF1010ADFE741F288310AA822F00F
:102C9000D9FFD6F878029FED759A03689FED77AA61
:102CA0009B6ADFED77AA9847D6F87802012184F075
:102CB00053FB744B1B680293D86A036801211B689D
:102CC00098478CF02FFB05908CF02CFBF0EE499A86
:102CD0000690002604F50059079A99F8383E934269
:102CE00040F0D88094F8C618384615F039FF00280F
:102CF00000F0D08004F5405BDBF8783293F8CB30FD
:102D00000493002B00F0C68041F288310BA822F01A
:102D100099FF8CF007FB059BC01A132840F2D9805D
:102D20008CF000FB059020460CF096FB5EF0C4FE94
:102D300082465EF057FED9F8443EDBF87802B3F9DC
:102D4000083000EE103AB8EEC00A20EE0A0A85F00C
:102D500075FF50465EF04EFE384615F023FF1CEE20
:102D6000100A13F00DF9D9F8443EDFED400AB3F92B
:102D7000083000EE103AB8EEC00AA22020EE0A0A8F
:102D8000B7EE001A26F0A8FFB4EEE90AF1EE10FA49
:102D90001CEE100A4FF000020CA958BFF0EE409A4A
:102DA000F0EE408A12F0D0FE08B900230C939DED9E
:102DB0000C8ADFED357AB4EE498AF1EE10FAF4EEC2
:102DC000E78A48BFB0EE498AF1EE10FA80F28F80B0
:102DD0009FED2E9ADFED2E8A4FF0000A94F8A6356B
:102DE0005FFA8AFB5B4540F296814FF00C0918AB05
:102DF00009FB0BF903EB0900B0EE490A2AF0ECF9E4
:102E000059463846CDED110A8DED121A8DED100A96
:102E100015F086FB7C23C0B203FB0040B0EE680ACD
:102E200000F214602AF0D8F93CAB13A910A8994419
:102E30008DED130ACDED140A8DED151A2AF0A0F9C7
:102E40000AF1010A09ED240A49ED230A09ED221AC3
:102E5000C4E700BF0D250D08FC240D08473A0D08F6
:102E60001B250D082D250D083D87002000000000C2
:102E700038250D084D250D0837CE0C086F12833A02
:102E80000000C8426885002000000034A4707D3F27
:102E90000AD7233C04F54059D9F8780203689B6AA5
:102EA0009847D9F87802002184F056FA029BD86A34
:102EB000036800211B689847002E40F05F81284678
:102EC000C94A052157F014FF3146384615F0B4FDC4
:102ED00070E1029B986A036805215B6898470BA81C
:102EE00022F0BCFEB0EE498AB0EE489AF2E64FF00E
:102EF00000094FF00C0B04F5B86A94F8A6255FFAA8
:102F000089F39A4222D919463846089315F008FBEE
:102F1000089B0BFB03F13CAB5A18A2F16C034FF07A
:102F20007C0CC0B2CDE908320CFB00A018AB1944F0
:102F300054302AF03BF9089B099A09F1010902ED86
:102F40001B0AC3ED010A83ED021AD6E7039B012B8E
:102F50004FF0000A46D19FEDA5BA9FEDA59A4FF01C
:102F60000C0B94F8A6355FFA8AF6B34240F28680DD
:102F70000BFB06F63CAB03EB0609A9F148030893EB
:102F800021ABB0EE680A98192AF036F9089B09EDD2
:102F9000120AC3ED010A83ED021A33ABB0EE4B0AFD
:102FA00098192AF019F92AAB98198DED100AB0EE8C
:102FB000490ACDED110A8DED121A2AF00DF913A967
:102FC00010A88DED130ACDED140A8DED151A2AF017
:102FD000EDF80AF1010A09ED090A49ED080A09EDBF
:102FE000071ABEE79FED819A9FED81BAF0EE088A3D
:102FF00094F8A6355FFA8AF94B4564D99DED0C0A21
:10300000B4EEE80AF1EE10FA35DB0C2303FB09F904
:103010003CAB03EB090621AB03EB09002AF0ECF80B
:1030200033AB46ED110A06ED101A06ED120A03EB5A
:103030000900B0EE490A2AF0CFF82AAB03EB0900E9
:103040008DED100AB0EE4B0ACDED110A8DED121A7E
:103050002AF0C2F813A910A88DED130ACDED140AB9
:103060008DED151A2AF0A2F806ED090A46ED080AB8
:1030700006ED071A049E0AF1010AB9E74FF00009AC
:103080004FF00C0A94F8A6355FFA89F6B34241D99D
:1030900033AB0AFB06302AF09DFC1BEE900AF0EEE3
:1030A000408A7AF01FFE07EE900AB8EE677A3CABD2
:1030B000C8EE877A03EB860609F1010967EEAA7A62
:1030C00046ED2F7ADEE74FF0000A4FF00C0B94F834
:1030D000A6355FFA8AF94B451DD933AB0BFB093096
:1030E0002AF078FCC8EE297A0AF1010A1BEE900A50
:1030F00067EE808A7AF0F6FD07EE900AB8EE677AFE
:103100003CABC8EE877A03EB890967EEAA7A49EDF2
:103110002F7ADCE7049E8CF005F9069BC01AB0F507
:10312000FA7F27D98CF0FEF804F50053DDED0D7A17
:10313000D3F8443E0C9A1B891392FCEEE77A339A3B
:103140001492ADF85C30349A159217EE903A359A95
:103150001692ADF85E30F0221423CDE90032B12191
:10316000069013AA287C55F003FB74F0B3FD297C6C
:1031700074F0A2FC0BA822F071FDB5E60399384665
:1031800015F05AFC00264FF00C0A94F8A635F1B25F
:103190008B4207D933AB0AFB0132384615F0CEFA21
:1031A0000136F2E7384615F0DBFA124A06212846C6
:1031B00057F09EFD104B002520465D7201F08CFB00
:1031C00004F512500A3049F0DFFB99F8493265F3F3
:1031D000C30389F849320AA822F040FD40463DB0B9
:1031E000BDEC0A8BBDE8F08F9DDC0E08A4707D3F1E
:1031F0000AD7233C55250D083D870020F0B5544FD4
:10320000D7F8003EDA0785B0044600F19F8000F54C
:103210004055D5F8783293F8C120002A40F09680C6
:1032200093F8CB30002B00F08E8095F94832002BBC
:10323000C0F2898000F5A04393F85030002B40F095
:10324000858000F580469FED430AD6F8840E6C30E9
:1032500029F0C2FFCDED020A60EEA00ADFED3E7A52
:103260008DED010AE0EE000A8DED031AF4EEE70A97
:10327000F1EE10FA67DCD6F8843E9FED387AD3ED94
:10328000377AF4EEC77AF1EE10FA04D5D5F8783231
:103290001B7A002B57D0B5EE007AF4EEC77AF1EE28
:1032A00010FA50D404F59C40683083F0B5F8DFED97
:1032B0002C7AB4EEE70AF1EE10FA44D8D6F8843E40
:1032C0009FED287AD3ED367A67EE877AB3EE0E7AE1
:1032D000F4EEC77AF1EE10FA35DA234AB4F9A41005
:1032E000138801339BB2138019B9B4F8A210A4F863
:1032F000A410B4F8A410994228D80026168052F0E1
:10330000F9F80122192152F051F8D5F87802036832
:103310005B699847431C04F54050144A31462030FD
:1033200054F0F2F9D5F87832012283F8C120D7F8A9
:10333000003E5B070AD504F59450183005B0BDE88F
:10334000F04067F099BF084B00221A8005B0F0BD2D
:10335000384C00209F0CB3454054094A6666663FCE
:10336000000000B4E02E6542AE8500206C250D08FB
:10337000F0B52DED028B4A4BD3F8003E9B0785B08C
:1033800004461FD400F58046DFED468AD6F8840E49
:1033900003681B699847D0ED017AF4EEE87AF1EE04
:1033A00010FA0FDB04F5405304F5A045D3F878225A
:1033B00092F8C110543549B1002303A9284603935C
:1033C00053F0CEFC05B0BDEC028BF0BD92F8CB20E3
:1033D000002AF1D093F94832002BEDDB04F5A04729
:1033E00097F85030002BE7D1D6F8840E03681B699C
:1033F0009847D0F8A430D6F8840E039303681B696D
:10340000984704F58C7200F1A401284653F0A6FDFC
:10341000DDED037AB0EEC08AF0EEE77AF4EEC87A1A
:10342000F1EE10FA03D503A9284653F099FCD6F81B
:10343000840E03681B699847D0ED040AF4EEE80A8D
:10344000F1EE10FABEDBF6EE087A60EEA77AF4EE43
:10345000C87AF1EE10FA1BD58BF064FF3B6E42F296
:103460001072C31A9342ADD9DFED0F7A386668EE59
:10347000277A04F5405417EE900AF9F745F82034FE
:10348000CDE90001094A0021204654F03DF999E7B1
:103490009DED030A26F01CFB0028DDD192E700BF5A
:1034A000384C0020000000340000C84288250D0878
:1034B00010B5044600F59F40783063F08DFF04F5A9
:1034C000A0400121BDE8104018306CF09BB800000E
:1034D0002DE9F04100F58046044696F9F83F5BB3CC
:1034E00000F5405500F5A04895F8483298F80C20B2
:1034F000DB43C3F3C01363F3C30200F59F4700F53A
:103500009C4088F80C20683082F086FFDFED3E7A20
:10351000783720EE670A384663F0DEFF98F85030BF
:1035200053B9384663F084FFD5F8783293F8CB303E
:1035300023B9364B00221A80BDE8F08198F80C3090
:10354000DB07F9D4D5F8540203689B6B9847002831
:10355000EFD095F94832002BEBDB2C4D2B884BB983
:10356000B6F9FE3F33B1642213FB02F3D6F85C2EAA
:103570009A42E1DB384663F0CBFFD6F8843E9FEDFC
:10358000247AD3ED367A67EE877AB3EE0E7AF4EECC
:10359000C77AF1EE10FA05D82B88002BCCD0013B6E
:1035A0002B80C9E7B4F9A4301BB9B4F8A230A4F851
:1035B000A4302B88B4F8A420B4F9A4001549934290
:1035C0003CBF01332B802B88D6F8342E012B01D140
:1035D0000A60B1E709689142ABDD18B9B4F8A220DE
:1035E000A4F8A420B4F8A4209A42A5D800232B80E4
:1035F00051F080FF02220C2151F0D8FE2046BDE898
:10360000F041FFF755BF00BF0AD7233CAC8500202F
:10361000E02E6542A885002008B500F5804292F9A9
:10362000F83F6BB300F5405393F94832002B0EDAA4
:1036300000F54050134A0621203054F065F851F04F
:1036400059FF0322BDE808400F2151F0AFBEB2F987
:10365000FE3F8BB1D2F85C2E642113FB01F39A423A
:103660000ADA00F54050084A0121203054F04CF8A5
:1036700051F040FF0222E5E7BDE80840FFF718BF20
:1036800008BD00BFA0250D08B2250D0870B52DEDB1
:10369000028B00F540555D4ED5F8783293F8CB306B
:1036A0008CB0044643B195F94832002B04DB00F599
:1036B000005393F9A6342BB9002333800CB0BDEC32
:1036C000028B70BD00F5A04393F85030002BF3D16E
:1036D00001F074FB00287FD1D5F8540203689B6B7E
:1036E00098470028E8D004F59C40383053F08EFB12
:1036F0002AF070F9F0EE087AB4EEE70AF1EE10FA6B
:10370000F0EE408AD8DA04F5805303F5C66203F27E
:103710003463D3ED007A92ED000A20EE270AB2F06E
:10372000E3FDDFED3B7A20EE270AB2EE0E7AB4EE2F
:10373000C70AF1EE10FABFD904F58043D3F8843EEE
:1037400093ED368A28EE278AF3EE0E7AB4EEE78AF6
:10375000F1EE10FAB0D904F59F50002309A9083002
:1037600009930A930B930EF069FF00283DD133882B
:10377000B4F9A42001339BB23380002A40D0B4F8BE
:10378000A420B3EB420F99DB51F0B4FE01220C21CF
:1037900051F00CFE1F4B002218EE900ACDE90623D3
:1037A000F8F7B2FE1C4BCDE90401002218EE100A16
:1037B000CDE90223F8F7A8FE04F540542034CDE902
:1037C0000001164A2046002153F09EFF01220C21E1
:1037D0001348FAF7FDFB71E7D5F854020368DB6C78
:1037E000984700287FF478AF66E709A82AF0F2F836
:1037F000F2EE047AB4EEE70AF1EE10FAB7DB5BE71B
:10380000B4F8A220A4F8A420B9E700BFA485002042
:10381000E02E65420000084000003E40C8250D082B
:10382000985B0020F0B52DED028B8BB00023079341
:103830000893099305AB0446019300F59F5007AB2D
:10384000009302AA04AB03A908300EF00FFE04F5A2
:1038500040570546387528B9002528460BB0BDEC01
:10386000028BF0BD8BF052FDBB699FED347AC31A19
:1038700007EE903AF8EE677A064667EE877A04F527
:103880003F5006AA02A93030CDED067A53F066FB10
:1038900004F53F5006AA03A93C308DED020A53F00F
:1038A0005DFB04F5405006AA04A9083004F5005455
:1038B0008DED030A53F052FBBE6104F5956393ED61
:1038C000008AB5EEC08AF1EE10FAC5D9DDED080A1E
:1038D0009DED070AB2F0D4FBDDED090AB2F0D0FB92
:1038E000D4F8982FDDED037AB4EEC08AF1EE10FA29
:1038F00094BF012300231AB194F89C2FD20712D44D
:1039000038EE087AB4EEE77AF1EE10FA0BD802330B
:10391000DBB2DDED027AB4EEE78AF1EE10FA09D8F7
:10392000002B99D099E7B4EEE78AF1EE10FAF0D8BF
:103930000133EDE7012B90D88EE700BFBD37863508
:1039400070B500F54055044695F86D3243F0040318
:1039500085F86D3251F0CEFD0122112151F026FD86
:10396000D5F8783293F8CB30002B43D0D5F85402F9
:1039700003681B68984709280AD1204608F032FBE3
:1039800030B104F5AB401030BDE8704008F012BB18
:10399000194BD3F8540203681B69984704F5005388
:1039A00040B993F9A534032B24D10621204608F011
:1039B00005FB0DE093F9A5140229F6D195F86D32B7
:1039C000DB07F2D40622204602F006F80028ECD0ED
:1039D0000A4BD5F8540201225A7303681B6C9847AE
:1039E000034604F54050064ABDE8704002212030ED
:1039F00053F08ABE70BD00BF385C00203D870020B8
:103A0000FC250D0808B500F5405292F86D325907B3
:103A100017D56FF3820382F86D320A4B5A7B42B19D
:103A2000002200F540505A730221074A203053F01B
:103A30006BFE51F05FFDBDE808400022112151F0FE
:103A4000B5BC08BD3D87002020260D08F0B5054611
:103A500085B005F59F576846083714F03BF869466E
:103A600038460EF0DFFD80B105F51253D3ED0A7A2A
:103A7000374CF5EEC07AF1EE10FA08D8354A00233B
:103A800028462380D373FFF7BDFF05B0F0BD28465D
:103A9000FFF7C8FE064628460BF090FF10B92846EF
:103AA0000BF066FFA378002E18BF00200343DBB2A3
:103AB000A370002BE9D06378A8BB83BB23780133C4
:103AC000DBB2082B237003D14EB338460EF03AFD1B
:103AD0002378092B02D138460EF02CFD2378092BD0
:103AE0001DD94FF48573238051F004FD022210216B
:103AF00051F05CFC8BF016FC6368C01A47F230533F
:103B0000984209D905F54050134A0221203053F05C
:103B1000FBFD8BF007FC60602846FFF711FF0D4BA3
:103B20006278DA73B1E72678002EF8D0013EF6B25B
:103B30002670002BF3D0002EF1D1667051F0DAFC24
:103B40003246102151F032FC2846FFF75BFFE6E7D2
:103B5000B08500203D87002038260D0800F5405331
:103B600093F86D325B0701D5FFF7EABE704700009E
:103B700073B5044600F59F5001A9083004F50055BF
:103B80000EF0BEFAD5F8DC3F834206460CD004F5B1
:103B90008043D3F8840E7DF0BBFDC5F8DC6F51F097
:103BA000A9FC3E2151F0E2FB04F5805695F9E01F97
:103BB00096F9F82696F8F83691421BD0FF2B19D0CB
:103BC00004F58043D3F8840E7DF0A2FD96F8F83614
:103BD00085F8E03F51F08EFC95F8E02F182151F068
:103BE000E5FB04F5405095F9E03F034A04212030FD
:103BF00053F08AFD02B070BD48260D082DE9F04350
:103C00008FB005468BF08EFB002305930693079338
:103C1000089309930A930B930C930D9305F59F5802
:103C200004AB019308F1080803AB009306460BAB05
:103C300008AA05A940460EF0F9FBDFED487A9DED94
:103C4000077AB4EEE77AF1EE10FA074632DB9DED23
:103C50000A7AB4EEE77AF1EE10FAACBF0124002440
:103C600005F54059404699F81430002B08BF00274D
:103C70000EF0EEFB8046FFB9444605F5005797F974
:103C80009C3D012B29D164B1D9F8783293F8CB400F
:103C90003CB1D9F8540203685B69984780F0010091
:103CA000C4B297F8E43FCBBBCCB9C7F8E86F0FB00C
:103CB000BDE8F0830024D3E7002CDDD005F53F50AC
:103CC0003C3053F04BF890ED007AF7EE007AB4EE0A
:103CD000E77AF1EE10FAD0DCCEE70024E1E7D7F87E
:103CE000E80F301AB0F57A7FE1D9C7F8EC3F01242C
:103CF00005F5804387F8E44FD3F88C3E83F80C44F5
:103D000051F0F8FB22461D2151F050FB144A05F5F5
:103D100040500221203053F0F7FCC8E714B1C7F837
:103D2000EC6FC4E7D7F8EC0F43F69823361A9E429F
:103D3000BDD905F58043C7F8E84F87F8E44FD3F8BD
:103D40008C3E83F80C44C7F8EC4F51F0D3FB22466D
:103D50001D2151F02BFB034AD9E700BF00000034BE
:103D600060260D087A260D080A4B10B5012204467C
:103D70005A728BF0D7FA04F5A042D36BC31A142BF6
:103D800007D9D06304F59C501430BDE8104044F0CE
:103D900067BD10BD3D8700202DE9F743044604F5BB
:103DA000405600F51250002320300DF107018DF828
:103DB000073049F05FFBD6F8780290F9C03002680E
:103DC00083B3083BDBB2012B95692BD93221A8477D
:103DD00004F1100012F04EFA204B04F540581F6811
:103DE0004FF0000908F12008F86A0368DB6998477A
:103DF00001281ED18BF096FA41F28733A0EB09021D
:103E00009A42054605D9164A0621404653F07CFCE5
:103E1000A9462046FFF7A8FFB86A036803215B683C
:103E20009847E1E704F500539269B3F8B41490475A
:103E3000CEE70121D6F8780283F08EFAD6F8780220
:103E40000368DB6A98475DF035FAF86A03681B6817
:103E5000012103B0BDE8F043184700BF688500208A
:103E600098260D0870B5044600F540502DED028BE4
:103E7000184A194E9FED198A0621203053F044FC50
:103E80002046FFF789FF2046FFF76EFF20460BF024
:103E9000E3FA3368986A036803215B6898475DF02A
:103EA0000BFE05465DF09EFD04F50053D3F8443E3D
:103EB000B3F9083000EE103A04F54053B8EEC00AEA
:103EC000D3F8780220EE080A84F0B8FE28465DF0A8
:103ED00091FDD8E7BC260D08688500206F12833A53
:103EE0002DE9F047044600F540502DED028B2A4A9B
:103EF000DFF8AC900621203053F006FC2046FFF797
:103F00004BFF5DF0D9FD04F5405605465DF06AFDB6
:103F1000B7EE000AD6F8780284F090FE28465DF0ED
:103F200069FD8BF0FFF941F2873A07468BF0FAF909
:103F3000C01B5045D9F8008017D99FED188A284634
:103F40005DF050FDB0EE480AD6F8780284F076FEB7
:103F500028465DF04FFD2046FFF706FFD8F8280001
:103F6000036803215B689847E9E728465DF03AFD5E
:103F7000B7EE000AD6F8780284F060FE28465DF0BD
:103F800039FD2046FFF7F0FED8F82800036803212A
:103F90005B689847CAE700BFEC260D0800000000E8
:103FA00068850020F7B500F540530446D3F8783211
:103FB00093F9C030032B2AD0354E652500F5A04774
:103FC000013D15F0FF050BD0BB6B4BB93368986A08
:103FD000036814215B68984720460BF03DFAEFE731
:103FE00004F53D5001212030F9F7DAFD04F50053C6
:103FF00078B993F9A03453B1092B08D08DF8070094
:1040000004F512500DF10701203049F033FA03B0E6
:10401000F0BD93F9A024032A34D8DFE802F002258A
:104020002D30D3F8443EB3F9082040F2B5339A421C
:104030002ADD04F5125001250DF1070120308DF81D
:10404000075049F017FA04F54050124A0221203077
:1040500053F05AFB104B5D720D4B1C68A06A03684D
:1040600005215B689847F9E7D3F8443EB3F9082087
:1040700040F2B5339A4207DD2046FFF7F3FE2046B3
:10408000FFF72EFF092AC2D000238DF80730B7E7CB
:104090006885002010270D083D87002000F540505E
:1040A0000B46024A0421203053F02EBB30270D0866
:1040B00010B5044651F01EFA0022052151F076F9A0
:1040C00004F54050034ABDE810400421203053F06D
:1040D0001BBB00BF3C270D0813B50B464AB100F5CA
:1040E000405000920421054A203053F00DFB02B0ED
:1040F00010BD02B0BDE81040FFF7D0BF54270D0837
:1041000008B500F54050064A0421203053F0FCFA6F
:1041100051F0F0F9BDE808400022082151F046B9FD
:1041200068270D0838B504460D468BF0FBF804F5FA
:1041300040533DB9D3F86422C3F868020AB9C3F802
:10414000640238BDD3F86822801A642884BF002234
:10415000C3E99922F5E7000037B5044600F59C4015
:10416000683082F03FF904F54052C0F3803592F890
:104170004A32C3F34001A9421CD065F341031446FF
:1041800082F84A3220346DB151F0B4F902220B2189
:1041900051F00CF9084A0221204603B0BDE8304036
:1041A00053F0B2BA51F0A6F92A460B2151F0FEF8AD
:1041B000024AF0E703B030BD80270D089C270D08A8
:1041C00038B50A460C460621054601F005FC28B123
:1041D000054A137843F00803137038BD214628467A
:1041E000BDE8384007F0EABE5C87002038B50A46D3
:1041F0000D461521044601F0EFFB28B1094A13785A
:1042000043F00803137038BD04F5405004212030FA
:10421000054A53F079FA29462046BDE8384007F0B0
:10422000CDBE00BF5C870020AC270D0838B50A461C
:104230000D461521044601F0CFFB28B1094A137839
:1042400043F00803137038BD04F5405004212030BA
:10425000054A53F059FA29462046BDE83840FFF791
:10426000AFBF00BF5C870020D4270D0838B50A46D1
:104270000D461B21044601F0AFFB28B1094A137813
:1042800043F00803137038BD04F54050042120307A
:10429000054A53F039FA29462046BDE83840FFF771
:1042A0008FBF00BF5C870020EA270D0838B50446A1
:1042B00000F540500D4620300421044A53F024FA02
:1042C00029462046BDE8384007F078BEFC270D0897
:1042D00010B500F5405494F84A329A0623D4D4F825
:1042E000540203681B689847032808D005D80228A1
:1042F0000ED194F84802C00914E01B28F9D194F8B3
:10430000480200F0A000A0F180035842584109E0A3
:10431000B4F8480220F4FE4020F07F0080B200385C
:1043200018BF012010BD0120FCE7000038B500F5E2
:104330004055044695F86D32184A43F00803284664
:1043400085F86D320221203053F0DEF951F0D2F8B9
:104350000122172151F02AF82046FFF7B9FF40B19A
:1043600004F53D500122BDE8384015212030F9F711
:104370002FBED5F8540203681B689847062806D15B
:1043800004F5AD402830BDE8384009F021B820469A
:104390000B21BDE83840FFF713BF00BF10280D0800
:1043A00070B500F54055D5E999239B1A41F2883242
:1043B0009342064611D9D5F8540203681B6D9847FD
:1043C000044695F86D32C3F3C003A34213D034B151
:1043D0003046BDE87040FFF7A9BF0024F1E751F077
:1043E00089F82246172150F0E1FF95F86D3264F309
:1043F000C30385F86D3270BD0B4610B511460446F7
:10440000072B07D8DFE803F02A041316191C24270A
:1044100007F0D4FD04F50053D3F8A03D9B061DD54D
:1044200004F594501830BDE8104066F025BFFFF742
:10443000C7FEEFE7FFF7FAFEECE7FFF7D7FEE9E785
:1044400000F53D50012214212030F9F7C1FDE1E7CC
:10445000FFF70CFFDEE7FFF729FFDBE710BD0000E9
:10446000F8B5044604F5005751F044F8012205213F
:1044700050F09CFF97F88A34072B98BF304A2046AB
:1044800094BFD55C0125FFF723FF68B12D4A2E4963
:104490002046FFF721FE04F53D5001221021203077
:1044A000F9F796FD002514E004F54056D6F85402BD
:1044B0000368DB6C984798B196F8153883B196F984
:1044C0001438012B0CDC214A21492046FFF704FE59
:1044D0000125294620460322BDE8F840FFF78CBF9E
:1044E000D6F854020368DB6C984718B1D7F8A03DA2
:1044F000190715D4D6F8540203681B689847032897
:1045000003D1D7F8A03DDA070DD4D6F854020368DA
:104510005B6A984768B90C492046FFF7BFFDD8E7AA
:104520000A4A0949D1E70B4A07492046FFF7D4FD5B
:10453000B8E7D7F8A03D5B07EDD5074AF4E700BF21
:10454000F0280D0830280D08EEFD0D083A280D085A
:104550004D280D085D280D086D280D0838B5044656
:10456000154650F0C7FF0122062150F01FFF2046DC
:10457000FFF7AEFE98B104F53D500122072120302F
:10458000F9F726FD144A15492046FFF7A5FD002539
:10459000294620460422BDE83840FFF72DBF04F528
:1045A0004053EDB2D3F854020368DB6C984768B10E
:1045B00004F50053D3F8A03D1B0707D535B1084AD1
:1045C00006492046FFF788FD0125E1E7034920461B
:1045D000FFF764FDDCE700BF30280D088A280D08CE
:1045E0003A280D082DE9F041044604F5005750F033
:1045F00081FF0122082150F0D9FE5BF06FFB97F894
:104600007934072B98BF384A04F5405698BFD55CDB
:10461000D6F8783293F8CB8088BF0225B8F1000F26
:104620000BD132492046FFF739FD002529462046A7
:104630000522BDE8F041FFF7DFBE2046FFF748FE48
:1046400060B104F53D50012212212030F9F7C0FC81
:10465000274A26492046FFF73FFDE6E7D6F85402F1
:104660000368DB6C984768B196F8153853B196F932
:104670001438012B06DC1F4A1F492046FFF72CFD8A
:104680000125D3E7D6F854020368DB6C984718B1CC
:10469000D7F8A03D190713D4D6F8540203681B6855
:1046A0009847032803D1D7F8A03D9A070BD4D7F831
:1046B000A03DDB0609D40D492046FFF7EFFCB5E726
:1046C0000C4A0A49D9E70D4AC3E7D6F854020368F1
:1046D000DB69984706460028EDD1094A0349204680
:1046E000FFF7FAFC3546A1E7F8280D0840140D083D
:1046F00030280D083A280D0884280D0892280D0846
:10470000A7280D08F8B500F50055044695F9793449
:10471000BBB300F54056D6F8D87197B38AF002FEC5
:1047200005F6F85595ED000ADFED167A9FED161A9D
:10473000DFED160AC71B20EE270A8D2025F0CCFAE4
:10474000BCEEC00A10EE103A9F420CD296F86D32C1
:104750009A0716D520460021F9F796FD2046BDE8B8
:10476000F840FFF7CDBC0CD996F86D329B0708D402
:1047700020460121F9F788FD2046BDE8F840FFF703
:1047800031BFF8BD00007A440000804F00000000F7
:104790002DE9F341074600F59C40683081F022FE88
:1047A00007F54054C0F3804801908AF0BBFD94F8AF
:1047B00070324345454606460CD0204684F8708248
:1047C0002030002D41D03C4B3C4AC4F87462022199
:1047D00052F09AFF94F8703207F5005843B394F8FA
:1047E00071322BBBB8F90E3E9FED350A9FED351A9D
:1047F000DFED350A07EE903AF8EEE77A40F257100F
:1048000027EE800A25F068FABCEEC00AD4F87402DC
:1048100010EE103A361A9E420AD9012307F540508D
:1048200084F87132294A244B0221203052F06CFF67
:1048300098F90D3E002B94F86D320DDC6FF34513A3
:1048400084F86D3202B0BDE8F0811B4B204AC4F8F9
:10485000748284F87182BAE7C3F34012AA42F1D09D
:1048600065F3451384F86D329B06EBD5194BD3F8ED
:10487000540203681B6998470028E3D050F03AFEC1
:1048800001221F2150F092FD3846FFF721FD48B16B
:1048900007F53D5001222121203002B0BDE8F04152
:1048A000F9F796BB98F80D1E3222384602B0BDE8E3
:1048B000F041FFF7A1BD00BFC0280D08CF280D08AB
:1048C00000007A440000804F00000000E5280D0839
:1048D000DA280D08385C002008B5044B01221A7054
:1048E0008AF014FD024B186008BD00BFB985002096
:1048F000BC850020014B00221A707047B98500204A
:104900002DE9F04104468AF001FD2A4BB4F8BE209F
:104910001988294E914205460ED01A80274B1860FF
:104920003378A3B10024347050F0E4FD2246132103
:10493000BDE8F04150F03ABD3378214FDBB93B7808
:104940002BB11E4B1F4A1B68C31A934201D8BDE806
:10495000F0810123337004F54053D3F8780290F8C6
:10496000CB3013B103689B6A984750F0C3FD012216
:10497000132150F01BFD3B78002BE8D03378002B3F
:10498000E5D00E4A10491368EB1A8B42DFD904F5C3
:1049900040541560D4F8780290F8CB30002BD6D074
:1049A000002182F0D9FCD4F878020368BDE8F04118
:1049B0005B6A1847BA850020B8850020BC850020B6
:1049C000B985002080841E0040420F002DE9F84385
:1049D00000F5405500F500580446D5F8540298F803
:1049E00034730368DB6C9847014650B995F9483237
:1049F000002BA5BFD5F8783293F8CB00012180F0C9
:104A0000010104F50B5909F13809484667F03CFCEF
:104A1000D5F8783293F8CB300646002B7BD00028AF
:104A200065D03E4B93F94832002B04DB02463C49EB
:104A3000484667F003F898F9FE7257B195F9483285
:104A4000002B0EDA04F53D5001220F212030F9F73A
:104A5000BFFA50F04FFD3246BDE8F843092150F04F
:104A6000A5BCD5F8540203685B69984758B195F91D
:104A70004932002B07DA95F86D32DA0703D498F83B
:104A80003433DB07DED53146484667F063FCDFEDA3
:104A9000257AB4EEE70AF1EE10FA05DD0A220921C3
:104AA000204600F099FFD4E7023F032F11D801A35D
:104AB00053F827F09D4A0108C54A0108E34A010856
:104AC000E94A01080A221521204600F085FF002846
:104AD000BFD10A220621204600F07EFF0028B8D16F
:104AE000DCE70A221121F6E70A221521F3E797B144
:104AF00098F834337BB9094B93F94832002B06DB25
:104B000004F54050084A0521203052F0FDFD50F0D8
:104B1000F1FC0022A0E7BDE8F88300BF385C00206C
:104B200000290D080000C84209290D0870B500F5DC
:104B3000005300F59C45683586B093F8E41F0446A1
:104B4000284681F0FDFB02A812F0C4FF04F59F5037
:104B500002A908300DF016FD04F58043049AC3F84D
:104B6000602E059AC3F8642E284681F03BFC82062D
:104B70001AD5284681F044FC04F59C45FDEEC07A28
:104B8000583504F5805417EE901A0222284617EE85
:104B9000906A12F0A5FF94F86436DB0706D4012270
:104BA0003146284612F09CFF06B070BD0121284610
:104BB00013F028F80028F2D0F6E7000070B500F5F1
:104BC000A04486B0B4F86C308B420D46164602D134
:104BD000A36E93421ED08AF0A5FB636EC31A132BFB
:104BE00018D9A666A4F86C50606650F083FC0446A1
:104BF0008AF0A0FB084B094A1B68CDE90453084B17
:104C00000193084B0093CDE90201074B0749204669
:104C100050F0FCF906B070BDC085002020290D08B9
:104C200038290D08C4FE0C0800E20C0833290D08D1
:104C300038B500F540540D4694F84932C3F380135B
:104C40008B420BD021B150F055FC112150F08EFB5E
:104C500094F8493265F3861384F8493238BD000070
:104C6000F0B52DED048B00F540568BB0D6F87832B8
:104C700093F8CB30054600F58044002B67D096F9B9
:104C80004832002B63DBD6F8540203685B6998470F
:104C9000002861D1D4F8840E9FED440A6C3028F0CE
:104CA0009BFA0AAACDED080A8DED091A8DED070AC7
:104CB00012E9070004AB01AF83E8070087E80700AB
:104CC000384627F0D5FFD4F8843E05F59C403830AF
:104CD000D3ED368AB0EE409A52F098F828F07AFE7A
:104CE000D4F88C3ED6F85402D3EDDB9A0368DB6C23
:104CF000B0EE408A9847DFED2E7AB4EEE79AF1EEF7
:104D000010FA02DC96F850320BB100283AD0DFEDF1
:104D1000297A68EEA78AF3EE0E7AF4EEE78AF1EECE
:104D200010FA2FDCF0EE087AB4EEE78AF1EE10FA12
:104D300028DCF5EEC09AF1EE10FA23DAD4F8840EEE
:104D400003689B6F98470BB0BDEC048BF0BDD4F8A3
:104D5000840E03689B6F0FE005F50055D4F8840EB0
:104D6000D5F8442E0368B2F90820002A03DCD6F8EF
:104D70004C22022AEED1DB6F0BB0BDEC048BBDE8F8
:104D8000F0401847D4F8845EDFED0B0A2B68D3F8A7
:104D90008060D4F88C3E40F2AB1093EDC90AB7EEB8
:104DA000001A24F099FF2846B047CCE79F0CB34582
:104DB0000080BB44E02E65420000000000F540503A
:104DC00090F85002704700002DE9F04100F5405581
:104DD000064695F84832B1EBD31F0C4648D0254B18
:104DE00000221A6000293FD050F084FB122150F0BD
:104DF000BDFA95F8483264F3C71385F8483284F059
:104E0000010873F0A7F8414673F080F806F50057E3
:104E1000B8F1000F06D097F80E341BB98AF082FA69
:104E2000C7F8100487F80E8414B3B7F85C345B0736
:104E30001ED5D5F8783293F8CB30CBB1D5F85402E3
:104E400003685B69984798B9D5F854020368202134
:104E50009B69984760B106F53D500122BDE8F041DD
:104E60000D212030F9F7B4B850F044FB1C21BEE707
:104E7000BDE8F081C08500202DE9F04F2DED0A8BB3
:104E800000F540558DB0D5F8783293F8CB6000F539
:104E9000A042044601921EB90121FFF795FF0BE0E5
:104EA00095F94822002A66DAD5F8540203689B6C0B
:104EB00098470646002842D04FF0000B95F948224B
:104EC000B44E002AC0F25981D6ED007AB4F9A4207C
:104ED000B8EE677A1AB9B4F8A220A4F8A420B4F8FE
:104EE000A430DFEDAD6A07EE903AF8EEE77A67EEB0
:104EF000A67AB4EEE77AF1EE10FAACBF01210021F8
:104F00002046FFF795FE95F94822002A95F8492298
:104F1000B8BF4BF0010B5306019B93F8502048BFDC
:104F20004BF0020B0AB14BF0080B32685946204691
:104F30000DB0BDEC0A8BBDE8F04FFFF73FBED5F8D2
:104F40007832204693ED0C8AF9F770FAB4EEC80A6D
:104F5000F1EE10FAB0D5D5F8783293F8A130032BE2
:104F6000AAD14EF0D3FD4FF4801142224EF086FDBF
:104F70003146204691E7019A92F85090B9F1000F1E
:104F800003D0844A0023136096E700F5804A93F823
:104F90000780DAF8840E03685B6F98470746009035
:104FA000D5F8540203685B69984720B1D5F84C32B4
:104FB000022B00F0E480B8F1000F0CBF4FF0000BA3
:104FC0004FF4007BB7EE00BA17B14BF4806B00963C
:104FD00004F5A047183738466AF034FB0130DAF898
:104FE000840E9FED6E0A9FED6ECADFED6E8A0CBFD8
:104FF000012302236C3008EE103A28F0EDF80CABD8
:10500000CDED0A0A8DED0B1A8DED090A13E90700A3
:105010000DF10C0E0DF1180C8CE807008EE807005E
:10502000704627F025FE04F58042DFED5F7AD2F866
:10503000842E92ED36AA2AEE27AAB4EECC0AF3EE1D
:105040000EBAF1EE10FA04F59C40B4EEEBAAC8BF1C
:105050004BF4807B3830F1EE10FAC8BF4BF4807B04
:10506000F0EE40AA51F0D2FE28F0B4FCB8EEC88AA7
:1050700004F59C40B4EEC80AF1EE10FA00F16800A5
:1050800098BF4BF0800BF0EE409A81F0C5F968EEC6
:10509000288AB0EEC09AB4EEE89AF1EE10FA2046F3
:1050A00048BF4BF0400B0AF0C1FA002847D14BF043
:1050B000200BB24638466AF0C5FA012850D14BF0B1
:1050C000100BB1463349B8F1000F54D0009B002BB0
:1050D00051D0F4EECCAAF1EE10FA4CDCB4EEEBAA0F
:1050E000F1EE10FA47DCF4EEC89AF1EE10FA42D86D
:1050F000B4EEE89AF1EE10FA3DD5BAF1000F3AD0CD
:10510000B9F1000F37D00A68B4F9A40007EE902A6D
:10511000B8EE677A18B9B4F8A200A4F8A400B4F8FD
:10512000A43007EE903AF8EEE77A67EE8B7AB4EEA9
:10513000E77AF1EE10FA19D501320A60BEE604F5FD
:105140003950203051F00AFEDFED187A90ED007AE8
:10515000B4EEE77AF1EE10FAA9D44FF0000AA9E70D
:1051600038466AF06FFA0130ACD1A8E70121204639
:10517000FFF72AFEA2E60022DFE70121C0E6B8F130
:10518000000FB0EE08BA0CBF4FF0000B4FF4007BDD
:105190001BE700BFC0850020CDCC4C3E9F0CB34523
:1051A0000080BB440000C842E02E65420000484336
:1051B00030B500F5B9531833044693E8070089B0B9
:1051C00002AD85E807009FED1D7ADDED047A77EEEC
:1051D000877A9FED1B7ACDED047AD4ED2B7AF0EE31
:1051E000E77AF4EEC77A04F59C40F1EE10FA00F18C
:1051F00038000BD5B4F9A23007EE903AF8EEE77A12
:10520000F7EE006A86EEA77A84ED2B7AD4F8AC30FC
:10521000019301AA294651F0C7FE2046FFF72CFE54
:105220002046FEF755F92046FEF730FA2046FDF7F6
:10523000E5FF2046FEF79CF809B030BD0AE81C41A6
:105240000000003410B504462DED028B1D205CF0EB
:10525000F1F960B304F54053D3F8540200F0BAFA00
:10526000192108EE100A04F5736048F055FD022874
:105270001AD00338012808D804F53950203051F0ED
:105280006DFD90ED008ABDEEC88AB8EEC88A9FED2C
:10529000090A28EE000ABDEC028B04F5A040183084
:1052A000BDE810406AF054BA9FED038AEDE7BDEC0B
:1052B000028B10BD0AD7233C00000000134A026095
:1052C000134A426002F17801816002F52951C16000
:1052D000043101610839416124398161A1F56A51C4
:1052E000C1610C49016202F62861416202F6EC11CB
:1052F000816202F51F61C16202F6F41102F6F81232
:105300004263054A01638263704700BFB03B0D08EA
:1053100088500020BC7A0020502D002017294BD83F
:10532000DFE801F0100C1417231F2B1B4A274A2F0C
:105330004A4A4A33364A3A4A4A3D414600F5A04075
:105340007430704700F5AE403430704700F5A1402E
:10535000FAE700F5A1407030704700F5A940083029
:10536000704700F5AB405830704700F5AA404C300C
:10537000704700F5AB401030704700F5AD40283065
:10538000704700F5A9404830704700F5A540FAE79E
:1053900000F5AC401430704700F5AE40DBE700F597
:1053A000AF404030704700F50050D0F8F80C70471F
:1053B00000F5AA40043070470020704773B50B68B1
:1053C00005461B6C08460C4616469847034605F5ED
:1053D00040500F4A00960421203052F095F950F0C9
:1053E00089F8236805461B68204698470A2102462B
:1053F00028464FF0DBFF074B93F849329B0641BF2D
:10540000054A137843F00403137002B070BD00BF67
:105410003C290D08385C00205C87002038B50C4A18
:10542000182305460C464EF0B9F978B121462846B6
:10543000FFF774FF30B10146064A2846FFF7BEFF6A
:10544000002038BD28464EF0EFF8F9E70120F8E7D4
:10545000BC290D085C290D0810B500F50053002289
:1054600083F8F42E094B044693F8481200F5804364
:1054700004F54054D3F8840EC9097AF0F5FDD4F848
:1054800054020368BDE81040DB681847385C002010
:1054900070B50546086803685B690C461646984770
:1054A00090B1306803685B69984768B905F5405367
:1054B000D3F8782292F8CB2032B193F94832002BFE
:1054C00002DB2846F8F7C8FF04480AF085FE20688A
:1054D0000368BDE870409B68184700BF9C860020A9
:1054E00070B500F540550446D5F854020B4E0368DC
:1054F000DB6998473074D5F8540203681B689847F5
:10550000F070D5F8540203685B6C9847014604F5C7
:105510009C501430BDE8704043F0D4B93D87002062
:1055200070B52DED028B244B93F86D32DB0782B002
:1055300006460D461446B0EE408AF0EE608A06D567
:1055400000232B60236002B0BDEC028B70BD5AF0CB
:10555000C5FC037F002BF3D0F36A9FED181A1B687C
:105560009FED170AB3F9083007EE103AB36A1B68CB
:10557000B3F9083007EE903AB8EEC77AF8EEE77A5A
:1055800067EE000A68EE811A27EE800A28EE011AFB
:1055900001A9684625F094FADFED0A6A9DED007ACC
:1055A000DDED017A27EE267A67EEA67A85ED007AA0
:1055B000C4ED007AC7E700BF385C00200AD7233C5F
:1055C000530469390000C84270B52DED028B88B0D4
:1055D000002302930393364B93F86D3213F0010FBF
:1055E0000646B0EE408A06AD02AC03D15AF076FC16
:1055F000037F5BB994E8030085E803009DED060A8C
:10560000DDED070A08B0BDEC028B70BDB36ADFEDBB
:10561000296A1B68B3F9083007EE903AF36A1B68F1
:10562000B3F9083007EE103AB8EEC77AF8EEE77A29
:1056300027EE267A67EEA67AF1EE476ACDED026A8A
:10564000DFED1D6ACDED037AB0EEC77AB4EEE67AEF
:10565000F1EE10FA06D5F0EEE77AF4EEE67AF1EE26
:1056600010FAC7D403AA21461448F8F725FFDDED48
:10567000027A9DED037AF0EEE77AB0EEC77AF4EEA7
:10568000477AF1EE10FACCBFB0EE670AB0EE470AE7
:10569000204627F03BFA04A88DED040ACDED050A5B
:1056A00027F0E6FA204688EE000A27F05FFAA1E725
:1056B000385C00205304693900000034382C002085
:1056C000094B93F94822002A0CDAB5EEC00AF1EE34
:1056D00010FA07D9D3F8783293F8A100C31E5842C4
:1056E0005841704700207047385C0020436A1B68AF
:1056F00093F8CB3043B1054B93F8480200F0A0007B
:10570000203818BF0120704701207047385C002006
:1057100010B5436A04461868D1B1022181F02CFE0D
:10572000236A9FED0C1A18680368F0EE410ADB6AE1
:10573000B0EE410A9847236A074A1868D2ED000A7A
:1057400003689FED040A5B6EBDE810400021184716
:105750000121E3E7000000009050002010B5436AEB
:1057600004461868002930D0022181F005FE236A22
:1057700018687AF049FC636A1B6893F8A130012B22
:1057800004D8236A012118687BF0D8F96369186886
:105790007EF0E4FA636918687EF040FB63699FED70
:1057A0000C0A18687EF066FD636918687EF0D4FD07
:1057B000236A9FED071A18680368BDE81040DB6A8A
:1057C000F0EE410AB0EE410A18470121CDE700BFD3
:1057D0000000000013B5044601A90C4809F0B6FF0B
:1057E00010B1019802B010BD636918687DF0C0F96E
:1057F00018B9074BD3F85C0EF4E7064801AA032159
:1058000012F0A4F90028F4D0EBE700BF382C0020F8
:10581000386C0020907A002070B504462DED028B84
:1058200000296AD18368B3F92E58642DB8BF642566
:10583000FFF7D0FFA8426268A4BF324B93F84952E9
:10584000B2F93430ACBFC5F380150125002BDBBFA6
:1058500063691B685B4293EDC48AC8BF07EE903A48
:10586000B2F93230C8BFB8EEE78A002BB8BF5B424E
:105870009BB25B4207EE903AA368F8EEE77AB3F981
:105880002E68F4EEC87AF1EE10FAD8BFB0EE678A4F
:105890002046642EB8BF6426FFF79CFF6369A26BA5
:1058A0001B68D2ED001A93EDC61AD3ED0E0A311A19
:1058B00000EE101AB8EEC00A24F0F0FC6368B3F9E9
:1058C0003230002BB8BF5B429BB25B4201EE103A14
:1058D00040F29720B8EEC11AF0EE480A24F0FCF925
:1058E0006369294618687DF0E7F9BDEC028B6369AE
:1058F000BDE8704018687EF02FBD9FED030A0025BB
:10590000EEE700BF385C002000000000436A186822
:1059100003681B691847000038B52DED028B03683A
:105920000446D3F880309847236B2A481B68F0EE72
:10593000408AB3F9085009F017FE4FF47A72041E3A
:105940004FF000012846D8BF4FF4FA7424F002FA51
:105950008442B6EE000A2ADD07EE900AB8EEE77A36
:1059600007EE904A27EE007AF8EEE77A87EE278A6C
:105970004FF46D7038EEC00AF5EE087AB1EE400AC9
:1059800080EE270AB7EE001AFEEE000A24F0A4F912
:10599000F7EE007A77EEC07A28EE000A20EE080AC9
:1059A00020EE080AA7EE880ABDEC028B38BD031B67
:1059B00007EE103AC4F57A74B8EEC77A07EE904A4B
:1059C00027EE007AF8EEE77A87EE278A38EE008A2B
:1059D000CEE700BF382C00202DE9F0472DED028BDB
:1059E00000F5A04300F5405893F8704083F870200C
:1059F0000546D8F85402036882B01B680F46164665
:105A00009847B84223D105F500531A2E83F80C6449
:105A100009D140B905F5804503F6D453D5F8842E55
:105A20001B68C2F8FC308D4B93F84932980606D4B7
:105A30000124204602B0BDEC028BBDE8F087B442E1
:105A4000F6D0874A137843F002031370F0E7022E72
:105A50000CD01B2F12D105F5A1403146703002B099
:105A6000BDEC028BBDE8F04701F06AB93946284623
:105A7000FFF7D4FC04460028EBD1DAE73946284684
:105A8000FFF74CFC0446019018B928464DF0CCFDB8
:105A9000CFE7D8F8783293F8CBA003685B699847D2
:105AA000019A05F5A94348338AF001099A4208BFD3
:105AB0000120BAF1000F08D10198036849465B68DC
:105AC0009847044648BB674A22E098F94832002BC1
:105AD00080F2B580002800F0B280DFF880A1DAF80B
:105AE000540203685B6998470446002840F0A78089
:105AF0000198FFF711FFAAF54050B0EE408AF8F781
:105B000095FCB4EEC08AF1EE10FA40F39880564A44
:105B100001992846FFF752FC8BE705F5495101AA88
:105B20001431284605F50054FFF7B2FC0198C8F877
:105B3000540284F80C6403681B6898473246014697
:105B400005F58F504EF0E8FF05F54050002120305C
:105B500059F0D8FA94F9FE3223B105F50B503830DC
:105B600066F01CFCD8F8540203681B689847C21EF4
:105B700005F580435042504104F6A45183F8140FB8
:105B8000D3F8842E0968C2F8F81004F6D451D3F87B
:105B9000842E0968C2F8FC10012F01D00B2F06D10A
:105BA00004F6BC54D3F8843E2268C3F8FC2028468F
:105BB000FFF796FC294B93F849329B063FF541AF1E
:105BC00036E705F5005393F8F822002A3FF474AF46
:105BD000B3F81423D1077FF56FAF93F83423002A6D
:105BE0003FF46AAFD8F8782292F8CB20002A3FF42D
:105BF00063AF93F80C340A2B7FF45EAF98F9483208
:105C0000002BFFF659AF194A01992846FFF7D6FB3A
:105C100000240EE7164809F013FF0028D1D1D8F868
:105C2000540203685B6998470028CAD0019803684A
:105C30005B69984704460028C3D10E4A68E701987B
:105C400003681B6998470028E4D0094809F0E6FE7C
:105C500004460028DED1084A5AE700BF385C00201D
:105C60005C8700203ED70E0884290D08A8290D085E
:105C7000382C002096290D08D2890E080148FFF71C
:105C8000ABBE00BF382C002013B504468DED010AD1
:105C900069F070FC6369A26B1B6892ED001A93EDCA
:105CA0000E0AD3EDC60A01A968F0F2FA9DED010AC9
:105CB00002B010BD436A186803685B6A18470000A9
:105CC00038B5436A1C6894F8CB10054661B9204684
:105CD00081F052FB6B6A1B6893F8A10018B1012890
:105CE00014BF0320022038BD164803783BBBFFF7E2
:105CF000E7FC20BB144A92F8483203F0A003202BA3
:105D000017D0B5EEC00AF1EE10FA10D592F84A326B
:105D10005B070CD40121204681F02EFB6B6A1B68C7
:105D200093F8A130012B0CBF02200320DBE70221F6
:105D3000F1E72046022181F01FFB0420D3E7012078
:105D4000D1E700BF9C860020385C002010B52DED07
:105D5000028B134B93F86D32DB07044604D59FED9D
:105D6000110ABDEC028B10BD5AF0B8F8037F002B6E
:105D7000F5D0636B18685AF0DBF9A368DFED0A7A97
:105D800003F5116292ED008A03F61413D3ED000AB5
:105D900028EE278A24F04EFE28EE000AE1E700BF35
:105DA000385C0020000000000000C8420148F8F7FD
:105DB000B1BB00BF382C00200148F9F74FB800BF35
:105DC000382C00200148FFF707BE00BF382C002008
:105DD00070B52DED028B7D4D95F849328CB00026C3
:105DE000044658060496059603D5636918687CF046
:105DF00033FD95F86D32D9075DD463689B899A07A6
:105E00001BD5734850F0AAFFDFED727A90ED007A4F
:105E1000B4EEE77AF1EE10FA0FDD4FF06BFB3D21A7
:105E20004FF0A4FA6C4809220521FFF7D5FD20B9EF
:105E3000092202212046FFF7C5FF636893F9543019
:105E4000CBB365489FED658AF9F708F8E3689FEDE5
:105E5000647A1B68D3ED0A7AF4EEC87AF1EE10FA90
:105E6000B8BFF0EE477AB6EE000A27EE800A204669
:105E7000FFF7AAFB8DED040AB0EEC00AB4EEC80A23
:105E8000F1EE10FACDED050A06D5F0EEE00AF4EEDB
:105E9000C80AF1EE10FA0ED495F84A321B0704D462
:105EA0004FF028FB49214FF061FA95F84A3243F050
:105EB000080385F84A3295F84B326FF3820385F870
:105EC0004B32606909960A9609AD2A4604A9006812
:105ED00001237CF02BFD636918687DF09FFF6369E7
:105EE00018687DF077F8A3688DED060ACDED070AF6
:105EF0008DED081AD3ED007AF5EEC07AF1EE10FAC6
:105F000052DD384B9FED388AB3F94C3400EE903AAD
:105F1000F8EEE00A2046CDED030AFFF75BFCA3682C
:105F2000DDED030AD3ED001A9FED2A0AB7EE002A31
:105F300007EE900A31EE822AB8EEE71A22EE082A1E
:105F400061EE881A23F008FEDFED287A20EE270A9A
:105F5000DFED277A20EE270AB0F062F9DFED257A2F
:105F600020EE270A06A820EE088A26F081FEB4EE6D
:105F7000C08AF1EE10FA17D5C8EE006A63699DED8C
:105F8000067ADDED077A27EE267A67EEA67A8DEDA2
:105F9000067ACDED077A1B68D3F88823C3F89423DB
:105FA000D3F88C23C3F89823236A13491C68284626
:105FB000FCF7ECFA0B9B009395E80C0006A9204631
:105FC0007AF0D4F80CB0BDEC028B70BD385C0020C8
:105FD000847A002000002F44382C00200000003478
:105FE00000007A43384C00200000C8420AD7233C06
:105FF00035FA8E3C0AE81C417485002013B504462E
:106000000191FFF7E5FE0199204602B0BDE810407E
:10601000FFF702BC0148FEF7D7BE00BF382C0020B6
:1060200000487047585C00200148F8F761BA00BF8B
:10603000382C002030B50F4D87B000230446694648
:10604000D5F88C0E0093019302937CF0DBFFD5F81A
:106050008C0E02A97DF02AF8009B0393019B049308
:106060000222029B059303A9204612F03FF8204626
:1060700007B030BD386C0020014B01221A70704708
:10608000C485002000207047002070470020704722
:1060900000207047002070470020704700207047A4
:1060A0000020704700207047002070479FED010AD4
:1060B000704700BF000000000020704700207047BC
:1060C0000020704701207047002070470020704773
:1060D0000120704700207047012070470120704761
:1060E0000020704701207047012070470020704752
:1060F00000487047D4290D0800487047D4290D087E
:10610000836893F82439DB0706D5002380F83C30F8
:10611000024B0222C3F84C2201207047385C002059
:1061200090F83C3043B9836893F82439DB0742BFC9
:10613000034B0122C3F84C22002380F83C30704707
:10614000385C0020012380F83C3070472DE9F04393
:106150002DED0C8BF0EE409A20EE000A97B0002552
:10616000A0EEA00A04468946B0EE41CAF0EE60AA4D
:1061700090461F4601950295039504950595069551
:10618000B0F064FAF7EE00CAB4EEEC0AF1EE10FAE1
:10619000C8BFCCEE807AA36803F50E6203F6E40371
:1061A00092ED009A9FEDC5DAD3ED000AC4BF69EE07
:1061B000A79A6AEEA7AAB0EE690A24F03BFCA3688E
:1061C00029EE0D9A03F50E6203F6E403D2ED008A80
:1061D000D3ED000A29EE009AB0EE6A0A24F02AFCF8
:1061E000A36868EE8D8A03F6F80203F6FC03D3ED8C
:1061F000000A92ED008A68EE808AB0EE4C0A24F024
:1062000019FC636828EE0D8A93F9703028EE008A35
:10621000002B00F0D980236A9FEDA90A18686C3022
:1062200026F0DAFFB0EE60AACDED080A8DED091A6E
:106230008DED070A23F0FAFCBDEEC0BAA14940F685
:10624000B8321BEE100A23F075FD434207EE903A78
:106250006368F8EEE77A93ED1A7A67EE877AB0EE24
:106260004A0ACDED017A23F0E1FCFDEEC0BA40F61A
:10627000B83294491BEE900A23F05CFD42426368F9
:10628000039507EE902A93ED1B7A93F97030F8EEA0
:10629000E77A022B67EE877ACDED027A6ED18A4BD0
:1062A000B3F94C340AEE103AB8EECBBAB8EECAAA3B
:1062B000236AB4EECABAF1EE10FA1A683DDDA3689B
:1062C000DFED820AA16B92ED051AD1ED001A03F5FC
:1062D0000E6393ED007A27EE0D7A3AEE4B0AC7EE85
:1062E000200A23F0DBFFDDED017A37EE800A8DED29
:1062F000010AB8EEEB0A236AB4EECA0AF1EE10FA0C
:106300001A6834DDA368A16B92ED061AD1ED001A6C
:1063100003F50E63D3ED000A20EE8DDADFED6B0A94
:106320003AEE400ACDEE200A23F0B8FFDDED027A06
:1063300037EE800A8DED020A20E0B1EE4A0AB4EE93
:10634000C0BAF1EE10FAD4D5A368A16BDFED5F0AF5
:10635000D1ED001A92ED051A03F50E6393ED007A64
:1063600027EE0D7A30EE4B0AC7EE200AB9E7B1EE00
:106370004AAAB4EECA0AF1EE10FAC3D4236AD3F8DB
:1063800000C00CF184030FCB12AD85E80F000EAEF8
:106390000AAD86E80F0085E80F0004AB01AA294684
:1063A00060467AF07FFB636893F97030022B16D158
:1063B000DDED047A39EE279ADDED057A78EEA78ACD
:1063C000DDED067A38EE278A89ED009AC8ED008A5D
:1063D00087ED008A17B0BDEC0C8BBDE8F083F0EEC2
:1063E000E99AF0EEEAAAF4EEE9AAF1EE10FA48BF53
:1063F0006D46CDED009ACDED0AAAD5ED007ADFED20
:10640000340AB0EECCCAF4EECC7AF1EE10FAD8BF72
:1064100035468DED0ECA95ED007ADFED2E7A87EECA
:10642000270AAD20B7EE001A3CEEC00A23F054FC58
:10643000E369D3ED937A04A820EE270A26F0CCFE78
:10644000F0EEC07A8DED061AB0EEC91A31EE671A79
:106450008DED040AB0EEC11A39EE000ACDED050A41
:10646000B520F1EE410A23F037FCB0EE409A9DEDE5
:10647000050AB0EEE81AF0EEC07A31EE671A38EE8F
:10648000800AB0EEC11AF1EE410ABA2023F024FCD2
:10649000F0EE408A9DED060AB0EEC81AF0EEC07A22
:1064A00031EE671A38EE000AB0EEC11ABF20F1EEE5
:1064B000410A23F011FCB0EE408A85E70000C84293
:1064C0009F0CB34548F4FFFF384C002000007A448D
:1064D0000000000000A08C4510B52DED028B836AF2
:1064E000044686B0186859F023FEE36A1868B0EED7
:1064F000408A59F01DFE636B8DED010A186859F052
:1065000017FE05ABB0EE401A03A92046DDED010AE7
:1065100004AAB0EE480AFFF719FE636A186890F8FB
:10652000CB1000293AD180F027FF2046FFF7F4F97D
:10653000636A1B6893F8A1100129B0EE408A3DD030
:10654000032944D051B9236A012118687BF0ACF9C2
:10655000236A186879F042FD9FED208A236AA268B9
:10656000186892F8242903689DED030ADDED040AFA
:106570009DED051A92074CBFDB6B9B6B9847236A16
:10658000174A1868D2ED000A036800215B6EB0EE6E
:10659000480A984706B0BDEC028B10BD114B93F929
:1065A0004922002A06DBD3F84C32022B04D190F8A2
:1065B000A1300BB90121B6E70221B4E7236A1868BC
:1065C0007BF072F9236A186879F01EFDC4E7D97967
:1065D0000029C3D12046FFF71DFDBFE700000000E2
:1065E00090500020385C0020836893ED040AB5EEDB
:1065F000C00AF1EE10FA01DCFFF788B9704700001D
:10660000704700000020704701207047022070474B
:10661000002070470020704701207047002070471D
:1066200081F0010070470000012070470120704791
:10663000004870476C2A0D0800487047782A0D08FA
:1066400038B54369044618687CF0B4FB18B963692F
:1066500018687DF033FD636920461D68FFF7E4FC90
:106660006368B3F93820B3F9363000EE903A43420C
:1066700001EE102A00EE103AB8EEC11AF8EEE00A68
:10668000B8EEC00A28467CF081FA636920461D688E
:10669000FFF7CAFC6368B3F93820B3F9363000EE6F
:1066A000903A434201EE102A00EE103A2846B8EE26
:1066B000C11AF8EEE00AB8EEC00A7CF0E1FA012057
:1066C00038BD000030B52DED028B0446436985B01E
:1066D0001D68FFF7A9FC6368B3F93820B3F93630B9
:1066E00000EE903A434201EE102A00EE103AB8EE66
:1066F000C11AF8EEE00AB8EEC00A28465B4D7CF0FD
:1067000045FA2046FFF758FBB5F94C3408EE103A2D
:10671000236A186803689B6E9847B8EEC88AF0EE43
:10672000400A02AA01A9B0EE480A2046FEF7F8FE88
:106730002046FFF70BFB236B1B68B3F90830F0EE24
:10674000408A00EE103A2046B8EEC00AFFF72EFB52
:106750002046B0EE408A8DED030AFFF765FC6368C2
:10676000B3F9363001EE103A434200EE903AB8EEFB
:10677000C11AF8EEE00A2B20B0EE480A23F0ACFA7A
:1067800020468DED030AFFF79BFA042813D8DFE8B3
:1067900000F0032F252A4B00236A186879F01EFCAD
:1067A000236A002118687AF0C9F963699FED300AFD
:1067B00018687DF05FFD236ADDED020A18689DED23
:1067C000010A0368B0EE681ADB6A984763691868C3
:1067D0007DF0C2FD05B0BDEC028B30BD236A012106
:1067E00018687AF0ABF9236A186879F00DFCDCE7D9
:1067F000204D2B7863B963689FED1F1ADFED1C0AEB
:1068000093ED040A452023F067FA284609F0CCFCF2
:1068100020469DED030AFFF737FA16488DED030A6F
:1068200003A909F0FBFCC6E7636A0221186880F03F
:10683000A3FDB5F94C34114800EE103A02AA01A9A3
:10684000B8EEC00A67F054FA20469DED030AFFF740
:106850001BFA0B488DED030A08F096FF63699DED66
:10686000030A18687CF018FAA5E700BF384C00202E
:10687000000000009C86002000007A44E07B00209D
:10688000205B00200020704790F8B931002B14BF26
:106890001B20032070470000002070470120704734
:1068A00090F89001062804D0A0F10A0358425841FC
:1068B0007047012070470000012070470120704799
:1068C00090F8B901034A044B002814BF104618463B
:1068D000704700BF102B0D08FF9D0E0890F8B901FE
:1068E000034A044B002814BF10461846704700BFE7
:1068F0001C2B0D08FF9D0E0890F890010B3818BF57
:106900000120704790F8B9312BB9044BD3F8F00D42
:1069100000F0010070470020704700BF384C002095
:1069200090F8903123B9034B187880F0010070473C
:10693000002070478086002038B590F89041012CE7
:10694000054601D0002038BDC368186803681B697C
:1069500098470028F6D1EB681B68204683F8B848B2
:10696000F1E70000C3681B68002283F8B828012003
:106970007047000070B52DED028B002380F8B9310F
:10698000B0F87030012B84B004460D4601D80029C0
:1069900046D0636A254E1B6893F8CB3073BB2448FE
:1069A000072384F890310368022B02D10021FBF702
:1069B000F7FB9FED208AE368F0EE480A1868B0EE16
:1069C000481AF0EE481AB0EE480A01257EF04AFF58
:1069D00084ED738A84ED748A84ED758A84F8B851E5
:1069E00004F59A7027F0E0F8134804F0FFFD96F8DC
:1069F0004A326FF3C30386F84A3211E096F94832FF
:106A0000002BCCDA04F13C0029F0A6F90546002859
:106A1000C5D12046FFF704FB084A022150F074FE5E
:106A2000284604B0BDEC028B70BD00BF385C00206E
:106A3000748500200000000084810020242B0D08B4
:106A400010B50446094890F83031012B03D100F508
:106A5000967027F011F9064890F89D1F00F62470F3
:106A60005BF0BEFE002384F8B93110BD387C0020F5
:106A7000386C002010B52DED028B094B0446D3F87D
:106A8000900EB0EE408A7EF085FA9FED060A28EE61
:106A9000008A012084ED748ABDEC028B10BD00BF1A
:106AA000386C00200AD7233C10B52DED028B094B22
:106AB0000446D3F8900EB0EE408A7EF07BFA9FED4C
:106AC000060A28EE008A012084ED758ABDEC028B4F
:106AD00010BD00BF386C00200AD7233C10B52DED47
:106AE000028B094B0446D3F8900EB0EE408A7EF03C
:106AF0006FFA9FED060A28EE008A012084ED738A62
:106B0000BDEC028B10BD00BF386C00200AD7233CBF
:106B1000C3681B6818697CF08FBB000038B5D0F8DB
:106B2000943104460D461BB988F0FCFBC4F894016F
:106B300088F0F8FBD4F89431C01A4FF47A73B0FBA4
:106B4000F3F0B4F89231984209D32046FFF768FA7F
:106B50002B88044A062150F0D7FD012038BD0020C3
:106B6000FCE700BF402B0D0890F89031052B05D1B4
:106B7000054BD3F8983ED8687CF0D6BAC36818683D
:106B80000368DB68184700BF386C002008B590F830
:106B90009031052B0BD1094BD3F8983ED86824309F
:106BA00026F066F8BCEEC00A10EE100A08BDC368F5
:106BB000186803689B689847F4E700BF386C0020AA
:106BC00090F890318B4206D00B2B80F8901102D1B7
:106BD0000148FCF7C3BF7047382C002073B5012370
:106BE0001E4E80F87530D6F85432834205460A4668
:106BF00014D1012485F8B941D6F8540201920368F2
:106C00001B689847019A014615484DF085FF96F894
:106C100049329A061BD4204602B070BD019103216F
:106C2000FFF7D0F8019A04460028E2D185F87500F4
:106C30004EF060FC1B220A214EF0B8FB96F8493258
:106C40009B06E8D5074A137843F0040303E0054A9E
:106C5000137843F002031370DDE700BF385C0020B7
:106C6000183E00205C87002030B585B004460D46F4
:106C700001466846FFF7DEF9694604F13C0029F059
:106C80001DFEC8B94EF036FC1B220A214EF08EFBC9
:106C90000D4B93F849329B0604D50C4A137843F008
:106CA000040313702046FFF7BBF9094A042150F092
:106CB0002BFD002005B030BD2946204605B0BDE8BB
:106CC0003040FFF78BBF00BF385C00205C8700209E
:106CD000542B0D0830B585B004460D460146684674
:106CE000FFF7A8F9694604F13C0029F00BFEC8B98A
:106CF0004EF000FC1B220A214EF058FB0D4B93F87E
:106D000049329B0604D50C4A137843F004031370F0
:106D10002046FFF785F9094A042150F0F5FC0020D0
:106D200005B030BD2946204605B0BDE83040FFF72C
:106D300055BF00BF385C00205C870020902B0D08F9
:106D40007FB505460E4605F13C0401466846FFF74F
:106D500071F96946204629F0D5FDC0B9204669463B
:106D600029F0ACFD044690B94EF0C4FB1B220A2169
:106D70004EF01CFB0D4B93F849329B060FD428466E
:106D8000FFF74EF90A4A042150F0BEFC04E03146F8
:106D90002846FFF723FF0446204604B070BD054A8D
:106DA000137843F004031370E9E700BF385C002058
:106DB000C82B0D085C87002030B5044685B00F480D
:106DC00008F02CFE0546B0B1072384F8903100236B
:106DD000019302930393E36801A918687EF074F8A5
:106DE000E3681868036801A95B68002298470448B3
:106DF0000021FBF7D5F9284605B030BD382C00201E
:106E000074850020F0B5424FD7F8642ED7F8603E65
:106E10002DED028B1343D7F85C2E134387B0054644
:106E20000C460CD14CF072FE40F275124FF48011FA
:106E300007B0BDEC028BBDE8F0404CF01FBE80698E
:106E40007FF0DEFA2046B0EE408A10F073FE032891
:106E50003AD1EB6801A918687EF012F9064698B39A
:106E6000DDED017A6368009338EE678A294BDFED28
:106E70002A7A93F948329FED290A2948002BA8BFA6
:106E8000B0EE670A38EE008A009BBDEEC88A00218A
:106E900018EE102A9342ACBF00930092FBF780F9E2
:106EA0006B6918687DF00AF9DDED007A1D48B8EECF
:106EB000E70A314609F032FC00212846FFF780FE40
:106EC00007B0BDEC028BF0BD94E80F0002AE86E87F
:106ED0000F00D7F8603E04936A46D7F8643E0593E6
:106EE0000221304610F032FE78B94EF003FB022248
:106EF00015214EF05BFADDED037AF8EEE77A77EED6
:106F0000887AFDEEE77ACDED007A0026AEE700BF85
:106F1000386C0020385C0020000000000000C842EF
:106F2000748500208086002030B52DED028BC3686B
:106F300087B0044618680D467EF096F800284BD1BD
:106F400094F8902100230093019302936AB9314889
:106F5000039303A90493059309F012FC28B1039B42
:106F60000093049B0193059B029394ED730A9FED9C
:106F70002A8AE368DDED000A9DED011ADDED021AB3
:106F80001868B4EEC80AF1EE10FAAABFDFED237A52
:106F90009FED230A20EE270A7EF064FCD4ED747A7C
:106FA000F4EEC87AF1EE10FA07DBE3689FED1B0AF6
:106FB000186827EE800A7DF0EDFFD4ED757AF4EEC7
:106FC000C87AF1EE10FA07DBE3689FED140A18683F
:106FD00027EE800A7DF0EEFFE368294618687EF010
:106FE00069FB054688B10F4B1B68022B09D0032BA8
:106FF00003D10D4B93F97D341BB10A480021FBF7F7
:10700000EFF801212046FFF7DBFD284607B0BDEC75
:10701000028B30BD80860020000000340000C84292
:107020000000000074850020384C002010B52DEDC4
:10703000028BC368DFED348A1B684269D3ED0A0A0C
:107040009FED328A93ED060AF4EEE80A0446F1EE6B
:1070500010FA1068B8BFF0EE480A7BF07DFBE368D9
:1070600062691B681068D3ED0A0A93ED060AF4EE14
:10707000E80AF1EE10FAB8BFF0EE480A7BF0E4FB44
:10708000636918687BF074FD18B9636918687CF04F
:10709000AFFDE36862691B68106893ED080A93ED21
:1070A0000C1AD3ED070AB0EEC00A7BF06FFDE3685F
:1070B00062691B68106893ED080A93ED0C1AD3ED12
:1070C000070AB0EEC00A7BF0DBFD636918687BF04D
:1070D00071FE18B9636918687CF0F0FF00210C4854
:1070E000FBF75EF80B4868F0CBFB0B4AB2F84A326C
:1070F00023F48163A2F84A32BDEC028B20460221C0
:10710000BDE81040FFF75CBD0000003400007A438A
:1071100074850020507C0020385C002010B50C4B9A
:107120000446D3F8980E90ED0B0A90F8502000F129
:107130001C017DF011FC07480368022B02D00821D6
:10714000FBF72EF820460521BDE81040FFF738BDBB
:10715000386C002074850020F0B52DED028B4A4D6F
:10716000DFED4A8AB0EE408A8FB00446D5F8980E1B
:107170000E4617467DF066FAF0EEC87AF4EEE87A2D
:10718000F1EE10FA07D49FED420AD5F8980E28EEDA
:10719000000A7DF0BDFAD5F8980E90ED0B0AB0EE1E
:1071A000C00A0FB1B1EE400A7DF0A2FA0023D5F873
:1071B000980E079302AA07A9089309937DF0C4FAD1
:1071C000DFED347A9DED027AB4EEE77AF1EE10FA53
:1071D00056DD022207A90AA810F088FF7168019104
:1071E000304610F0A7FC019902460AA810F078FC7E
:1071F000E3680AA918687EF05DFA10B92648FDF721
:1072000095F8A0697FF0FAF802684368D5F8980EFF
:10721000049303A91C30039225F05CFC05A88DEDB6
:10722000050ACDED060A25F023FD1C4B1B68022B39
:107230001BD0D5F8983E1948D3ED0A7AF4EEE87AD7
:10724000F1EE10FAB8BFD3ED047AF4EEC07AF1EEA5
:1072500010FA4FF0000110D5DFED117AB4EEE70A15
:10726000F1EE10FA09DDFAF7BBFF04212046FFF723
:10727000A7FC0FB0BDEC028BF0BDFAF791FFF4E76D
:107280002046FFF74BFFF4E7386C00200000003485
:107290000000C84200009643382C0020748500206E
:1072A0000000FA4370B52DED028B294BDFED298AE2
:1072B000D3F8904ED3F88C5ED4ED0A0A9FED268A5F
:1072C00094ED060AF4EEE80AF1EE10FAB8BFF0EE1B
:1072D000480A064628467BF03FFAD4ED0A0A94EDA8
:1072E000060AF4EEE80AF1EE10FAB8BFF0EE480A2A
:1072F00028467BF0A9FA28467BF03AFC10B92846CC
:107300007CF076FC94ED080A94ED0C1AD4ED070A93
:10731000B0EEC00A28467BF039FC94ED080A94EDE3
:107320000C1AD4ED070A2846B0EEC00A7BF0A8FC80
:1073300028467BF03FFD10B928467CF0BFFE074889
:107340000021FAF72DFFBDEC028B0123337070BDD5
:10735000386C00200000003400007A43748500205F
:1073600008B50748D0F8F03D9B0704D50121A0F5EA
:107370000050F6F723FFBDE80840024809F02EB898
:10738000384C00208086002030B589B00446FEF7D6
:10739000ADF930B10021204609B0BDE83040FEF71C
:1073A000DDB9636A022118687FF0E6FFE3681868B8
:1073B00003685B69984701461048FCF7B3FE6369B0
:1073C00018687CF0C9FF236A1D68636918687BF040
:1073D00001FE05AC20460A498DED020ACDED030AF7
:1073E0008DED041AFBF7D2F8079B009394E80C008C
:1073F00002A9284678F0BAFE09B030BD382C00202A
:107400007485002038B50446FEF770F9054628B1AA
:1074100020460021BDE83840FEF7A0B9636A02218A
:1074200018687FF0A9FF29462046BDE83840FEF7DE
:10743000E5BD00000148002106F0E4BBE082002029
:1074400030B5174D9FED170A05F5804389B0044606
:10745000D3F8980E7DF0E0FA01462846FCF762FE6C
:10746000636918687CF078FF236A1D68636918688F
:107470007BF0B0FD05AC20460B498DED020ACDED49
:10748000030A8DED041AFBF781F8079B009394E83B
:107490000C0002A9284678F069FE09B030BD00BF93
:1074A000382C0020000000007485002030B589B021
:1074B0000446FEF71BF930B10021204609B0BDE8B3
:1074C0003040FEF74BB9636A022118687FF054FF21
:1074D000E368186803685B69984701461048FCF741
:1074E00021FE636918687CF037FF236A1D686369B1
:1074F00018687BF06FFD05AC20460A498DED020A45
:10750000CDED030A8DED041AFBF740F8079B0093BD
:1075100094E80C0002A9284678F028FE09B030BD96
:10752000382C00207485002030B52DED028B83B0FF
:107530000446FEF7DBF820B9636A1B6893F8CC3089
:1075400043B90021204603B0BDEC028BBDE83040BA
:10755000FEF704B994F89831DA071DD4E3681D6882
:107560002B6828469B689847D5ED097A94F898319E
:10757000B4EEE70AF1EE10FA4CBF0122002262F3EA
:10758000000384F8983107D4204603B0BDEC028B89
:10759000BDE83040FFF7F8BE94F898319B0734D42B
:1075A000E368DFED458A1B686269D3ED0A0A9FED47
:1075B000438A93ED060A1068F4EEE80AF1EE10FA39
:1075C000B8BFF0EE480A7BF0C7F8E36862691B6851
:1075D0001068D3ED0A0A93ED060AF4EEE80AF1EE1C
:1075E00010FAB8BFF0EE480A7BF02EF9636918680C
:1075F0007BF0BEFA18B9636918687CF0F9FA94F860
:10760000983143F0020384F898312D4BD4F8A0212F
:10761000D3F85C3E9B1A07EE903AB8EEE78AF1EE9B
:10762000047AB0EEC87AB4EEE77AF1EE10FA38D503
:1076300094F8983143F0040384F89831204684ED9F
:10764000678AFEF7C5FB6369A26B1B68D2ED001A5F
:1076500093EDC61AD3ED0E0AB1EE480A22F01EFED3
:1076600063691B6840F2AA4093EDC31AD3EDC40AC4
:1076700022F032FB2046FEF707FB12488DED010A8F
:1076800008F082F863699DED010A18687BF004FB3D
:107690006369186803B0BDEC028BBDE830407CF034
:1076A0005BBED4ED677A68EE277AF5EEC07AF1EE2C
:1076B00010FAC3D5BCE700BF0000003400007A43D5
:1076C000386C0020205B002030B52DED028B83B09C
:1076D0000446FEF70BF820B9636A1B6893F8CC30B8
:1076E00043B90021204603B0BDEC028BBDE8304019
:1076F000FEF734B86369DFED347A1B6894ED710AE4
:1077000093EDC31AD3EDC40A20EE270A40F2C44019
:1077100022F0E2FA2046FEF7B7FA236A18680368F7
:107720009B6EB0EE408A9847284BB3F94C3407EE75
:10773000903AB4F8BC316425F8EEE77A13FB05F310
:10774000B4EEE70A07EE103A94F9BE31F1EE10FA02
:10775000D8BFF0EE407A13FB05F39FED1D0AF8EE5B
:10776000C76A07EE103AF4EE407AB8EEC77AF1EE47
:1077700010FA58BFB0EE670A6846CDED006A8DED8D
:10778000017A25F0C7FA236ADDED010A1868B4F81A
:10779000C03102689DED000A126B13FB05F301EE88
:1077A000103A0121B8EEC11A90476369B0EE480A59
:1077B00018687BF071FA636918687CF0CDFD03B03E
:1077C000BDEC028B30BD00BF0000C842384C002029
:1077D00000007A442DE9F0432DED028BB64F85B0C1
:1077E0000446D7F85402FDF781FF48B1D7F8540298
:1077F000002105B0BDEC028BBDE8F043FDF7AEBF44
:1078000007F58056D7F8780202217FF0B5FDD6F84B
:10781000843E93ED378A87F085FDB7F8483203F44C
:10782000814305467BB1D6F88C0E7BF015F82378A2
:10783000022B08D156F048FEA04BA14A06214FF07A
:1078400063FF0323237063F03DFD63F027FD48B120
:1078500063F038FD63F02CFD20B12378012B10D9A3
:10786000022B1DD02378082B00F28581DFE813F06E
:107870002100390063000A013E0145015A015C0103
:107880002A0056F021FE8D4B8E4A06214FF03CFF18
:10789000D6F88C3ED3F85433636108232370E1E7B4
:1078A00056F012FE854B884A06214FF02DFF032328
:1078B000F4E7D6F8900E03681B69984710B120468C
:1078C000FFF7F0FC2378082B00F27381DFE813F058
:1078D0005C01640164017A017A017A017A01820112
:1078E0008201A560D6F88C3E9FED787AD3F85433A8
:1078F0006361774B03F56362D2ED007AF4EEC77AE9
:10790000F1EE10FA4EDB9FED737A67EE877AD6F8C8
:10791000903E93ED087AB0EEC77AF4EE477A4FF0D6
:107920007E53F1EE10FA48BFB0EE677A236102236E
:1079300084ED067A2370D4ED016A9FED647AD6F85F
:107940008C3EF0EEE67AF4EEC77AF1EE10FA0AD445
:10795000D4ED057A93EDD56A77EEC67AF4EEE76A50
:10796000F1EE10FA29D4DFED5C6AD4ED067A67EE09
:10797000A67AD3EDDB6AF4EEE76AF1EE10FA26DCC4
:10798000A368D4ED047AEB1AB3F5FA6F21D2B4EE02
:10799000678AF1EE10FAC8BFB0EE678A84ED048AF8
:1079A000E5608FE7B3F98234002BB8BF5B429BB22E
:1079B00007EE903AF8EEE77AA9E70623237056F02F
:1079C00083FD3E4B454A04214FF09EFE7AE7A560B9
:1079D00078E7DFF8FC8008F62463D3ED006A67EEF1
:1079E000A67AF4EEC87AF1EE10FAD9D408F628692E
:1079F000D9ED007AF4EEC77AF1EE10FA22DB98F8AE
:107A0000583E33B90623237056F05EFD2B4B344AA3
:107A1000D9E7A8F5005007F009FE98B198F96E3E35
:107A200083B9B8F95A3ED9ED007ADFED2A6A07EE3C
:107A3000103A67EEA67AB8EEC77AB4EEE77AF1EEBE
:107A400010FAADDCE068281AB0F5FA7F7FF63AAF9D
:107A50000323237008F6246856F036FD98ED007A6B
:107A6000D4ED047A67EE277A054617EE900AF4F70C
:107A70004BFD124B1B4ACDE90001062128464FF071
:107A800043FE1FE7D6F88C0E7CF094FB63F01AFCE3
:107A900063F004FC68B156F017FD084B124A06214A
:107AA0004FF032FE63F00EFC63F0E6FB042323701C
:107AB00008E70523FBE700BF385C0020142C0D0805
:107AC000222C0D082C2C0D08432C0D08000000342E
:107AD000384C00200000C842333373BF552C0D08CA
:107AE000702C0D08A02C0D08C82C0D0863F0EAFBC3
:107AF00063F0D4FBC0BB05232370404BE068DFED8F
:107B0000407AD3ED006A9FED3F7A2D1AA6EEA77A50
:107B100007EE905AF8EE677AF4EEC77AF1EE10FAB3
:107B20003FF5D0AE07232370D6F88C3E9FED367A12
:107B3000D3EDC37AD3EDC66A67EE877AB6EE007AE4
:107B400067EEA77A67EE877A87EEA67AD4ED057A94
:107B500077EEC77A93EDD57AF4EEC77AF1EE10FAA4
:107B60003FF6B0AE0823A2E763F0ACFB63F0A0FBE6
:107B70000028C0D1A6E64BF0C9FF40F29C524FF45A
:107B800080114BF07BFF9DE6204805B0BDEC028BD9
:107B9000BDE8F043FFF7F8BBD7F85402FEF718F939
:107BA00094ED060A0121B1EE400AD6F88C0E7BF066
:107BB00083F8D6F88C0E05B0BDEC028BBDE8F0431F
:107BC0007CF0CABBD7F85402FEF702F99FED100A09
:107BD0000021EAE79FED0E8AD7F854028DED038A63
:107BE000FEF7F6F8D6F88C0E0123B0EE480A03AA89
:107BF00004F114017BF066FEDBE700BF645A00204D
:107C000000007A440000FA43CDCCCC3D287D002012
:107C10000000000030B590F8B83185B00446F3B1EB
:107C200068460FF057FF424869460AF0FBFC50B126
:107C300004F13C0028F02EFE002384F8B83104F54E
:107C40009A7025F0B1FF94F890310B2B2DD8DFE816
:107C500003F0294C50544C582C5C60642C6800F59F
:107C60009A7025F0A1FF04F13C0590B194F84030E2
:107C7000012B0ED194F89031012B0AD1284628F01F
:107C800077FC50B12046FEF7CBF92A4A02214FF08B
:107C90003BFD284628F09AFCD5E72046FEF7C0F9C0
:107CA000254AF3E72046FFF75BFB94F844303BB9E5
:107CB00094F8463023B994F840309A1E5342534109
:107CC00094F8B9218AB383BB84F8B9311B4CD4F83A
:107CD000540203681B6898472D220146A4F5F15011
:107CE00005B0BDE830404CF017BF2046FFF74CFB15
:107CF000DBE72046FFF786FBD7E72046FFF79AFB36
:107D0000D3E72046FFF79CFBCFE72046FFF7CEFBEB
:107D1000CBE72046FFF708FCC7E70948FFF75AFD05
:107D2000C3E72046FFF7D0FCBFE705B030BD00BF7A
:107D300020400020E42C0D080C2D0D08385C00209C
:107D4000C48500202DE9F0412DED028B074684B05B
:107D500008460E460FF0EEFE032880466D4628D1F9
:107D6000FB6818687CF0E6FF012822D121482946EB
:107D700007F0ECFC0446B0B17B69DDED007A1B68CE
:107D8000F8EEE77A93EDF27A77EEC77A4246FDEEA7
:107D9000E77A17EE901AC829CDED007AB8BFC8214E
:107DA00030460FF09DFE204604B0BDEC028BBDE8CE
:107DB000F081114B0FCB85E80F0030460FF0BAFE73
:107DC000014628460FF01EFF04460028EBD07B69D1
:107DD000DDED017A1B68B8EEE78AD3EDF27A28462A
:107DE00038EE678A0FF0A6FEBDEEC88A024618EE8E
:107DF000101AD5E7382C0020907A002010B543697E
:107E00009FED126A1B68D3EDF06A93EDF17AD3ED22
:107E1000F27A86B066EE866A27EE067A67EEC67A52
:107E200068460C46CDED006A8DED017ACDED027A03
:107E300025F096F903A920468DED030ACDED040A3D
:107E40008DED051A10F0A6F906B010BD0AD7233C37
:107E500030B5083204461D460FCA84E80F001343AC
:107E600001BFAB68A360EB68E360636885B093B95A
:107E700020460FF05FFE03AA014628460FF066FE7B
:107E800060B10399019120460FF054FE019902461A
:107E900020460FF025FE204605B030BD69680191EF
:107EA0002846F1E730B50B6985B004460BB94B693C
:107EB00053B30023C4F8B43108310FC96D4685E8C7
:107EC0000F0029462046FFF73DFF98B9124B0122CB
:107ED000D3F85C1E28460FF003FE4DF00BFB022288
:107EE00015214DF063FA2046FEF79AF80B4A02215D
:107EF0004FF00AFC29462046FFF716F810B908484B
:107F0000FCF714FA05B030BD0123C0F8B43105B058
:107F1000BDE83040FFF78AB8386C0020402D0D08CE
:107F2000382C002070B51A4B04460E460FCB88B093
:107F30006D4685E80F0020462946FFF75FFFE3689E
:107F400018687DF091F898B1E368186803681B69B8
:107F5000984768B1E368294618687CF0F7FE38B99D
:107F60004BF0D4FD40F295624FF480114BF086FD4A
:107F7000214604A82B463246FFF76AFF04A9204693
:107F8000FEF7D2FF10B90348FCF7D0F908B070BD76
:107F9000907A0020382C002070B5154B0C46064610
:107FA0000FCB88B06D4685E80F0029463046FFF7B5
:107FB00025FF2B462246314604A8FFF749FF628879
:107FC000A388122A4FEA132305D1227ED20744BF89
:107FD00003EB83035B00227A07EE903AC2F3400280
:107FE000B8EE670A04A93046FFF7B6F808B070BDCE
:107FF000907A002038B504460D46FFF793FF002322
:10800000C4F89431AB88A4F8923138BD7FB50D46E1
:108010000446FFF787FF05F108010FC96E4686E8A1
:108020000F00134306D1234BD3F8602ED3F8643EE0
:108030000292039304F5D072012130460FF086FDC1
:1080400094F8983170B923F0050343F0050384F8E0
:1080500098312046FDF7E4FF174A06214FF054FB04
:1080600004B070BD23F0070384F898310023C4F8EE
:108070009C31E36862691B68106893ED080A93ED10
:108080000C1AD3ED070AB0EEC00A7AF07FFDE36860
:1080900062691B68106893ED080A93ED0C1AD3ED22
:1080A000070AB0EEC00A7AF0EBFD08212046FEF781
:1080B00087FDD5E7386C00206C2D0D082DE9F043C5
:1080C0008DB06D4688461C46074613460A46014653
:1080D0002846DDE91469FFF7BBFE95E80F0084E848
:1080E0000F0007A80FF0F6FCB8F80430F3B9B8F8A1
:1080F0000010013105AA89B207F13C0027F0E4FD28
:10810000A0B1234605AA39462846FFF7A1FE95E807
:108110000F0086E80F00BDF81630A3F1520253425B
:10812000534189F800300DB0BDE8F08394E80F00AA
:1081300086E80F000023F4E770B58B8892B0044600
:108140000D461646002B47D10DA80FF0C3FC298819
:1081500001310BAA89B204F13C0027F0B5FD0028DB
:108160003AD0BDF82E1052291CD019D8112913D895
:108170000F2913D933462A46214603A8FFF768FE84
:1081800003AB214607A80BAAFFF762FEE36807A925
:1081900018687DF0CFFA01E01329EBD012B070BD62
:1081A0005E29FAE707AD03A80FF094FC28460FF00C
:1081B00091FC0DF10B03CDE90053324603AB0BA943
:1081C0002046FFF77BFFE0689DF80B3000682A46E9
:1081D00003A97DF085FAE1E70120DFE770B5214BC7
:1081E00004460E460FCB88B06D4685E80F0020464A
:1081F0002946FFF703FEE36818687CF035FF98B165
:10820000E368186803681B69984768B1E368294602
:1082100018687CF09BFD38B94BF078FC40F2166290
:108220004FF480114BF02AFC214604A82B4632461D
:10823000FFF70EFE04A92046FEF776FE20B90A4895
:10824000FCF774F808B070BD0023C4F89431B3880B
:10825000A4F8923104AA31462046FFF76DFF0028AA
:10826000F0D1ECE7907A0020382C0020F0B5324BAA
:1082700004460E460FCB91B004AD85E80F002046B2
:108280002946FFF7BBFDE36818687CF0EDFE98B166
:10829000E368186803681B69984768B1E368294672
:1082A00018687CF053FD38B94BF030FC4FF4DF62B6
:1082B0004FF480114BF0E2FB0CAF08A80FF00AFC62
:1082C00038460FF007FC0DF10F03CDE900732A4685
:1082D00008AB31462046FFF7F1FEE0689DF80F300D
:1082E00000683A4608A97DF041FD20B91348FCF723
:1082F0001DF811B0F0BD0023C4F89431B388A4F880
:10830000923108AA31462046FFF716FF0028EDD02B
:108310000B4B1B68022B09D0032B03D1094B93F99C
:108320007D341BB106480021F9F75AFF0121204690
:10833000FEF746FCDDE700BF907A0020382C0020D5
:1083400074850020384C002037B504460D4686F071
:10835000E9FFC4F8A801D5ED027AF5EEC07AF1EE96
:1083600010FA17DD9FED137A67EE877AFCEEE77A55
:10837000C4ED697A2046FDF753FED4F8A4214FF4EA
:108380007A73B2FBF3F30C4A062103B0BDE8304028
:108390004FF0BAB963F086FA0023009395F90D20E7
:1083A00095F90E3095F90C1063F018FAC4F8A40191
:1083B000E0E700BF00007A44842D0D0810B5B1F944
:1083C0000A30A0F8BC3191F90C3080F8BE31B1F917
:1083D0000D30A0F8C031B1F90F3007EE903AF8EE49
:1083E000E77A0446C0ED717A86F09CFF0B21C4F851
:1083F000C8012046BDE81040FEF7E2BB38B5044690
:108400000D4686F08FFFC4F8B001D5ED027A9FEDDE
:10841000047A67EE877AFDEEE77AC4ED6B7A38BDB1
:1084200000007A444A7C06480B46003A91F9101045
:10843000D3ED030A93ED020A18BF0122F9F7DABE61
:108440007485002070B51B4E0446D6F854020368AC
:1084500086B01B680D469847042806D16B88102B00
:108460000FD0732B20D000201CE0D6F854020368F4
:108470001B6898470328F6D194F89031062BF2D167
:10848000ECE705F108010FC902ACDFED0B0A84E847
:108490000F00002309480093B0EE600A1A462146F7
:1084A00002F0E6FE06B070BD20462946FFF7BAFF8F
:1084B0000120F7E7385C00200000000084810020E4
:1084C00038B5D1F8093007EE903AF5EEC07AF1EE02
:1084D00010FA05460C4605DD0B7A022B03D01ED997
:1084E000032B0ED038BD154B9FED150AD3F8900E17
:1084F00027EE800A7CF04EFDD4F80930C5F8D03163
:10850000F0E70E4B9FED0E0AD3F8900E27EE800A8F
:108510007CF050FDD4F80930C5F8D431E2E7074BC0
:108520009FED070AD3F8900E27EE800A7CF050FDED
:10853000D4F80930C5F8CC31D4E700BF386C00203E
:108540000000C84238B5114D0C4605F6247095F868
:108550009D1F5AF027F958B195F89D1F05F6247014
:108560005AF028F920B994ED040A0948F9F7E0FE19
:1085700094ED041AD4ED020A94ED030A95F89D1FB8
:108580000448BDE8384000225AF04CB9386C00204D
:10859000748500205C7B0020F0B50B69214F85B00D
:1085A00005460E460BB94B6953B300233B7006F1E9
:1085B00008030FCB6C4684E80F0021462846FFF7DE
:1085C000C1FB98B9184B0122D3F85C1E20460FF06E
:1085D00087FA4CF08FFF022215214CF0E7FE284667
:1085E000FDF71EFD114A02214FF08EF82146284664
:1085F000FEF79AFC38B90E48FBF798FE05B0F0BDBF
:108600003846FEF74FFEB38807EE903AF8EE677AE9
:1086100009212846C7ED017A05B0BDE8F040FEF714
:10862000CFBA00BFC4850020386C0020942D0D08FF
:10863000382C002010B5044C237813B1034867F0A0
:1086400019F9207810BD00BF80860020507C0020E2
:108650000078072894BF00200120704713B5094B0C
:1086600001910446D3F8900E03681B69984730B116
:108670000199204602B0BDE81040FEF74FBA02B0A3
:1086800010BD00BF386C002090F8983113F0010045
:1086900018BFC3F380007047094A034692F8E50605
:1086A00068B192F8E426043A012A07D85B6A1B688D
:1086B00093F8A100431E584258417047002070476C
:1086C000387C002010B5044686F02CFED4F8B0317A
:1086D000C01AD4F8AC3123EAE37398424FF000009B
:1086E00084BFC4F8AC01012010BD000010B50368C0
:1086F0000446DB6D9847D4F8AC3123EAE373984223
:108700004FF000003CBFC4F8AC01012010BD0000D8
:1087100008B504480321F9F743FDBDE808400148C6
:10872000F9F762BE7485002070B51C4B0446D3F87F
:10873000900E03681B690E469847054610B9002540
:10874000284670BDD4F894315BB986F0EBFDB4F8DF
:108750009231C4F8940123B1114A537843F00103D4
:10876000537086F0DFFDD4F89421B4F89231801A6A
:108770004FF47A72B0FBF2F09842E0D323B9084A82
:10878000537843F0010353702046FDF749FC3388CA
:10879000044A06214EF0B8FFD2E700BF386C002033
:1087A0005C870020402B0D0810B590F89031042B09
:1087B0000446164B0AD1D3F8900E03681B699847FC
:1087C00018B12046FEF7AAFC002010BD0A79D3F8A4
:1087D000983EDFED0F6A93ED0E6A07EE902A0A7E4F
:1087E000920748BF9FED0B7AF8EE677A48BF67EEB5
:1087F000877A86EE267AB0EEC77AB4EEE77AF1EEA3
:1088000010FAACBF01200020DFE700BF386C002069
:10881000DB0FC9400000803B13B5094B01910446B2
:10882000D3F8900E03681B69984730B10199204630
:1088300002B0BDE81040FEF771B902B010BD00BF34
:10884000386C002010B5044686F06CFDD4F8A831D1
:10885000C01AD4F8A43198424FF0000084BFC4F885
:10886000A401012010BD000038B505460C4686F075
:1088700059FDD5F8C831C01A23894FF47A72534391
:10888000984294BF0020012038BD0000C3681868DA
:1088900008B190F8B808704710B5012104460A489D
:1088A00004F030FD28B120460321BDE81040FEF75A
:1088B00087B94BF02BF9BDE8104040F26B124FF432
:1088C00080114BF0DBB800BFE082002090F89031BF
:1088D000022B04D0032B04D1034804F0E3BC012095
:1088E00070470020704700BFE082002038B50C4B75
:1088F000D3F8F05D90F89031032B044605F00405A1
:108900000AD1084804F0E6FC94F8903135B110B96A
:10891000023B5842584138BD0020F5E70120FAE7F4
:10892000384C0020E082002010B50F4A137843F045
:10893000800313700D4B93F94822002A044609DB8B
:10894000FEF73AFA70B920460822BDE81040092126
:10895000FDF738BABDE8104001220E21A3F1A000B6
:10896000F5F736BB10BD00BF5C870020385C0020E7
:10897000F8B5D0F8B44105465CB1012C1AD04BF0E3
:10898000C5F840F643024FF480114BF077F801240C
:1089900007E0184BD3F8900E03681B69984710B98D
:1089A00000242046F8BD2846FEF740FB0123C5F809
:1089B000B431F6E7104F97F94832002BF0DA436AEA
:1089C0001B6893F8A160012EEAD13C3027F0D2F960
:1089D00004460028E5D1D7F8783293F8CB3033B18C
:1089E00032460D21A7F1A000F5F7F2FAD9E7344697
:1089F000D7E700BF386C0020385C002038B56E4BDC
:108A0000D3F854226D4B9A4204460D4601D0002003
:108A100072E04B885E2B55D8512B0CD8103B9AB284
:108A20000F2A29D92046FDF7FBFA6B88644A0421F6
:108A30004EF06AFE59E0523B0C2BF3D801A252F8DB
:108A400023F000BF9B8B0108258A01085D8B01087C
:108A5000718B0108258A0108258A0108258A0108E9
:108A6000258A0108258A0108258A0108258A010826
:108A7000A18B0108798B01080F2BD3D801A252F8E2
:108A800023F000BF6B8B01080F8A0108818B01085E
:108A9000878B0108958B0108718B01085D8B01089C
:108AA000258A0108258A0108258A0108258A0108E6
:108AB000258A0108258A0108258A0108258A0108D6
:108AC0008D8B0108732B74D006D8702B6ED0722B4F
:108AD000A8D1FFF70BFE44E04AF2CF62934262D086
:108AE000A0D8B32B09D8B12B9CD92046FDF798FA12
:108AF000298853F001F8012038BDBC3B9AB2132AF3
:108B000090D8132B8ED801A252F823F0EB8A0108DB
:108B1000EB8A0108258A0108258A0108258A0108AF
:108B2000258A0108258A0108EB8A0108258A01089F
:108B3000EB8A0108258A0108258A0108258A01088F
:108B4000EB8A0108258A0108258A0108258A01087F
:108B5000EB8A0108258A0108EB8A01082046FFF705
:108B600069FD00283FF453AFBFE7FFF7DDFDF8E7ED
:108B70002046FFF7FDFEF4E71248FFF769FDF0E736
:108B8000FFF712FEEDE7FFF769FDEAE7BDE83840C1
:108B9000FFF77ABDFFF780FDE3E7FFF73DFEE0E773
:108BA000FFF750FEDDE7FFF75FFEDAE7FFF78AFD2C
:108BB000D7E7FFF7ADFDD4E7385C0020287D002023
:108BC000C82D0D08C485002090F89031032B0BD0E0
:108BD000062B06D0012B0AD1C368186803681B68EE
:108BE0001847044801F036BF034804F0E5BB0020F5
:108BF000704700BF84810020E08200208B88012B19
:108C000005D00B693BB94B692BB9CB681BB904483C
:108C10000021F9F7F9BE024800220831F9F716BF22
:108C2000382C002010B54B885E2B04460A464DD8E0
:108C3000512B05D8103B99B20F2921D900209DE076
:108C4000523B0C2BFAD801A151F823F0B78D010843
:108C50003D8C0108718D0108878D01083D8C01084C
:108C60003D8C01083D8C01083D8C01083D8C0108BC
:108C70003D8C01083D8C0108BF8D0108C78D01089E
:108C80000F2BDBD801A151F823F000BF7F8D010825
:108C9000918D0108998D0108A18D0108B18D010800
:108CA000878D0108718D01083D8C01083D8C0108FC
:108CB0003D8C01083D8C01083D8C01083D8C01086C
:108CC0003D8C01083D8C0108A98D0108B32B00F0F3
:108CD000848016D8732B7DD00ED8702B77D0722B52
:108CE000ACD1D1ED027A9FED447A67EE877AFDEE42
:108CF000E77AC0ED6B7A40E0B22B9FD1FFF7E0FB43
:108D00003BE0CD2B2CD8BB2B98D9BC3B112B95D855
:108D100001A151F823F000BF7B8D01087B8D010874
:108D20003D8C01083D8C01083D8C01083D8C0108FB
:108D30003D8C0108E18D01083D8C0108E18D0108A1
:108D40003D8C01083D8C01083D8C0108E18D010836
:108D50003D8C01083D8C01083D8C0108ED8D01081A
:108D60004AF2CF6293427FF469AFFFF727FB04E03A
:108D700002F108012046FEF745F8012010BD11461A
:108D8000FFF72CFAF9E711462046FFF78BF8F4E7D6
:108D90001146FFF7C7F8F0E71146FFF7FDF8ECE7DB
:108DA0001146FFF727F9E8E71146FFF72FF9E4E747
:108DB000FFF772FDE1E71146FFF758FADDE71146CC
:108DC000FFF7C2FAD9E71146FFF7E6FBD5E7FFF751
:108DD00015FBD2E7FFF726FBCFE7FFF70FFFCCE746
:108DE000064802F10801F9F7C3FAC6E71146204622
:108DF000FFF7A8FBC1E700BF0000C8427485002050
:108E000070470000704700007047000090F828008D
:108E100080F0010070470000024B436040F60503FC
:108E2000038170470001020490F85501704700006B
:108E30000F207047002070470020704700207047C7
:108E40000020704700487047742E0D080048704796
:108E5000802E0D0808B5094800F50053D3F8443EAC
:108E6000B3F9083000EE103AB8EEC00AF5F752FB3D
:108E7000BDE808400248FCF707BF00BF382C0020BF
:108E8000007F002010B514482DED028B1C4600F524
:108E9000005300F58040B3F94C34D0F8840E08EE4E
:108EA000103A036882B09B6ECDE900219847B8EE76
:108EB000C88AF0EE400ADDE90021B0EE480A074812
:108EC000FCF72EFB0548FCF741FF84ED000A02B0D9
:108ED000BDEC028B10BD00BF382C0020007F0020AD
:108EE000F8B51C4D05F5005405F580462846D6F822
:108EF0008C7EF5F7FDFAB4F9883401EE103AB4F936
:108F0000863400EE903A434200EE103AB8EEC11AB1
:108F1000F8EEE00AB8EEC00A384679F037FE284687
:108F2000D6F88C6EF5F7E4FAB4F9883401EE103A0D
:108F3000B4F9863400EE903A434200EE103A3046DF
:108F4000B8EEC11ABDE8F840F8EEE00AB8EEC00A83
:108F500079F096BE382C002038B5144C04F58045C5
:108F600004F58F54D5F8840E03689B6898476921EF
:108F700000F1940220464BF0A7FAD5F8840E03685E
:108F8000DB6898476A2100F1940220464BF09CFA76
:108F9000D5F8840E03681B6998476B2100F1940291
:108FA0002046BDE838404BF08FBA00BF382C002077
:108FB000014806F033BD00BF382C00203C3084F05F
:108FC0001DBD000008B54AF0A1FDBDE808407222B1
:108FD0004FF480114AF052BD08B54AF097FDBDE844
:108FE000084066224FF480114AF048BD08B54AF0A7
:108FF0008DFDBDE8084080224FF480114AF03EBD4F
:1090000073B51F4D0646D5F8540203681B6B98478D
:10901000044680B395F94932002B2FDBD5F878321E
:1090200093F8CB403CB395F8483203F0A003202BD3
:1090300024D1D5F8540203681B689847052808D046
:10904000D5F8540203681B689847A0F110035C42EE
:109050005C410C4A02F668630193A2F50053214675
:10906000D3F85C3F0093D2F88C3ED2F8842E304681
:1090700084F072FC0446204602B070BD0024FAE77A
:10908000385C0020386C00203C30FFF7B9BF00008E
:1090900038B5114D04461148F5F7E0FE95F9483210
:1090A000002B14DA236A93F8A120012A06D0D5F800
:1090B00054020021BDE83840FCF750BB0D21A5F15A
:1090C000A000F4F785FF95F94832002BEFDB20462E
:1090D000BDE8384084F07CBF385C0020382C00208C
:1090E0003C30FFF7D5BF00000120704701207047DA
:1090F000012070470120704707207047012070470A
:1091000000207047002070470120704700487047DA
:10911000C42F0D0800487047CC2F0D0870B52DEDF9
:10912000028B0025C36880F83C501B68DFED488A3D
:10913000D3ED0A0A42699FED478A93ED060AF4EEE1
:10914000E80A0446F1EE10FA88B01068B8BFF0EEF5
:10915000480A79F001FBE36862691B681068D3ED87
:109160000A0A93ED060AF4EEE80AF1EE10FAB8BF27
:10917000F0EE480A79F068FB636920461E68FCF748
:1091800053FF6368B3F93820B3F9363000EE903AF4
:10919000434201EE102A00EE103AB8EEC11AF8EE82
:1091A000E00AB8EEC00A304679F0F0FC6369204668
:1091B0001E68FCF739FF6368274CB3F93820B3F910
:1091C000363000EE903A434200EE103A01EE102A9B
:1091D0003046B8EEC11AF8EEE00AB8EEC00A79F0EF
:1091E0004FFDD4F8980E7BF0D3FBD4F8986E338BF8
:1091F0001B0723D504A80EF06DFC09F02FFC9FED92
:10920000170A044606F11C0023F0E6FF01AA04A990
:1092100020468DED010ACDED020A8DED031A09F00D
:10922000EBFB80B10322294604A80EF059FC0C4B3D
:10923000186804AA90F8791059F010FC0948082120
:10924000F8F7AEFF012008B0BDEC028B70BD00BF87
:109250000000003400007A43386C00200AD7233C19
:10926000D89000207485002030B52DED048BC368A4
:109270009FED898A1B684269D3ED0A7ADFED870A80
:1092800093ED060AF4EEC87AF1EE10FA0446A8BF90
:10929000F0EE670A106889B079F05EFA63692046DB
:1092A0001D68FCF7C1FE6368B3F93820B3F93630A6
:1092B00000EE903A434200EE103A01EE102A2846A2
:1092C000774DB8EEC11AF8EEE00AB8EEC00A79F0B0
:1092D0005DFCD5F8980E7BF09DFCA5F5805393F8C6
:1092E0006D32D90747D4D5F8983E1A8BD20742D5AC
:1092F00093ED0A9AB4EEC89AF1EE10FAB8BF93ED66
:10930000049AE36A186856F013FFD5F8903ED3ED3F
:10931000067AA36B20EE270AD3ED007AF0EE498A95
:10932000E0EE278AB0EE490AF5EEC08AF1EE10FAB7
:10933000D8BFDFED5C8AF0EE680A20F0C9FB28B9DF
:10934000D5F8980EB0EE680A7BF0E2F9636893F9FD
:109350005130272B0FD0A36A186856F0E9FEF0EEC3
:10936000C07AF4EEC87AF1EE10FAB0EE407A20D569
:10937000002384F83C30236B1B68B3F9083000EEFF
:10938000103A2046B8EEC00AFCF710FD2046FCF764
:109390007BFC2046B0EE408AFCF7A8F9002848D0B4
:1093A0000021204609B0BDEC048BBDE83040FCF73D
:1093B000D5B9D5F8983E9FED3C0AD3ED0F7AD3EDA1
:1093C0000B6AA36B27EE800AF4EEC86AD3ED007A2D
:1093D000F1EE10FA67EE277A10DB9FED341ADFED1D
:1093E000310A552037EE800A20F076FC012384F8FC
:1093F0003C30D5F8980E7BF07BF9BCE79FED2C7ADA
:10940000F4EEC76AF1EE10FA05D89FED261ADFEDEB
:10941000290A5920E6E7F0EEE66AF4EEC86AF1EEB2
:1094200010FAE3D594F83C30002B08BFB0EE670A81
:10943000DCE7636A022118687DF09EFF1E4806F093
:10944000A3F9B0EE480AD5F8980E7BF0E5FA01468C
:109450001A48FAF767FE636918687AF07DFF236A95
:109460001D686369186879F0B5FD05AC204614499C
:109470008DED020ACDED030A8DED041AF9F786F899
:10948000079B009394E80C0002A9284676F06EFE34
:1094900009B0BDEC048B30BD0000003400007A43FD
:1094A000386C002000000000E02E65420000B4424D
:1094B000000000B40000B4C2205B0020382C002063
:1094C0007485002008B5064BD3F8983ED868243040
:1094D00023F0CEFBFCEEC07A17EE900A08BD00BF69
:1094E000386C0020024BD3F8983ED86879F01CBE47
:1094F000386C00200B207047012070470020704717
:1095000001207047002070470048704764300D0804
:10951000004870476C300D080120704708B5DFED3A
:10952000237AF4EEE70AF1EE10FA2DED028BF0EE5D
:10953000408AB0EE608A35DDDFED1D7AF4EEE70A91
:10954000F1EE10FA2ED5F6EE007A70EEE77ADFED46
:10955000196A9FED190ADFED190AF0EEE77A87EE36
:10956000A67A8720B7EE001A30EE470A20F0B4FB47
:10957000DFED137A9FED131ADFED130A20EE270AB1
:109580008A2020EE280A20F0A7FB30EE080ABDEC66
:10959000028BDFED0A0ABDE808408D20B7EE001A05
:1095A00020F09ABB9FED050AEFE700BFAC1C5A3EC6
:1095B000D578493F8FC2753E9A99993F00000000C7
:1095C000FAEDEBBA9A99993E9A9999BE30B52DED7C
:1095D000048B7D4BB3F94C3400EE903AF8EEE00A80
:1095E00083B0044601AA6946B0EE600AFBF798FF13
:1095F000A0697CF009FFE369D0ED008AD3ED946A9D
:10960000D3ED977A90ED016AA3689FED701ADFEDB4
:10961000700A27EEE80A68EEA68A03F6F803E6EE7B
:10962000278A05463B20DFED6B7AB0EEE87AB4EE90
:10963000E77AF1EE10FA58BFB0EE677ADFED667A9E
:10964000C7EE275AF7EE007A77EEE57A9DED007ABD
:1096500067EE877A93ED007A67EE877A9FED5F7AFF
:10966000A6EE260A87EE879A20F036FB3C209FED77
:10967000571ADFED570AB0EE408AB0EE680A20F0C4
:109680002BFB626B564B1268DFED567AB2F908205D
:10969000D3ED006A9FED541ADFED540A07EE102A4D
:1096A000B8EEC77AF0EE408A27EE277ADFED507ADF
:1096B000A6EEA77A4520F4EE007AA7EE678ABAEE06
:1096C000000A28EE000A83ED007A8DED000A20F0F2
:1096D00003FBDDED017A9FED477A474B8DED000AE4
:1096E000F0EEE77AF4EEC77AF1EE10FA51D593ED89
:1096F000007ADFED427A77EE277AB2EE007AF4EE66
:10970000C77AF1EE10FA58BFF0EE477AC3ED007A4F
:1097100067EEA87ACDED017A636A186890F8CB10ED
:10972000002939D17DF028FE636A1B6893F8A110E7
:10973000012939D0032940D039B9236A186877F054
:10974000FDF9236A186876F049FC236ADDED010A09
:1097500018689DED000A0368B0EE491ADB6A984765
:10976000204695ED028AFCF7D7F82046F0EE400A35
:10977000B0EE480AFFF7D2FE236A62681868D2ED9D
:10978000020A036801215B6E984703B0BDEC048BAD
:1097900030BD00221A60BFE7194B93F94932002B04
:1097A000B4BF01210221BDE7236A186877F0C6F92A
:1097B000236A186876F028FCC7E7D9790029C4D154
:1097C0002046FCF727FCC0E7384C002000000C4482
:1097D00000000CC40000FA4400409C4500003442E4
:1097E000E08500200AD7233D00A08C4500A08CC551
:1097F0008FC2753F00000034E48500208FC2F53C25
:10980000385C002016207047002070470020704709
:10981000012070470020704781F001007047000070
:10982000012070470048704704310D080048704718
:109830001B130D0803681BB1007900F0010070478D
:1098400018467047F0B5494D95F99D6F85B00446AF
:10985000A5F50055002E00F085804548FFF7EAFF8A
:10986000064600287ED0636920461F68FCF7DCFBB3
:109870006368B3F93820B3F9363000EE903A4342CA
:1098800001EE102A00EE103AB8EEC11AF8EEE00A26
:10989000B8EEC00A384679F079F9636920461F6846
:1098A000FCF7C2FB6368B3F93820B3F9363000EE39
:1098B000903A434200EE103A01EE102A3846B8EED4
:1098C000C11AF8EEE00AB8EEC00A79F0D9F905F548
:1098D0008043D3F88C0E79F06DFA18B96369186873
:1098E0007AF0ECFBB5F9A43004F13C001BB9B5F8F3
:1098F000A230A5F8A430B5F8A43007EE903AF8EEFF
:10990000677A04F1980203A90027CDED037A4DF0A0
:10991000B7FA04F15C00C4F8A07001906DF068FB28
:10992000002384F8A530B5F9A43001981BB9B5F827
:10993000A230A5F8A430B5F8A43007EE903AF8EEBE
:10994000E77AB7EE000A80EE270A6DF075FB09484A
:109950007CF056FDC4F8C870DFED077A20EE270AC8
:1099600084ED310A304605B0F0BD00BF384C002010
:10997000D05B0020A07A00200AD7233C10B5044613
:10998000FBF79CFC2046154B40F83C3B4DF004FA9D
:10999000134B2365134B9FED142A9FED141ADFED33
:1099A000140A9FED140A6365F1EE041A04F15C00D9
:1099B0006DF058FB002320460F49C4F8A830C4F8C6
:1099C000AC30C4F8B030C4F8B430C4F8B830C4F81F
:1099D000BC3042F003FF204610BD00BF0C320D0822
:1099E000CDCCCC3D000040400AD7233B00803B4516
:1099F0009A99993ECDCC4C3EA4310D082DE9F04307
:109A00002DED028B9BB0914604460D4685F08AFCF5
:109A1000B8499FEDB98A0646A1F1080023F05AF82B
:109A200094ED161ACDED110A7E20F1EE410A8DED6E
:109A3000100A20F051F994ED161A8DED100AF1EE8E
:109A4000410A7F209DED110A20F046F910A904F18A
:109A50003C008DED110A4DF031FAA848CDED130A06
:109A60008DED120A7CF0CCFCD4ED327AD4ED140AE0
:109A700094ED151AE0EE087A892004F15C074FF0A6
:109A80000008B0EE670A20F027F912A823F06EF85C
:109A90009B4812A909F034FA14A938468DED140A2E
:109AA000CDED150A6DF084F93846CDF85880CDF823
:109AB0005C806DF0C1F98DED160ACDED170AB9F194
:109AC000000F00F001810123C4F8D06084F8CC308D
:109AD0008C4E04F1A80116A823F024F8B6F94C34F2
:109AE00000EE103A16A8B8EEC00A23F03FF816A907
:109AF000A6F6184009F0F0F918A928468DED180AC5
:109B0000CDED190A23F00EF8B6F94C3495ED007A34
:109B100007EE903AF8EEE77AB0EEC77AB4EEE77A5D
:109B2000F1EE10FA00F3CE8095ED017AB0EEC77A2F
:109B3000F4EEC77AF1EE10FA4CBF0123002384F84B
:109B4000A530B6F94C3495ED000A5A4207EE903A2A
:109B500000EE902AB8EEE71AF8EEE00ACA2020F0EC
:109B6000BBF885ED000AB6F94C3495ED010A5A426E
:109B700000EE902A07EE903AF8EEE00AB8EEE71A07
:109B8000CB2020F0A9F885ED010A94F8A4305A1CE6
:109B900084F8A4201422B3FBF2F102FB1133DBB2F0
:109BA000002B34D14BF0A6FC064685F0C3FB804663
:109BB000D4F8AC000F46F2F7A7FCCDE90E01D4F8BB
:109BC000A800F2F7A1FCCDE90C01D4F8A000F2F74F
:109BD0009BFCCDE90A016868F2F796FCCDE9080123
:109BE0002868F2F791FCCDE906011398F2F78CFC96
:109BF000CDE904011298F2F787FCCDE90087CDE9A1
:109C00000201414B414A424930464BF0E9F91BB051
:109C1000BDEC028BBDE8F08312A823F029F8DFED3C
:109C20003D7AB4EEE70AF1EE10FA57D494F8CC304E
:109C300063B956E038466DF05FF994F8CC3084EDA6
:109C40002A0AC4ED2B0A002B3FF442AFDFED325A53
:109C5000DFED324A9FED324ADFED323A12AA2B464F
:109C600005F10801B2EE0E5AB7EE003AB2EC016A05
:109C700094F99D00B0EEC67A67EE256A07EE900A69
:109C800076EE842AF8EEE77AB0EE647AA7EE857A6B
:109C9000C3EEA27A27EE087A77EE837A27EE267A49
:109CA000B5EEC06A67EE877AF1EE10FA48BFF1EEC2
:109CB000677AE3EC017A9942D8D1CDF85C80CDF88F
:109CC000588005E701233AE794F8CC304BB1D4F83B
:109CD000D00040F6B833361A9E429DD9002384F84E
:109CE000CC3094F8A530002BA4D138466DF06AF939
:109CF000A3E700BFFC5B00200AD7233CA07A00202A
:109D000020400020384C0020F4FD0C0810310D08D4
:109D10001B130D089A99993E0000C8420000BE42EC
:109D2000000070420000FA432DE9F04F2DED048B46
:109D30000446A5B0BD487CF063FBBD4BDFEDBD7AAA
:109D40001B68DB6A93F89C3060EE278A33B9F1EE2A
:109D5000687AC4ED327AC4ED318A47E0B64D05F534
:109D60004053D3F8783293F8A090B9F1020FEED1B6
:109D700085F0D8FA05F58043D3F89C3EC01A40F22E
:109D8000DB539842E3D99FEDAD8A95F8B41D8DED74
:109D9000218A18AB21AA05F6C8008DED228A8DED27
:109DA000238A1EF03DF908B3A54821A921F094F8B3
:109DB000D4ED2C7A8DED210A37EE800AD4ED2D7A80
:109DC000CDED220A77EEA00A9E4884ED2C0AC4ED60
:109DD0002D0A8DED231AFFF72DFD60B985F0A2FA4B
:109DE00084ED2D8AC4F8C00084ED2C8A25B0BDEC2A
:109DF000048BBDE8F08F05F5005BD4F8C020DBF8DC
:109E0000CC3F42B9C4F8C03084ED2D8A84ED2C8A51
:109E100084ED328AEAE79A42E8D08B4804F1B00137
:109E200009F05AF889498DED190AF1EE607AA1F12D
:109E3000080010EE108A17EE907ACDED1A0ACDEDDB
:109E40001B7A8DED1C0A22F045FEDBF8CC3FD4F8DE
:109E5000C0208DED1D0AA3EB020ABAF5FA7FCDED05
:109E60001E0A04F1B8051DAE0CD996E80300C4F82B
:109E7000C03084ED2D8A84ED2C8A85E80300C4ED82
:109E8000318AC5E72946304622F024FE96E80300D1
:109E900085E8030094ED329ADBF8CC3F9FED6C6AC5
:109EA000C4F8C03039EE285A8DED1F0ACDED200AD6
:109EB0001FA91BAA0023F0EE489AF1EC017AF0EEFC
:109EC000E76AF4EEC66AF1EE10FA1FD4D2ED005A3A
:109ED000B0EEE57AB4EEC67AF1EE10FA16D485EE5D
:109EE000A77AB5EEC07AF1EE10FA0FD907EE903AE4
:109EF000F8EEE77A37EE457A77EEA67AE7EE269A1D
:109F0000FCEEE77ACDED177A9DF85C30B9F1010FE0
:109F100002F1040240F087802BB107EE903AF8EE90
:109F2000E77AC9EEA79A4FF4EC70F5EEC09AF1EE1D
:109F300010FA48BF79EEA99AB5EE001AFDEE000AB4
:109F4000B0EE690A1FF0C8FE39EE009A9FED410A93
:109F500094ED327ADFED407A29EE009AA7EE279A47
:109F6000D4ED147A84ED329A39EE289AB4EEE79A59
:109F7000F1EE10FA44BF77EEE87AC4ED327A94ED50
:109F8000329A4BF0B7FA054685F0D4F98146D4F8F9
:109F9000C400CDF850A00E46F2F7B6FACDE9120192
:109FA00018EE900AF2F7B0FACDE91001D4F8C80023
:109FB000F2F7AAFACDE90E0119EE900AF2F7A4FA27
:109FC00038EE899ACDE90C0119EE100AF2F79CFAE5
:109FD000CDE90A014046F2F797FACDE90801384683
:109FE000F2F792FACDE906012098F2F78DFACDE961
:109FF00004011F98F2F788FA184B194ACDE90201BB
:10A00000CDE90096174928464AF0EAFF2046FCF7BA
:10A0100007F81549B0EE490A4DF002FE84ED2D8A8D
:10A0200084ED2C8A97E64FF0010946E7A07A0020DC
:10A03000688500200AD7233C382C0020000000004F
:10A0400040430020D05B002020400020FC5B00202B
:10A050000AD7233DCDCC4C3ECDCC4C3F30310D0802
:10A060003C310D0873310D0878310D082DE9F041B0
:10A070002DED048B044688B0FFF756FE6369204639
:10A080001D68FBF7D1FF6368B3F93820B3F93630A8
:10A0900000EE903A434200EE103A01EE102AF8EE3C
:10A0A000E00AB8EEC11AB8EEC00A284678F06EFD94
:10A0B00004F13C052046FBF77FFE28464CF0FAFEF3
:10A0C000D4ED260A1FF004FDB74BA0B9B3F9A420C4
:10A0D0001AB9B3F8A220A3F8A420B3F8A43007EE6D
:10A0E000903AF8EE677A04F1980206A92846CDED79
:10A0F000067A4CF0C5FEAD4DDFEDAD8AD5F8443E95
:10A10000B3F9083000EE103AA5F50050B8EEC00AD9
:10A11000F4F700FA2046B0EE408A8DED030AFBF713
:10A1200083FFB5F9863401EE103A434200EE903ACF
:10A13000B8EEC11AF8EEE00AF820B0EE480A1FF0B7
:10A14000CBFD20468DED030AFBF700FE2046B0EE66
:10A15000409A9DED030AFBF7B3FD074605F698709C
:10A16000FFF768FBD8B195F8B83F9FED927AD4ED30
:10A17000286A07EE903AF8EEE77A67EE877A9FED65
:10A180008E7AE6EE877A8D4EC4ED287A042F22D897
:10A19000DFE817F00800BF00E200E700F200F0EE91
:10A1A000687AF0E7864B0021D3F878027DF0E4F876
:10A1B000D6F8840E75F012FFD6F8840E012176F0E1
:10A1C000BDFCD6F88C0E9FED7A0A7AF053F804F1B4
:10A1D0005C006CF00DFFD5F83C3ECDED048AB3F980
:10A1E0000880D5F8403ECDED058AB3F90870B5F981
:10A1F0004C3408EE103A236A186803689B6E98473F
:10A20000B8EEC88AF0EE400A05AAB0EE480A04A9E2
:10A210002046FBF785F994F99C3094ED287A07EEF7
:10A22000903AF8EEE77AF1EE489AB4EEE77AF1EE7A
:10A2300010FA37DB85F076F8D6F89C3EC01A40F667
:10A24000B83398422ED958EA070306A914BF012251
:10A2500000222046CDED068ACDED078AFFF7CEFB22
:10A26000F6EE007A69EEA70A28EE271A4FF4A570D9
:10A270009DED060A8DED011ACDED000A1FF02CFDB3
:10A2800040F24B108DED060A9DED011ADDED000A3E
:10A290009DED070A1FF020FD06A904A88DED070A11
:10A2A00022F040FCB0EE481AF0EE690A9DED040A77
:10A2B0004FF4A7701FF010FDB0EE481AF0EE690AD7
:10A2C0008DED040A40F24F109DED050A1FF004FDCC
:10A2D000B5F94C348DED050A00EE103A05AA04A933
:10A2E000B8EEC00A374863F003FDD6F8840EDDED02
:10A2F000050A03689DED040ADB6AB0EE491A984727
:10A30000636918687AF028F808B0BDEC048BBDE8E2
:10A31000F0812B4B2C4FD3F8780202217DF02CF8E2
:10A320003B786BB963689FED291ADFED210A93ED45
:10A33000040A4FF48C701FF0CFFC384605F034FF50
:10A3400020469DED030AFBF79FFC1F488DED030A95
:10A3500003A905F063FF3EE7236A0121186876F040
:10A36000EDFB236A186875F04FFE63699FED100AD4
:10A37000186879F07FFF2EE7114F0221D7F8780295
:10A380007CF0FAFF20469DED030AFBF77DFCA7F564
:10A390008C708DED030A05F0F7F963699DED030AF2
:10A3A000186878F079FC16E7382C0020384C00202B
:10A3B00000000000D0CC4C3D3333733F386C00209C
:10A3C000385C0020E07B00209C86002000007A445E
:10A3D0001720704701207047002070470020704709
:10A3E000012070470048704794320D0800487047BC
:10A3F00020130D0883689FED067A03F63803D3ED2A
